:100000005555AAAAF20300000000000000000000FD
:100010006284010000000000000000005F08162A52
:10002000002810002D110000590200006F0200008E
:10003000850200009B020000B102000000000000E9
:10004000000000000000000000000000DD280000AB
:10005000ED28000000000000EF280000FF2800004D
:1000600003290000272700001D2900006127000048
:100070001F29000023290000332900004329000024
:10008000C702000061290000632900006529000003
:1000900067290000692900006B29000000000000AA
:1000A0000000000000000000000000000000000050
:1000B0000000000000000000000000000000000040
:1000C0000000000000000000000000000000000030
:1000D0000000000000000000000000000000000020
:1000E000F203000000F002F800F062F80AA090E8C5
:1000F000000C82448344AAF10107DA4501D100F0E3
:1001000057F8AFF2090EBAE80F0013F0010F18BF4D
:10011000FB1A43F001031847C4F50000E4F50000A2
:100120000A444FF0000C10F8013B13F0070408BF1D
:1001300010F8014B1D1108BF10F8015B641E05D0BB
:1001400010F8016B641E01F8016BF9D113F0080F70
:100150001EBF10F8014BAD1C0C1B09D16D1E58BF02
:1001600001F801CBFAD505E014F8016B01F8016B39
:100170006D1EF9D59142D6D37047000000230024AC
:1001800000250026103A28BF78C1FBD8520728BFA7
:1001900030C148BF0B6070471FB5024802490FF0DD
:1001A0009FF81FBD000810000028100010B510BDFA
:1001B000DFF80CD0FFF7F0FF02F0E4FC0FF091F94C
:1001C0000028100003B4FFF7F1FF03BC0FF0BCF9E7
:1001D0001A4B19680868B0E8F00F80F309884FF0EF
:1001E000000080F311884EF00D0E704700000000F3
:1001F00003480068006880F3088862B600DF00BF2B
:1002000008ED00E0EFF309800C4B1A6820E9F00FCD
:10021000106008B54FF0200080F3118800F02FFD2A
:100220004FF0000080F31188BDE8084019680868A5
:10023000B0E8F00F80F30988704700BF0428100071
:1002400001B44FF0200080F3118801BC704701B465
:100250004FF0000080F3118801BC704740BA70472E
:10026000C0BA7047401E0028FCDC704700BE7047D3
:1002700040BA7047C0BA70471EF0040F0CBFEFF3CE
:100280000880EFF309804FF0010102F094BA1EF0EC
:10029000040F0CBFEFF30880EFF309804FF0020169
:1002A00002F089BA1EF0040F0CBFEFF30880EFF3E1
:1002B00009804FF0030102F07EBA1EF0040F0CBF5C
:1002C000EFF30880EFF309804FF0040102F073BAF6
:1002D0001EF0040F0CBFEFF30880EFF309804FF01E
:1002E000050102F068BA1EF0040F0CBFEFF308809E
:1002F000EFF309804FF0000102F05DBA10B504463B
:1003000000F029FC20460EF091FE044600F0BAFBF6
:10031000204610BD10B5040008D000F01CFC20469B
:100320000EF0B3FEBDE8104000F0ACBB10BD00F114
:1003300008014FF0FF32C0E90112C16001610021E4
:1003400001607047002101617047426853684B604B
:1003500043688B605368996051604160086101682F
:10036000491C0160704710B50B685A1C02D000F19F
:10037000080202E0026904E05268546824689C4262
:10038000FAD953684B6099608A60516008610168CE
:10039000491C016010BDD0E901128A60D0E9011248
:1003A000516001694A68824201D182684A60002234
:1003B00002610868401E08607047000010B5031F06
:1003C0004FF0807420381C6081610021416140F849
:1003D000202910BD1D4810B5016841F47F0101605E
:1003E000016841F07F4101604FF0E0201849416110
:1003F00007210161174900200860FFF7F9FE00207E
:1004000010BD704711494FF080501C39086070478B
:1004100010B5FFF715FF0F480168491C016010BDBA
:100420000C490868401E086001D1FFF710BF7047F3
:10043000064910B51C394FF080500860FFF700FFE7
:1004400000F0D5FABDE81040FFF701BF20ED00E055
:1004500098990300002810002DE9F0410E46050090
:100460004FF000072AD05020FFF748FF040025D0A6
:10047000B84605FB06F0401CC4F84C80FFF73EFF71
:100480002060C0B105FB0601C4F838806160A0603F
:10049000691E01FB0600E563E060781EC4E9106098
:1004A000A06404F11000FFF742FF04F12400FFF7FD
:1004B0003EFF274602E02046FFF72CFF3846BDE806
:1004C000F08170B50446FFF7A3FF04F12405A06C8A
:1004D0000AE0606A50B1284600F0E6FC08B100F07E
:1004E00035FDA06C401EA0640028F2DC4FF0FF3602
:1004F000A664FFF795FFFFF78BFF04F11005606C12
:100500000AE0206950B1284600F0CEFC08B100F0A6
:100510001DFD606C401E60640028F2DC6664BDE86E
:100520007040FFF77DBF10B51346026C04466AB1F8
:1005300083B1E0680EF0F4FDE168206C091AE16017
:100540002268914202D26168081AE060A06B401CE8
:10055000A06310BDA0680EF0E3FD216CA068084404
:10056000A06061688842F1D32068A060EEE72DE9C1
:10057000FF41002582B01F46884604464FEA050623
:10058000FFF746FFA16BE06B814213D23A4641462A
:100590002046FFF7C8FF606A38B104F1240000F07C
:1005A00083FC012801D1FFF72DFFFFF739FF012060
:1005B00006B084E7049808B11DB106E0FFF730FFEC
:1005C0001DE0684600F098FC0125FFF729FF00F0C8
:1005D000C2FAFFF71DFF606C401C00D16664A06C7E
:1005E000401C00D1A664FFF71BFF04A9684600F079
:1005F00089FC30B12046FFF764FF00F043FA002089
:10060000D6E7FFF705FFA06BE16B884210D1FFF73B
:1006100007FF04F11000049900F02DFC2046FFF7BD
:1006200050FF00F02FFA0028AAD1FFF7EBFEA7E752
:10063000FFF7F6FE2046FFF744FF00F023FA9FE79E
:10064000944AC16C1268914201D000207047002387
:100650001A4619468BE72DE9F0411E4615460F460E
:100660000446FFF7EDFDA06BE16B884217D23246DE
:1006700039462046FFF757FFA06C411C03D0401CB1
:10068000A06401240CE0606A0028FAD004F1240080
:1006900000F00AFC0028F4D001202860F1E70024D3
:1006A000FFF7D5FD20460AE730B403680D46002B5E
:1006B0000CD0026CC1688C18C46041688C4200D3B5
:1006C000C360C168284630BC0EF02ABD30BC7047FC
:1006D0002DE9FF43002683B09846894604463746F5
:1006E00000F12405FFF794FEA06B30B36948E6687B
:1006F0000068E06449462046FFF7D6FFB8F1000FD6
:100700000ED0E660606A28B1284600F0CDFB08B143
:10071000FFF778FEFFF784FE012007B0BDE8F08305
:10072000A06B401EA06320690028F3D004F11000E4
:1007300000F0BAFB0128EBD0ECE7059808B11EB138
:1007400006E0FFF76DFE1DE0684600F0D5FB0126D0
:10075000FFF766FE00F0FFF9FFF75AFE606C401CE1
:1007600000D16764A06C401C00D1A764FFF758FE5D
:1007700005A9684600F0C6FB30B12046FFF7A1FE90
:1007800000F080F90020C8E7FFF742FEA06B38B107
:10079000FFF746FE2046FFF794FE00F073F9A1E74D
:1007A000FFF73EFE2846059900F065FB2046FFF75F
:1007B00088FE00F067F9002894D1FFF723FE91E747
:1007C00070B515460E460446FFF73AFDA06BC8B15A
:1007D00031462046FFF768FFA06B401EA063606CA7
:1007E000411C03D0401C606401240CE020690028F7
:1007F000FAD004F1100000F057FB0028F4D00120DB
:100800002860F1E70024FFF722FD204670BD10B5F7
:100810000446FFF7FDFDA46BFFF702FE204610BD66
:10082000806B704710B504461B48002100EBC102E5
:100830005368A34203D1002240F8312002E0491C52
:100840000A29F3D32068FFF765FD2046BDE8104074
:10085000FFF760BD806B08B1002070470120704732
:10086000816BC06B814201D101207047002070472D
:1008700010B5094B002200BF53F832401CB1521C86
:100880000A2AF9D310BD43F8321003EBC2014860C5
:1008900010BD000004281000982A10002DE9F05F18
:1008A0008346DDE90A6815469A46894648200C9F2A
:1008B000FFF724FD04004AD01FB9A800FFF71EFD72
:1008C0000746676338003FD0A900A5220EF06DFCF3
:1008D0006FF0030101EB8501606B3546084420F0A1
:1008E00007074946102204F138000EF0AFFC002043
:1008F00084F847000F2D00D30E25E5622086608620
:10090000201DFFF71FFD04F11800FFF71BFDC5F1C7
:100910000F012461A1615246594638466462FFF7CF
:100920004DFD2060B8F1000F01D0C8F80040FFF77E
:100930006FFDFB4D6868401C68602868DFF8E48341
:1009400040B1686968B331E02046FFF7E3FC4FF03F
:10095000FF3449E02C606868012827D15FF0000768
:1009600007EB870108EB8100FFF7E1FC7F1C0F2FED
:10097000F6D3ED48FFF7DBFCEB481430FFF7D7FC6C
:10098000E9482830FFF7D3FCE7483C30FFF7CFFCBD
:10099000E5485030FFF7CBFCE34828631430686328
:1009A00004E02868C06AB04200D82C60E06AE968B8
:1009B000884200D9E860A96A491CA962296988426D
:1009C00000D9286100EB800108EB8100211DFFF7B1
:1009D000BCFC0124FFF724FD686928B12868C06ABF
:1009E000B04201D2FFF70EFD2046BDE8F09F2DE991
:1009F000F041CB4CA06920B1E069401CE061BDE84A
:100A0000F081A068401CA060A0684FF0FF3570B96D
:100A1000206B616B21636063606A401C6062206BC5
:100A20000068A8B1206BC068C0684068E062A06838
:100A3000E16A8842E3D3BB4F206B006850B1206B62
:100A4000C068C668A1687068814205D2E062D6E7D6
:100A5000E562ECE7E562D2E7301DFFF79CFCB06A87
:100A600018B106F11800FFF796FCF06A2169884278
:100A700000D9206100EB800007EB8000311DFFF7FB
:100A800064FCD9E72DE9F0470026FFF7C1FCA44C30
:100A9000A069401EA061A069A8BB606898B3DFF898
:100AA0008882002508F12808DFF878921AE0C068EB
:100AB000C76807F11800FFF76EFC381DFFF76BFCE5
:100AC000F86A2169884200D9206100EB800109EBB6
:100AD0008100391DFFF739FCF86A2168C96A88422C
:100AE00000D30125D8F8001040460029DFD1E06985
:100AF00028B909E0FFF77BFFE069401EE061E0698B
:100B00000028F7D105E009E0012D02D0206A012874
:100B100004D1002001262062FFF774FCFFF780FC5F
:100B20003046BDE8F08770B57D4C054620684560CD
:100B3000A0682168854201F1040104D2606BBDE820
:100B40007040FFF710BC206BFFF70DFCE06A854298
:100B500000D2E56270BD72488169491C81617047AD
:100B600010B50B460246FFF7F6FF10686C49C41833
:100B70008B68984205D9A0420ED98868844202D871
:100B80000AE0A042F9D914600868001DFFF703FCD1
:100B90002046FFF7C8FF00E01460FFF773FF00284E
:100BA00003D1BDE81040FFF72DBC10BD10B5020009
:100BB0000FD0FFF7D0FF5A48816800688C18001DDD
:100BC000FFF7E9FB2046FFF7AEFFFFF75BFF0028CA
:100BD00003D1BDE81040FFF715BC10BD10B50446A9
:100BE000FFF716FC0CB94E480468E46AFFF718FCDE
:100BF000204610BD2DE9F04100270D4606460F297D
:100C000000D30E25FFF704FCDFF81481D8F80000AC
:100C1000864201D1002608E03EB13446E06AA8428F
:100C200029D0854204D926B904E0D8F80040F5E778
:100C300006B90127C5F10F01E562A161394D00EB4D
:100C40008000616905EB8000814210D1201DFFF713
:100C5000A2FBE06AD8F810204146904200D9086112
:100C600000EB800005EB8000211DFFF76EFB012FDC
:100C700001D1FFF7C7FBBDE8F041FFF7D1BB284822
:100C80008269284922B1012101627047521E026126
:100C9000026902EB820251F82220002A0269F5D093
:100CA00002EB820201EB82014A68526801F10803FB
:100CB0004A609A4201D152684A60D1680160704727
:100CC00070B50646FFF7A4FB154D2868864201D192
:100CD000002619E0C6B13446201DFFF75CFBA06A70
:100CE00018B104F11800FFF756FB0F48211D3C30E6
:100CF000FFF72BFBFFF794FB002E0FD1686928B19B
:100D0000BDE87040FFF77EBB2C68E5E706483C3045
:100D100000686968884209D10020286070BD000021
:100D200004281000E82A1000142C1000BDE87040C0
:100D3000A5E7F04B426900219A4206D1806AA3F1EF
:100D40001402904201D000B901210846704770B5E5
:100D50000400E3D0E84D28688442DFD0FFF758FB59
:100D60002046FFF7E6FF012816D1201DFFF713FBF1
:100D7000E06A2969884200D92861E04900EB8000D7
:100D800001EB8000211DFFF7E0FAE06A2968C96ADB
:100D9000884201D3FFF736FBBDE87040FFF740BB48
:100DA000BCE770B500260446FFF7C3FF01281FD13A
:100DB000D14DA86920B1CF4804F11801143815E0CD
:100DC000E06A2968C96A884201D3012600E000264A
:100DD000201DFFF7E0FAE06A2969884200D92861FE
:100DE000C64900EB800001EB8000211DFFF7ADFA42
:100DF000304693E7C14C2068012801D9FFF702FB78
:100E00000DF058FDF7E71FB50024009401940294FB
:100E100023464022BAA1BC480394FFF73FFD0128B6
:100E200009D1FFF70DFAB448012141618460BDE8A2
:100E30001F40FFF7CFBA1FBD10B5FFF701FAAE494B
:100E400000204861BDE81040FFF7DBBA10B5FFF79E
:100E5000DFFAA9488468FFF7E3FA204610BD10B511
:100E6000FFF7EEF9A4488468FFF7F1F9204610BDBA
:100E7000A1484068704770B59F4D0C4629681831ED
:100E8000FFF771FA2868001DFFF785FA601C04D08F
:100E9000A8682044BDE8704045E62968BDE8704078
:100EA000091D9448FFF751BA70B5C068C46804F1D1
:100EB00018000646FFF76FFA8F4DA86918B18D48E4
:100EC000314614380DE0201DFFF765FAE06A296904
:100ED000884200D92861894900EB800001EB80003D
:100EE000211DFFF732FAE06A2968C96A884201D3F6
:100EF000012013E7002011E77F494A6A02608968F0
:100F00004160704770B50D460446FFF781FA2868C6
:100F1000411C14D0784A2168536A994203D0616811
:100F2000936899420DD9616893685B1A834208D22D
:100F30009268511A401A28602046FFF7DDFF00240E
:100F400000E00124FFF76CFA2046E7E66A49012039
:100F5000086270476848006870476748416919B17E
:100F6000806918B102207047002070470120704747
:100F700070B5614D064639B14FEA0104FFF748FAF2
:100F8000208E304211D101E02C68F7E7201DFFF7D9
:100F900002FAA06A18B104F11800FFF7FCF95548ED
:100FA000211D1430FFF7D1F96686FFF739FA686919
:100FB00018B1BDE87040FFF725BA6868012802D073
:100FC000BDE870405BE600202860A7E670B50546E6
:100FD00009B9494801680C46FFF71AFA608EA84320
:100FE0006086208EA8432086BDE87040FFF718BABF
:100FF000404B4269002114339A4206D1806AA3F122
:101000002802904201D000B901210846704770B50E
:1010100006460C002BD0384D2868844227D0FFF7B5
:10102000F7F9208E30432086608E30421BD0204658
:10103000FFF7DEFF012816D1201DFFF7ACF9E06AAB
:101040002969884200D928612C4900EB800001EB16
:101050008000211DFFF779F9E06A2968C96A884292
:1010600001D3FFF7CFF9BDE87040FFF7D9B955E6D6
:1010700070B5002605460C000DD0FFF7E1F8208E74
:1010800028432086608E284227D02046FFF7B0FFF5
:10109000012802D021E0304640E6174DA86920B172
:1010A000144804F11801143815E0E06A2968C96A87
:1010B000884201D3012600E00026201DFFF76BF9CE
:1010C000E06A2969884200D928610C4900EB800058
:1010D00001EB8000211DFFF738F9FFF7B8F8DAE7D8
:1010E000054810B50468FFF793F9248EFFF798F9C7
:1010F000204610BD502C100004281000E82A1000D3
:1011000049444C4500000000D50D0000F0B5844670
:10111000002004460C4F14E05CF824600323DD003B
:1011200046FA05F280EA02600825002802DA87EA1A
:10113000400000E040006D1E002DF6DC5B1EEED589
:10114000641C8C42E8DBF0BD1B0000800D4880472A
:101150000D480047FEE7FEE7FEE7FEE7FEE7FEE795
:10116000FEE7FEE7FEE7FEE7FEE7FEE7FEE7FEE757
:10117000FEE7FEE7FEE7FEE7FEE7FEE7FEE7FEE747
:10118000FEE7FEE799110000C50000004FF0005196
:1011900091F8210010F00C0008D0042808D008288D
:1011A00008D0782001F8280F087070470F20F9E761
:1011B0001E20F7E73C20F5E77047000010B508490E
:1011C000042001240023C1F8FC00064A14601360C7
:1011D000054BA0221A70C1F8FC01C86710BD0000C1
:1011E00084E000E0D403002202E400E010B5042013
:1011F00000F0D6F8052000F0D3F8062000F0D0F873
:10120000072000F0CDF8082000F0CAF87649002049
:10121000086075492031086074490880724A121DBF
:101220001060714A2432106088806F4A0832106062
:101230006D4A2832106008816B4A0C3210606A4A8D
:101240002C3210608881684A10321060664A303251
:10125000106008820621042000F0BAF8062105205B
:1012600000F0B6F80621084600F0B2F80621072083
:1012700000F0AEF80421082000F0AAF8042000F0E5
:101280009BF8052000F098F8062000F095F807205C
:1012900000F092F8082000F08FF8042000F074F8B5
:1012A000052000F071F8062000F06EF8072000F02D
:1012B0006BF8BDE81040082000F066B800EB800035
:1012C0004FF6FF7101EA4001474800220260C20662
:1012D0001186012101607047434900200860704772
:1012E00000EB80004FF6FF7101EA40013E4800220A
:1012F000001D02604FF0005291860121016070478D
:1013000039490020091D0860704700EB80004FF646
:10131000FF7101EA400134480022083002604FF0BA
:10132000005211870121016070472F4900200831C8
:101330000860704700EB80004FF6FF7101EA400142
:10134000294800220C3002604FF0005291870121A1
:1013500001607047244900200C310860704700EBA1
:1013600080004FF6FF7101EA40011F480022103053
:1013700002601E4A0E3211800121016070471A4935
:10138000002010310860704700F01F0201219140D9
:1013900040094FF0E02202EB8000C0F800117047D6
:1013A00000F01F020121914040094FF0E02202EBC2
:1013B0008000C0F88011704700F01F0201219140A9
:1013C00040094FF0E02202EB8000C0F88012704725
:1013D0004907090E002803DA00F00F00044A00E074
:1013E000044A815470470000240500223200002086
:1013F00014ED00E000E400E0594801210160002103
:101400000160704757480121016000210160704769
:1014100010B5002000F08BF8534800220260FFF75F
:10142000F1FFFFF7E9FF514802605149A020087021
:10143000002000F088F8BDE81040002000F06BB8F4
:101440004A4801211C38016000210160704710B535
:101450000446002000F06BF8434841490460012035
:101460000860002000F06FF8BDE81040002000F098
:1014700052B830B53C4889B00468002C11D0202106
:1014800068460DF0BCFE3B4800783A4B00216A46A6
:101490005B1C02E0CD5C5554491C8142FADB1146CD
:1014A000A04709B030BD2E4901201C3908607047A3
:1014B0003048203000782F4921310978401A00F057
:1014C0003F0070472C4902780A7042784A7082784F
:1014D0008A70C278CA7002790A7142794A71827937
:1014E0008A71C079C8717047244800684178827851
:1014F0004FF00050437A0374214B1B7843744389A7
:101500001B0A83744389C37401754275C17981755F
:10151000017AC175704700F01F0201219140400916
:101520004FF0E02202EB8000C0F80011704700F09D
:101530001F020121914040094FF0E02202EB8000A0
:10154000C0F88011704700F01F020121914040094E
:101550004FF0E02202EB8000C0F8801270470000DC
:101560005C840022A00000223C2810007C040022A1
:1015700000E400E000040020000200204C281000DD
:10158000A428100010B5092000F02AF80A2000F065
:1015900027F8092000F030F80A2000F02DF8052186
:1015A000092000F035F805210A2000F031F81E4826
:1015B0007F21417081700171002100F848191B4999
:1015C000096891F8C810CA0709D08A0707D510F82A
:1015D0004A2FC1F38203012199408A43027010BD52
:1015E00000F01F020121914040094FF0E02202EB80
:1015F0008000C0F88011704700F01F020121914067
:1016000040094FF0E02202EB8000C0F880127047E2
:101610004907090E002803DA00F00F00044A00E031
:10162000044A815470470000480000204C281000F4
:1016300014ED00E000E400E0704710B5A44C072072
:1016400060700020207044F2C000608000BF00BFC6
:1016500000BF4CF2C000608000BF00BF00BF4CF272
:10166000E00060800920FEF7FDFD44F2E0006080AC
:1016700000BF00BF00BF4FF48040608010BDF0B5D8
:1016800000252E464FF00054E02716E0883401F084
:101690003F0160702170678000BF00BF00BFD4F8B9
:1016A00008C043F825C06680883C00BF6D1C521EF0
:1016B000491C3F2901D9401CC0B2002AE6DCF0BD1C
:1016C0002DE9F047824C0026A41C05462680DFF851
:1016D00004920121C9F880104FF4C058A4F800808A
:1016E00000BF00BF00BF00BF00BF4FF4805727807E
:1016F0003520FEF7B7FD2680FFF79FFF00F0A9F821
:101700005C2000F0B7F82B46012202210720FFF7EA
:10171000B6FF2B1D012203210620FFF7B0FF05F1C4
:101720000803012204210520FFF7A9FF05F10C039E
:10173000012203210720FFF7A2FF05F11003012278
:1017400004210720FFF79BFF00F083F8FFF775FFE8
:10175000278000BF00BF00BF00BF00BF00BF00BFA9
:1017600000BF00BF00BFA4F8008000BF00BF00BFE3
:1017700000BF00BF4FF440602080C9F88060BDE822
:10178000F0872DE9F0439946079B002603B1802698
:101790000023504C1F4665044FF001081DE000BFB8
:1017A00085F8890001F03F0C4CEA060C85F888C0EA
:1017B00059F823C0C5F88CC0C4F8B080C4F8B07024
:1017C000491CC9B2402902D3401CC0B20021D4F840
:1017D000C0C0BCF1000FFAD15B1C9342E0DBBDE856
:1017E000F0834FF0005282F88900002319B1802065
:1017F00082F8880001E082F8883036480121C0F87C
:10180000AC10C0F8AC3000BFD0F8C0100029FBD13C
:10181000704738B50C4605460021F820FFF7E1FF78
:101820000020014600902B462246F820FFF7A9FF32
:1018300038BD38B50C46054601210020FFF7D1FF21
:101840000120002100902B4622460846FFF799FF11
:1018500038BD10B51E4C4FF48040A41C20800420DD
:10186000FEF700FD0020208000BF00BF00BF00BFCA
:1018700000BF10BD70B5164C2126A41C268000BFE9
:1018800000BF00BF00BF00BF40F02105258000BFA2
:1018900000BF00BF00BF00BF44F221010843208009
:1018A0000420FEF7DFFC258000BF00BF00BF00BFA3
:1018B00000BF268000BF00BF00BF00BF00BF0020E8
:1018C000208000BF00BF00BF00BF00BF70BD000090
:1018D0008800002000100022F8B5FD4C0026354697
:1018E00026700120A66000F064FC0E2000F061FC70
:1018F0000D2000F05EFC0C2000F05BFC032000F0EB
:1019000058FC012000F061FC0E2000F05EFC0D2070
:1019100000F05BFC0C2000F058FC032000F055FCAC
:1019200000F088FD6A460221EA4800F0F4FEEA4928
:101930009DF8010008709DF80000422800D00326A1
:101940000521012000F04DFC05210E2000F049FC8E
:1019500005210D2000F045FC05210C2000F041FC84
:101960000621032000F03DFC012000F016FC0E20B3
:1019700000F013FC0D2000F010FC032000F00DFC23
:10198000A57065703046F8BD70B5D14BD888C0F3EE
:101990008001C0F34016C0F300247140C0F3C022A0
:1019A0006140C0F3803551406940400840EAC13091
:1019B000D88070BD38B520F040400D4600901446E8
:1019C0000421684601F058FAC4494978C90602D58D
:1019D000062D00D1401C0099616484F8420038BD96
:1019E000906470472DE9F047BD4D0646BB4C286812
:1019F00090F83404800718D5607840F0800060705B
:101A0000FFF7C2FF296800F00700084490F835048A
:101A100084F83100FFF7B8FF2968C0F302100844CA
:101A200090F83504800084F83000AE484FF0000A8A
:101A300084F83AA0C0F30E074FF0E9084FF001090F
:101A4000042E06D0032E1AD0022E37D0052E4CD0ED
:101A500072E0A24A3146606AFFF7ACFFA06AA06458
:101A6000A787607880060028286890F88B0701DA3D
:101A700040F0060084F8410084F83E805CE0974A1C
:101A80003146606AFFF796FFA06AA064934804217C
:101A9000243001F0F1F9934901EB8000C0F30E000E
:101AA000A087607880060028286890F88B0701DA04
:101AB00040F0060084F84100ED2013E0874A3146EB
:101AC000606AFFF777FFA06AA064A7876078800646
:101AD0000028286890F88B0701DA40F0060084F8A7
:101AE0004100E52084F83E0026E06078800623D59A
:101AF0002868243400F2C930784A0178A173C1788B
:101B000021744178E1748078207584F8169031460C
:101B10002068FFF74FFF7348C830C0F30E002083E2
:101B2000286890F88B0720F0060040F002006077EC
:101B300084F81A80A4F12404286890F87A17CA0758
:101B40000CD06948090701D5514600E049460160BB
:101B500014F8400F40F00300207008E0617890F81E
:101B6000BA07890701D520F0030084F840005848DF
:101B70004670BDE8F047594800F0FEBC2DE9F0473B
:101B8000564C4FF00009564E84F83A90E123054632
:101B900084F83E303068DFF858C14D4F90F8881710
:101BA00084F83F1090F87A175FEAC1784F49C1F383
:101BB0000E022146497801D0012D02D0062D1FD0FA
:101BC0003AE0A37CFB7039710A23A37441F0010150
:101BD0006170A28790F8AD279CF8003002F0F00207
:101BE00003F00F031A43227690F8B4076076C80614
:101BF00002D5F12084F83E00384A2946012017E03A
:101C0000A28790F8AD279CF800C002F0F0020CF01B
:101C10000F0C42EA0C02227690F8B4076076C806F0
:101C200003D543F0100084F83E002C4A2946A068F2
:101C3000FFF7C0FEE068A0646078410794F83F10A9
:101C400002D521F0020105E0326892F8882702F0FF
:101C50000202114384F83F10C10705D094F83E10EA
:101C600041F0020184F83E10316891F87A27D307D9
:101C70001FD0062D04D0072D02D0012D05D020E065
:101C800014F8400F20F0030011E01748110706D5A3
:101C90000121016014F8400F40F0030007E0C0F894
:101CA000009014F8400F20F0030000F102002070B3
:101CB00007E0800791F8BA0701D520F0030084F807
:101CC00040007D70BDE8F047044800F011BC000002
:101CD0004028100004100020A4281000782C1000C8
:101CE0004C28100080840120280A00220080012056
:101CF000F607100006280CD007280AD0012808D0C3
:101D0000042805D0032803D0052801D0022801D1DA
:101D100068E633E770472DE9F843FC4D8146012919
:101D200001D1002068716C79FA4F641CF84EA7F15C
:101D300024080FE0306890F87A07C00702D057F8FF
:101D4000242001E058F8242069464846904701289D
:101D500005D0641C082CEDD90020BDE8F8836C7117
:101D60009DF80000F9E770B5017800292CD00146F4
:101D70004C22E94801F04CFBE54E306890F87A07B8
:101D8000C0070AD0E448017811F0760F05D04278F8
:101D9000920702D441F080010170DC4D6878002880
:101DA00012D10121DC48FFF7B6FF04000CD03068E7
:101DB00090F81801000708D500F09FFC0120A870DA
:101DC0000A2000F087FB6C7070BD00202870204650
:101DD000BDE870408EE7002070478268920005D011
:101DE0000078000602D50120087070470020704777
:101DF0008268920006D00078C00703D006200870E1
:101E00000120704700207047C269920006D0007818
:101E1000000703D507200870012070470020704795
:101E2000426A920008D0826A32B10078800603D5F7
:101E3000022008700120704700207047426A92001B
:101E400006D00078C00603D5052008700120704731
:101E500000207047426A920006D00078800703D5C0
:101E6000042008700120704700207047826A32B158
:101E70000078400703D50320087001207047002038
:101E8000704700200870012070471FB500F09FFACE
:101E900001208DF80000A148019000F590600290AB
:101EA000C83003909C484168684688471FBD2DE9AB
:101EB000F05FDFF85CA29A4E0025DAF800004FF0E0
:101EC000010B90F87017C9073AD0934935310A7859
:101ED0004F78B2FBF7F807B901278C4CDFF8409236
:101EE0006178042907D1407D2225420009EB400199
:101EF0008C4801F08DFA6078032813D1864840257C
:101F00000421243000F0B8FFDAF8002009EB800645
:101F1000107D527D00EB420209EB420142008248F3
:101F200001F076FA20466478022C0AD0052C0BD0FA
:101F3000042C10D0032C0ED0022C0CD0052C0AD06F
:101F400097E06225764E06E0DAF80010744E2225FE
:101F500091F87187C83681688946414576DCB9F1C8
:101F6000000F04D14FF4C87170480DF048F9674A6A
:101F70006E48042C03D0032C01D0022C0CD100217C
:101F800008E000BF50F8213036F911C0634440F832
:101F90002130491CA942F5DB052C0BD1002107E0BB
:101FA00050F8213036F911C0634440F82130491C03
:101FB000A942F5DB09F101019160414554DB0021A3
:101FC0009160042C03D0032C01D0022C38D1DAF814
:101FD00000105346D1F8744700212FE0D3F800C019
:101FE0009CF851815FEAC86819D5DFF8448198F8F8
:101FF0000080B8F1010F12D192F80180B8F1040FFE
:102000000DD19CF815C08C4509DD8C4430F8218039
:1020100030F82CC0C444DFF81C8128F811C030F817
:1020200021C0DFF814810CFB07FCACEB040C26F894
:1020300011C050F821C048F821C0491CA942CDDB8D
:102040005178052915D100213C4A0AE011E000BF72
:1020500030F8213026F8113050F8213042F8213084
:10206000491CA942F4DB04E02046FFF743FE4FF091
:10207000000B5846BDE8F09F2DE9FF41264D6878DA
:10208000400603D4FFF713FF002816D0204F1F4C43
:10209000386890F87A07C00708D06078012805D121
:1020A000E078A8742079687007F061FA00211A4876
:1020B000FFF731FE18B1FFF71DFEBDE8FF810026D6
:1020C0006670386890F87A17CA0706D00A071C4964
:1020D00002D501220A6000E00E601A4AA4211173A1
:1020E00090F81801000702D5A67000F001FB2078D7
:1020F000012829D08DF80060084801900848029016
:10210000C8300390696868468847D6E740281000C1
:102110004C28100098F50000782C10000080012059
:1021200080840120461A01206A1A0120908501202E
:1021300063281000B41D012020870120B0880120F1
:10214000280A00220010002002208DF80000D3E7AA
:10215000294810B500684FF0000290F818010107F7
:10216000264806D58178012907D002290ED00329F7
:1021700012D18270BDE8104087E60221817000F024
:10218000C1FABDE81040322000F0A4B903218170EB
:102190004078BDE81040ADE510BD00F01F02012100
:1021A000914040094FF0E02202EB8000C0F800119E
:1021B000704700F01F020121914040094FF0E022DA
:1021C00002EB8000C0F88011704700F01F0201216F
:1021D000914040094FF0E02202EB8000C0F88012ED
:1021E00070474907090E002803DA00F00F00044A7F
:1021F00000E0044A815470474C2810004028100029
:1022000014ED00E000E400E0F0B53A2500224FF4C0
:1022100080141146FE4B0020A65CC718521C401CBF
:1022200087F860600C28F7DB01F03F0040F0800089
:1022300083F83500491CA942EDDBF0BD2DE9F043E0
:102240000024F34E81462546274600209C4206DAAC
:1022500000EB060819F804C088F860C003E000EB42
:10226000060C8CF86070641C401C0C28EEDB5019C6
:1022700000F03F00084340F0800086F835006D1CF8
:10228000032DE2DBBDE8F08300B514233A220021E0
:10229000E048FFF7D3FFDF4820233D220021143020
:1022A0005DF804EBCAE7DC480168D94801F299718E
:1022B000183011F8122C00F8112C11F8112C00F81C
:1022C000102C11F8102C00F80F2C11F80F2C00F81E
:1022D0000E2C11F80E2C00F80D2C0A7842704A785A
:1022E00082708A78C270CA7802710A7942714A791A
:1022F00082718A79C271CA7902720A7A42724A7A02
:1023000082728A7AC272C54A127802730A7B427359
:102310004A7B82738A7BC273CA7B0274BF4A521C97
:10232000127842744A7C82748A7CC274CA7C0275B8
:10233000BA4B0A7DDB1E02F0F0021B7803F00F039C
:102340001A4342754A7D82758A7DC275CA7D0276BE
:102350000A7E4276B14A921E12788276AF4A521EA7
:102360001278C276CA7E02774A7F82778A7FC277E6
:10237000CA7F80F8202091F8202080F8212091F851
:10238000212080F8222091F8222080F8232091F843
:10239000232080F8242091F8242080F8252091F82B
:1023A000252080F8262091F8262080F8272091F813
:1023B0002F209B490A701E220270332048740B2084
:1023C00088747047974801680029FCD17047964887
:1023D0000022026094481C38026094480261012186
:1023E0000161826081600260016002608D49A0F538
:1023F00074700B68002BFCD185490B7B43F02003E4
:102400000B730B7B23F040030B730B7B23F08003D8
:102410000B730B7B23F020030B73C0F8D823C0F899
:10242000E0238348027070477E4818300168002915
:10243000FCD1704730B57D480024743004607B487F
:10244000803004607948C4600121C160C4600460C8
:1024500001600460724D2020AD1D287068706C49C9
:10246000593D0873A42008736E481830016800298C
:10247000FCD1FFF7ACFFFFF716FFFFF705FFFFF7F3
:10248000C3FE6C4804606B4820300460AC8530BDEE
:102490005F49426C4A73130A8B73130CCB73130E90
:1024A0000B7492FAA2F2B2FA82F24A7490F84220C5
:1024B0008A74806CC874020A0A75020C4A75020E8E
:1024C0008A75820F81F8402090FAA0F0B0FA80F06F
:1024D000C8757047574900220A600A069085012096
:1024E000086070474F48001F01680129FCD1704700
:1024F00010B50446FFF7CCFF4948A18F401C01806E
:10250000434994F84020193181F82120424A126849
:1025100002F2997253784B7093788B70237CCB7056
:10252000238A1B0A0B71A37C8B77E37C8B74637DFE
:102530004B77237D00F8013CA37DCB77E37DCB7403
:10254000237E0B7512780A7094F83E20427394F83B
:102550003F20543801F8112C627ECA76314A19396D
:10256000121F1368012BFCD190F861000873BDE8BD
:10257000104041F28830ADE770B50446FFF788FFA0
:102580004FF00053A08FA3F854002348016891F83E
:102590007A07C2071E4854D06578B1F87D272D060A
:1025A00091F8AA5709D594F83160354480F82A503B
:1025B00094F830502A4492B201E080F82A50827692
:1025C000120AC276193014F82C2FC2712288120A0E
:1025D0000272A27802736288120A4273A279827729
:1025E000E27983F85320E27AC277227B4275627BDC
:1025F000C275A27C83F86120627D00F80E2C91F8F0
:10260000992722F0070200F81929A27B2C3C13E03D
:1026100000100020B80210004C281000F90710002C
:1026200053000020040B00221C0C0022D0030022C7
:102630004128100020050022D20708D091F8CE17BB
:1026400007E091F89A27827691F89B27B9E794F8EA
:10265000341080F8361050490A68012AFCD194F8E9
:10266000401080F83A1093F861100173BDE8704093
:1026700041F288302EE74949494B0A6892F8892788
:1026800002700A68B2F89E27428009681B7801F23E
:10269000A27103F00F03CA7A02F0F0021A4302712A
:1026A0000A88C280B1F8052002814A7B8272CA7B07
:1026B000C272897C017370473A49027801F80C2C88
:1026C00082784A724288120A8A7202790A7682797C
:1026D0004A73C288120A8A73027A8A740289120AB9
:1026E000CA74827A8A76C27A0A77007BC877704782
:1026F0002C4904201539087370472A4920201539C0
:10270000087370472749C020153908737047264958
:1027100000200860704770B51F4C1C342368002BE4
:10272000FCD11D4603E0C6185B1C86F880508B4226
:10273000F9D32368002BFCD102E0C45CD4545B1CA9
:102740008B42FAD370BD10B5002000F0FAFE164996
:102750000020086015480078002810D00E48001DA1
:1027600001680029FCD10F481538C078400602D511
:102770000F4901200870BDE81040FFF77DBC10BD77
:1027800010B5002000F0DDFE074900200860BDE81C
:102790001040FFF7DDBC0000000B00224C281000A9
:1027A000F607100015100020200500224128100017
:1027B00040281000FEE70446012007F011F8002130
:1027C0000F20226807F021F801210F20626807F02E
:1027D0001CF802210F20A26807F017F803210F2030
:1027E000E26807F012F80C210F20226907F00DF8BB
:1027F0000E210F20626907F008F80F210846A26930
:1028000007F003F820210F20E26906F0FEFF3948A7
:10281000026821210F2006F0F8FF364810380268C0
:1028200022210F2006F0F1FF32480C3802682321E4
:102830000F2006F0EAFF2F480838026824210F20F5
:1028400006F0E3FF2B48001D026825210F2006F04B
:10285000DCFF28483438026826210F2006F0D5FF17
:1028600024481438026827210F2006F0CEFF2248A2
:1028700000683021C06AC0F106020F2006F0C5FFD3
:10288000FEE710B5012805D0022805D0032809D09D
:10289000032102E0012100E00221BDE810400320F5
:1028A00006F09EBF0021032006F09AFFFEE710B558
:1028B00004460146042006F093FF012C00D1FEE7F8
:1028C00010BD0146082006F08BBF0146062006F029
:1028D00087BF10B504460146072006F081FF24B1EA
:1028E000012C03D0022C02D1FEE7FEE7FEE710BD6B
:1028F0000220EEE738ED00E00428100010B50020BB
:1029000000F01FFEBDE81040FDF762BC704710B537
:10291000002000F016FEBDE81040FDF773BCFDF787
:1029200087BD1A4810B5016821F00401016000203C
:1029300000F007FEBDE81040FEF79BBD70470CF0AD
:1029400032BB10B5002000F0FCFDBDE8104006F0E1
:10295000EFBD10B5002000F0F4FDBDE8104007F019
:102960007AB910B5002000F0ECFD0948006890F835
:102970002901800703D5BDE8104006F0EDBD10BD6C
:1029800070477047704770477047704710ED00E020
:102990004C28100010B542218B480CF00EFC8A48E0
:1029A0008A498B4A018042808A4981808A4BC38050
:1029B0008A4C04818A4C44818A4C84818A4CC4812B
:1029C0008A4C04828A4C44828A4C84828A4CC48217
:1029D0008A4C04838A4C44838A4C84838A4CC48303
:1029E0008A4C04848A4C44848A4C84848A4CC484EF
:1029F0008A4C0485C387428781878949A0F84010A3
:102A0000884801688648B1F89C274280B1F8A02721
:102A1000C280B1F8A517018110BDF0B585B0FF22C5
:102A2000142168460CF0C1FB6846FEF749FE039886
:102A300003250127072645F2AA54A04202D0049894
:102A4000A04239D1DDE90001884206D002998842CE
:102A500003D00198884208D100900498A0420FD179
:102A60000098000E012804D006E00020FFF72DFF9B
:102A70000FE00098C0F301370098C0F3032602E08E
:102A80000120FFF722FF0398A04213D1009800F025
:102A900007056549887920F0F30207F0030040EA52
:102AA0000610104388716148017865F302010170D6
:102AB00005B0F0BD0220D9E70120FFF706FFF9E7D6
:102AC00070B55A493F20491C0870FEF75FFBFEF7BE
:102AD0009FFC544D28680078A52802D00120FFF7FC
:102AE000E6FE5348006810B10020FFF7E0FE2868BA
:102AF0004FF000064FF0010490F829118A074FF0BB
:102B0000085104D5C1F89863C1F8804301E0C1F8C9
:102B1000984390F82811474A01F00101116090F89C
:102B20002811121DC1F34001116090F87A17C907EE
:102B30000AD041490C60404908390C6090F87A0786
:102B4000000701D5081D0460FEF776FDFEF74EFB79
:102B5000FEF7C2FE032802D10020FFF792FEFEF727
:102B6000C3FCFEF72BFBFEF70DFDFFF756FF2868B1
:102B700090F829018107314801D5046000E0066022
:102B8000046070BD40F2F23010B501074881FFF7D4
:102B900097FFFFF7FFFE2A493F20086029490020E0
:102BA00008602A482849016001F5AA6028490860A0
:102BB000FDF746FB00F04EF800F062F8FDF747FB2A
:102BC000FEF721F9012010BD000001200080012046
:102BD00074A30120F4A70120420001208084012079
:102BE000E2190120061A0120DC1B0120001C012033
:102BF0007C200120A0200120C2160120E616012021
:102C0000461A01206A1A01202C1D0120FC1D0120FA
:102C1000501D0120741D01207E190120A2190120E0
:102C2000003810004C281000001000202000002068
:102C3000C810002288040022280A00227C040022F6
:102C4000AC1A0120A0281000C42C10007C28100011
:102C50008028100070B5454D002400210120FDF7AB
:102C6000FBFB45F8240020B1FDF7EAFC55F82400F1
:102C700010B90020FFF72DFE641C072CEDDB70BDA2
:102C80001FB53A48012100240091001FCDE901043D
:102C90002346402236A138480394FDF7FFFD012862
:102CA00002D00120FFF715FE3048062100911838A8
:102CB000CDE901040023402230A132480394FDF7FE
:102CC000EDFD012802D00120FFF703FE2748052172
:102CD00000911438CDE9010400234FF480722AA139
:102CE0002C480394FDF7DAFD012802D00120FFF7FC
:102CF000F0FD1E48022100910838CDE901040023AF
:102D0000B42225A126480394FDF7C8FD012802D06E
:102D10000120FFF7DEFD1548042100911038CDE9B0
:102D2000010400234FF4C8721EA121480394FDF74B
:102D3000B5FD012802D00120FFF7CBFD0B48032190
:102D400000910C38CDE9010400234FF4007219A161
:102D50001A480394FDF7A2FD012805D004B0012014
:102D6000BDE81040FFF7B5BD1FBD000024381000BE
:102D700054736B5F436D6400BDEF000054736B5F71
:102D8000527074009D9B000054736B5F53537973B2
:102D9000000000007D60000054736B5F535300001F
:102DA0009B88000054736B5F5363616E00000000EA
:102DB0009794000054736B5F4D740000E7CF0000E0
:102DC0002DE9F0479246012547F6F872564299469A
:102DD000AC460024089F16E030F8143031F8148017
:102DE000A8EB03031BB29A4200DD1A469E4200DAAA
:102DF0001E46002B02DA4FF0000502E001DD4FF025
:102E0000000C04F10104BC42E6DB55EA0C0306D0D9
:102E1000012D01D02DB108E0BCF1010F05D1002238
:102E200003E0BCF1010F00D1324600252C462B46B1
:102E300011E000BF30F8136031F813C01644ACEB5A
:102E4000060636B24E4505DAC9F1000C664501DDCD
:102E50003544641C5B1CBB42ECDB95FBF4F10A447B
:102E6000002105E030F8113013442AF81130491CD4
:102E7000B942F7DBBDE8F08770B503460020024693
:102E8000FE4C09E09D5C521C05F00F0604EB151585
:102E9000A65D2D78304428448A42F3DB70BD884219
:102EA00000D308467047884200D8084670478842D9
:102EB00000D30846904200D3104670472DE9F047F2
:102EC000D0F810C00568046A85FB0C12A1FB04123F
:102ED00042694368914683FB02628269E246A6FB2F
:102EE00002677618D0E9021781FB07C8C069ACFBFE
:102EF00000C81CEB060682FB0A2CA2FB011280FB19
:102F00000902A0FB0502401884FB0712A1FB031273
:102F10000818301A4FEAE071ACE72DE9F04389B0A8
:102F20000446006800906068019020690290606823
:102F3000039020690490A069059020690690A0691B
:102F40000790E06908900D466846FFF7B7FF804696
:102F5000A0680190E068049060690790894668461F
:102F6000FFF7ACFF064660680190A06802902069F8
:102F70000490E0680590A0690790606908900F468A
:102F80006846FFF79BFFC5E90401C5E90267C5E98B
:102F9000008909B0BDE8F0832DE9FF4F4FF0000A2A
:102FA00089B09B465746D146D0465646554654466C
:102FB000202168460CF023F90B9810E0099982440F
:102FC00031F9102000FB00F102FB01668844414307
:102FD00002FB009901FB004417440D44401C584576
:102FE000ECDD0B99ABEB0100401CCDE9000ACDE90B
:102FF0000654CDE90486CDE9027968460A99FFF7BF
:103000008CFF0DB0BDE8F08F9D480068017B427BCE
:1030100041EA0221827BC07B41EA024141EA006031
:1030200040007047964800680179427941EA0221E0
:103030008279C07941EA024141EA0060704700B5F7
:10304000FFF7E2FF4008400000BDF8B50E46044619
:10305000FFF7F5FF0090FFF7D7FF0546042168460C
:10306000FFF70AFF04EB400700240099204623469F
:103070004FF0010C0CFA03F20A4207D02A4204D0A6
:1030800037F8102026F81420641C401C5B1C122BFF
:10309000F0DBF8BDC6E7FCB50E460746FFF7CFFFED
:1030A0000190FFF7BFFF0090FFF7BCFF054604212A
:1030B00001A8FFF7E1FE044604216846FFF7DCFEA5
:1030C00000EB440007EB400700200099044603464C
:1030D0004FF0010C0CFA03F20A4207D02A4204D046
:1030E00037F8142026F81020401C641C5B1C202B91
:1030F000F0DBFCBD00B5FFF787FF40F0010000BD2D
:1031000090E7604A520102EB810101F10851086029
:10311000704701EB4010801001EB4101490018227B
:1031200091FBF2F300EB400000F5801002FB13115D
:10313000006820F07F40C84000F03F00704701EB7E
:103140004010801010B501EB41014900182391FB9C
:10315000F3F403FB141300EB400000F580103F2450
:1031600001689C40A1439A400A430270110A4170D1
:10317000110C817010BD2DE9F14FFFF7BBFF8046A8
:10318000FFF750FF00258446A946AB46AA462F46C6
:10319000012000FA07F111EA0C0F36D00024012DAE
:1031A00032DB37490968097D491EA9422CDD00261A
:1031B0000120B04010EA080F23D039463046FFF70F
:1031C000A8FFE4B1022C1ADB2D4909684A7D521E82
:1031D000A24214DD484512D0097D009A04FB015338
:1031E00032F9133004F1010202FB0152009931F966
:1031F0001210591A00D549428B440AF1010A81463E
:10320000641C761C1D2ED3DB6D1C7F1C202FBFDBA6
:103210009BFBFAF0BDE8F88F2DE9F74F184B4FF004
:10322000000B91B018681646DA4690F8770000F067
:103230000F08C8F11009FFF75DFF1090FFF7F2FECD
:103240000025AC4603950F9001200F9A00FA0CF16F
:1032500011427DD0002106910C460591012D78DBAD
:1032600007490968097D491EA94272DD002701202E
:103270001099B840084270D0614605E0BCF50000E6
:103280004C281000AC1A01203846FFF742FF0146D7
:10329000F4B3022C5BDBD6480068427D521EA2428A
:1032A00055DD039A914290F87A201DD1007DBA42F3
:1032B00004FB0053119A0BDD32F91320631C03FB4E
:1032C0000053119830F91300101A23E0404223E014
:1032D00032F91330621C02FB0052119830F91200CF
:1032E000181A2FE040422FE0BA4219DD007D119AF2
:1032F00004FB005332F9132004F1010303FB0053D4
:10330000119830F91300101A00D54042129A00E0CB
:103310001DE0801A0028D9DB069A1044069016E0BA
:10332000027D119804FB025330F9133004F10100BF
:1033300000FB0252119830F91200181A00D54042D1
:10334000129A801A0028CDDB059A1044059002E0FD
:103350001AE018E001E0641C03917F1C1D2F86DB3E
:10336000022D0CDB06990D98401A01D5C0F1000022
:10337000834405990C98401A00D54042824406982F
:103380000D9005980C906D1C9948006890F87B0092
:10339000604518DD316801FB08F109FB0B104FEAAD
:1033A000E07100EB11704FEA20103060B06800FB54
:1033B00008F009FB0A004FEAE07100EB11704FEAD8
:1033C0002010B0601CE003D14FF0000BDA4617E08C
:1033D000706800FB08F009FB0B004FEAE07100EB9E
:1033E00011704FEA20107060F26802FB08F209FBCE
:1033F0000A204FEAE07100EB11704FEA2010F060F4
:103400000CF1010CBCF1200FFFF61EAF14B0F9E572
:1034100004E000BF11F8013B00F8013B521EF9D255
:1034200070477CB50D460446FFF709FE0090FFF794
:10343000F9FD019000980421400800906846FFF7CC
:103440001BFD0646042101A8FFF716FD304482004B
:1034500021462846FFF7DCFF7CBD0B46644909681E
:103460004A7D097D521C4A43014652001846CFE767
:1034700070B504464C210BF0C2FE00235C4D237056
:103480006370286890F8CD0700F0010043EA40100F
:103490006070296891F88C17C1F3001140EA01109F
:1034A00060706360FFF726FEA060FFF7BBFD514E22
:1034B000E06070882082286800F2AC70C17AA17444
:1034C000017F2175817A6175017BA1750178E175B4
:1034D00049494078097800F0F00001F00F010843F5
:1034E0002076FFF7ACFD6062FFF79CFDA062F088DC
:1034F000A085E085286800F2AD70017F84F8321065
:10350000817F84F83310C17F84F8341010F83B1C9D
:1035100084F83510012184F83610417F84F8371083
:10352000417884F83810C17884F8391010F8021CFA
:10353000E174407B84F8400084F8313084F8303006
:1035400070BD10B50446FCF77BFE4FF00051012C16
:1035500009D12748006890F81801400703D527488B
:10356000007805280CD091F821003F2804D03F2096
:1035700081F82100FDF70AFEBDE81040FCF767BEA8
:1035800091F821003128F7D03120F1E7184B10B520
:103590001A68947E640704D5D28A0468A2EB0402F8
:1035A00002601A68947EA40703D5128B0C68121B64
:1035B0000A600268002A00DA002202601C68E48ABD
:1035C000A24200DD224602600A68002A00DA0022D8
:1035D0000A601C68248BA24200DD22460A601B6838
:1035E0009B7EDB0702D003680B60026010BD000009
:1035F0004C28100000381000F60710009428100026
:1036000010B501461022FB48FFF702FFFA48416857
:103610004FF40060FDF72CFD002803D0BDE81040FA
:10362000FCF7F0BE10BD70B594B006460D461446CA
:103630006846FFF71DFF14F0050F02D001208DF83A
:10364000000040F6E250044221D0EC48026892F8B3
:103650005001C0070ED192F8020258B992F8E00268
:10366000C00707D192F86002C00703D192F8B001F9
:10367000C0070CD092F87A07C0079DF8000002D06E
:1036800040F0060001E040F020008DF800009DF8B9
:103690000000ADF82E50ADF81060ADF82C5010F0D1
:1036A000B60F05D09DF8010040F004008DF8010030
:1036B000AFF2B300CF4D03244FF40066019068468B
:1036C000FEF751FB00213046FDF752FC0021304649
:1036D000FDF77CFC2878002804D0FFF7D2F8641EA0
:1036E000002CECDC14B070BD10B50446C00709D046
:1036F0004FF49061C2480BF060FD4FF49051C14807
:103700000BF05BFD14F0420F07D02421BE480BF0F4
:1037100054FD4021BD480BF050FDA0060AD5902174
:10372000BB480BF04AFDBDE810404FF48071B9482A
:103730000BF043BD10BD2DE9F0410746AF480068CE
:1037400090F82010490710D590F821000125C0F30A
:10375000011085400024B04E05E0F18870883A469B
:10376000FFF761FF641CAC42F7DBBDE8F0812DE997
:10377000FF4F83B08046FFF7C3FC0190FFF7BAFC10
:10378000009004216846FFF777FB0446042101A856
:10379000FFF772FB4443994801264FF42A61006801
:1037A00090F8210000F00707BE409C480BF027FD71
:1037B0000025DFF86892DFF860A2DFF838B21CE07D
:1037C000BAF8061042460498FFF72DFF18F0050FCF
:1037D00012D09349DBF8040005F0DFF9904A00208D
:1037E000494607E051F8203032F910C0634441F8EF
:1037F0002030401CA042F5DB6D1CB542E0DB18F028
:10380000050F0CD00020494607E000BF51F82020EA
:10381000059B3A4123F81020401CA042F6DB07B07C
:10382000BDE8F08F2DE9F74F744C84B092462068C4
:10383000B0F83B100391B0F83D10029190F8501190
:10384000C9070ED190F8021259B990F8E012C907D1
:1038500007D190F86012C90703D190F8B001C007F2
:103860007CD0FFF7ECFB0090FFF714FC01900421E3
:103870006846FFF701FB8146042101A8FFF7FCFA27
:10388000484445002068A046264690F821000124BF
:1038900000F00707BC40A90060480BF0B0FC31689D
:1038A00091F8F002C20706D0800704D491F8F10223
:1038B000044405F031FE0026C34630E05648DDE9F9
:1038C00004214088FFF7AFFEDBF80000494990F87B
:1038D000CD07D1F80880C00704D04246C968104619
:1038E00005F0E2F8DBF8000090F8F002C10708D01C
:1038F000800706D44B49404605F046F870B1DFF822
:1039000024810020454907E051F8203038F9102083
:103910001A4441F82020401CA842F5DB761CA64240
:10392000CCDB3E4C00215A461EE03C48136850F860
:10393000210093F8F06240FA07F05FEAC67C08D0F5
:10394000B60706D593F8F162761C4643B3F8F20247
:10395000301AB1EB490F02DA039B01E01DE0029B34
:10396000184424F81100491CA942DEDB106890F8C5
:103970005011C90703D190F8B001C0070DD00498C9
:1039800010F0220F09D02046DAF80010FFF75DFB97
:103990002046DAF80410FFF77EFB40E72DE9F047F8
:1039A0009A46164B894600210125194E1C681AE0DB
:1039B00032F8113030F81170DB1B1FB200230AE01F
:1039C00003EBC30C06EB8C0C5B1C3CF811801BB2A8
:1039D000B8442CF8118094F880C305EB9C1C9C45DE
:1039E000EEDC491C09B2637D8B42E1DC0020094A10
:1039F00033E00000A43810000C3810004C281000F0
:103A000042000120C2040120C2160120E616012056
:103A10008A1701203E18012000381000C42C100025
:103A200040890120C08D01203AF8103039F810107B
:103A3000591A0BB2002108E002EB8116491C36F836
:103A4000107009B21F4426F8107094F8806305EBDB
:103A500096168E42F0DC401C00B2217D8142E3DCF0
:103A6000BDE8F0872DE9F041064610F00C0F17D0A5
:103A7000FE4D286890F8D000400711D5FC4F002477
:103A80002868002300EB4400B0F8021104EBC400E6
:103A900007EBC0123046FFF76AFE641C042CEFDB14
:103AA00063E62DE9F047F14C824686B0216800F4C8
:103AB000126091F8801349073AD5002838D00025C4
:103AC000DFF8B083DFF8B093012615E000EB450086
:103AD0001421B0F8B27368460BF091FB05EBC501F9
:103AE00008EB8100009009EB851001906A46394689
:103AF0005046FFF797FE6D1C206890F8801306EB88
:103B00009111A942E2DC90F85011C90710D090F849
:103B1000911109060CD5407DD6494200D748FFF7E0
:103B200077FC2068D449007D4200D548FFF770FC3F
:103B300006B095E7F0B540F2824185B010EA010584
:103B400032D000F41263C948CE4A00240068D688F7
:103B5000012190F8802301EB921106E000EB44076D
:103B6000B7F8B273BE4202D0641CA142F6DCA14297
:103B70001CDD51071AD5CBB190F85011C90703D1FC
:103B800090F8B001C0070FD0BA4904EBC40001EBB4
:103B900080012422BC48FFF73BFCB748402200EBE1
:103BA0008411BA48FFF734FC05B0F0BD1421684613
:103BB0000BF025FBB4480090B44801906A463146AA
:103BC0002846FFF72FFEEFE72DE9F047A74C012528
:103BD000DFF8BC92206800F25640018882881144C8
:103BE0004F084188C088084446080020014618E074
:103BF00039F91130B2F85284434503DBB2F84E84F0
:103C000043450DDDB2F84E240025934208DD4FEA0E
:103C10004C029F499F48FFF7FBFB21680120497D2B
:103C2000491C226892F815C08C45E1D80022DFF8C3
:103C3000689218E039F91230B1F85484434503DB37
:103C4000B1F8508443450DDDB1F8501400258B4286
:103C500008DD4FEA4C0290499048FFF7D9FB2168F4
:103C600001200A7D521C216891F814C09445E1D8C6
:103C700091F84924520701D501280AD0012D09D015
:103C8000242187480BF099FA402186480BF095FAD9
:103C90000020E5E600207C4C814D024611E000BF8B
:103CA00034F91030B1F85AC4634503DBB1F856C497
:103CB000634503DDFB1A25F8103001E025F81020DC
:103CC000401C4B7D8342EBD80020704D754C10E0BA
:103CD00035F91030B1F85C74BB4203DBB1F85874AD
:103CE000BB4203DDF31A24F8103001E024F8102061
:103CF000401C0B7D8342EBD8CAE72DE9F04180469A
:103D00006948002637460078800628D5002504E05B
:103D1000012C02D14046FFF70DFFFFF755FF044687
:103D2000012806D101F079F901266D1C032DEFDB86
:103D300017B1012E0CD00FE00120FEF7C2FD2421A7
:103D400057480BF03AFA402156480BF036FA06E095
:103D500056490878401C0870C22005F0D2FD434C3B
:103D600001234F492068427D474804F0E1FB206869
:103D700001234C49027DBDE8F041444804F0D8BB22
:103D8000F0B53A480068437D017DB0F84C44B0F886
:103D90004A6447484B4300EB410500210A46084668
:103DA0000AE000BF35F91070A74201DD491C02E0AE
:103DB000B74200DA521C401C9842F3DB914201DD0D
:103DC0000120F0BD0020F0BD2DE9F04180463948CA
:103DD00000252E460078800623D50024294F0AE0CE
:103DE000012808D100F037FC012579880023304AEA
:103DF0004046FFF7BCFCFFF7C3FF48B1641C032C2F
:103E0000EEDB012E04D0BDE8F0410020FEF759BDE5
:103E1000C12005F076FD012D03D124490878401C0E
:103E20000870A2E42DE9F041234D002307465C1EF3
:103E3000224619462868FCF74BFC00232246194607
:103E4000E868FCF745FC17F040040AD024220E492C
:103E50001A48FFF7DDFA194840220C492430FFF7D1
:103E6000D7FA3846FFF740FC15482BE04C281000E5
:103E7000C20401208A1701203E1801201A180120CF
:103E80003E19012000381000C2160120E61601205C
:103E9000461A01202C1D01206A1A0120FC1D012058
:103EA000888E0120AC8E01205C281000A52810000F
:103EB000420001205828100024381000403810001B
:103EC000542810000178012904D1002101703846DE
:103ED000FFF731FC3846FFF7C5FD3846FFF7E1FD37
:103EE00017F0010606D08D4800238D4A41883046E0
:103EF000FFF73DFCF0078B4E16D0306890F820009D
:103F0000000709D58648FFF736F98749874A0860D0
:103F100001468348FFF780F9306890F84904C007EC
:103F200002D03846FFF750FF3846FFF703FE3068EF
:103F300090F84904800702D53846FFF7DEFE5CB1F1
:103F4000306890F88003400706D57B49784B794A62
:103F5000A1F12400FFF722FD78490120087078497B
:103F6000087005F0CEFA2868FCF76AFBE868BDE83F
:103F7000F041FCF765BBF0B46A490022714C0B6854
:103F8000B3F80211814214D2B3F80811814201D86A
:103F900003220EE05FF0010103EB4105B5F8025189
:103FA000A84201D10A4602E00DD2A1F101028A42E3
:103FB0000DD102EBC20004EBC011F0BC4FF49062D3
:103FC0005748FFF725BA491C0429E5DBF1E703EB65
:103FD0004103534DB3F80021B3F80231801A0002B7
:103FE0009A1A90FBF2F301EBC10100204FF4107616
:103FF00004EBC11101EB4002A2F5906231F91040CF
:10400000B2F90020A41A5C4302EB242225F8102008
:10401000401CB042EEDBF0BC70472DE9F041414955
:104020000025494A0968494EB1F8B23383421AD291
:1040300091F880339C0901EB4407B7F8B2738742CB
:104040000AD9012404EB931313E000BF01EB4407EA
:10405000B7F8B273B84201D1254602E008D2A4F104
:104060000105A5421CD191F85001C00708D103E019
:10407000641CA342EADCF6E791F8B001C0074CD01B
:1040800005EBC50002EB800124222A48FFF7C0F9A6
:1040900006EB8511BDE8F04140222548FFF7B8B98D
:1040A00001EB4405B5F8B033B5F8B253C01A0002BD
:1040B000EB1A90FBF3F391F85001C00703D191F88C
:1040C000B001C00729D01B4D04EBC401002002EB56
:1040D000810100BF01EB400231F9107032F9242C4C
:1040E000BF1A5F4302EB272225F81020401C12283C
:1040F000F0DB0F4D002006EB841100BF01EB400206
:1041000031F9104032F9402CA41A5C4302EB24220E
:1041100025F81020401C2028F0DBC1E400381000F6
:10412000420001204C281000842810006437100041
:10413000E6160120C2160120643810006228100023
:104140008F281000C20401208A1701203E18012088
:104150002DE9FC5F0024A146A646A3460226FE4A9E
:104160001268537D127D5B1E951E2EE002FB06F742
:1041700001EB470C00EB4707BCF902C0B7F902702E
:10418000009702271EE000BF06FB0278CDF80480EE
:1041900031F918A030F91880CDF80480E2450BD031
:1041A000DDE9008CBCEB080C01D5CCF1000C6444BB
:1041B00009F1010C1FFA8CF9DDF80480D4467F1C4C
:1041C000CDF80080BD42DFDA761CB342CEDAB9F119
:1041D000000F01D0B4FBF9F4022639E002FB06F728
:1041E00001EB470C00EB4707BCF902C0B7F90270BE
:1041F00000974FF0020728E006FB027931F919A079
:1042000030F91990BAEB0C0C01D5CCF1000C0FFA77
:104210008CFCDDF80080BCF1000FA9EB080C06D087
:10422000BCF1000F01DACCF1000CACEB040CBCF1DA
:10423000000F01DACCF1000C1FFA8CFCF44500D918
:10424000E646D4467F1CCDF80090BD42D4DA761CF9
:10425000B342C3DA012635E006EB420731F917C055
:1042600030F9177000974FF0030728E007FB026949
:1042700031F919A030F91990BAEB0C0C01D5CCF139
:10428000000C0FFA8CFCDDF80080BCF1000FA9EBEC
:10429000080C06D0BCF1000F01DACCF1000CACEB3D
:1042A000040CBCF1000F01DACCF1000C1FFA8CFCFD
:1042B000DC4500D9E346D4467F1CCDF80090BB42D4
:1042C000D4DA761CB542C7DA02B05A467146BDE868
:1042D000F05F032005F058BB0388934200D90280A9
:1042E0000888904200D20A807047F0B587B0064631
:1042F000002047F6FF71ADF80810ADF80400ADF8E6
:104300001010ADF814000227934C10E0012508E0CE
:1043100007FB005001A936F8102002A8FFF7DCFFC8
:104320006D1C2068007D411EA942F1DC7F1C2068C5
:10433000407DB842EADC002512E0284405A936F8A1
:10434000102004A8FFF7C8FF2068417D007D01FB15
:10435000005005A936F8102004A8FFF7BDFF6D1C1A
:104360002068007DA842E8DC012514E0007D05A955
:10437000684336F8102004A8FFF7AEFF2068691CD8
:10438000007D484306EB400005A930F8022C04A844
:10439000FFF7A2FF6D1C2068417D491CA942E5DCA6
:1043A000BDF80420BDF80810012005F0EDFABDF8B5
:1043B0001420BDF81010022005F0E6FA07B0F0BD99
:1043C00070B50C460546FFF790FF21462846BDE82C
:1043D0007040BDE610B5014610226048FFF718F89E
:1043E0005F4841688020FCF743FE002803D0BDE809
:1043F0001040FCF707B810BD30B593B004466846CE
:10440000FFF736F80021012C02D0022C08D016E06C
:1044100001208DF800008DF815108DF814100EE0B5
:104420004D48006890F87A07C00701D0062000E0E8
:1044300020208DF800008DF834108DF833109DF891
:104440000100AFF26F0140F04C00444D01918DF836
:10445000010003246846FDF786FC00218020FCF75C
:1044600087FD00218020FCF7B1FD2878002804D0CA
:10447000FEF707FA641E002CECDC13B030BD0246D8
:104480001621012000FA01F3134201D1491EF9D58A
:10449000491C8840104370472DE9F05FFEF72AFE63
:1044A0000546FEF72DFE2C4C0746206890F88C0739
:1044B000C00603D52846FFF7E2FF05464FEA550937
:1044C0004FF4906127480AF078FE4FF01D084FF036
:1044D000000A0120FFF790FF20480026D0F804B022
:1044E0001D480068047D34E0012000FA06F111EA5D
:1044F000090F2DD000250120A840384225D029469B
:104500003046FEF706FE1449DFF858C009683CF94A
:104510001430B1F83421991A3BF91430A3EB02029C
:1045200000D54942002A00DA5242914204DD0E4988
:104530002CF8143021F814003F2805D2401CC2B2D8
:1045400029463046FEF7FBFD641C6D1C202DD2DB96
:10455000761C4645C8DB09E04C281000B438100032
:104560000C38100074A30120F4A70120FDF74CFEC5
:104570000AF1010ABAF1400FABDB0120FFF73CFF63
:10458000F848DFF8E4B3002500684FF0010A067D23
:104590000AFA05F111EA090F0FD000240AFA04F013
:1045A000384207D01BF816002146C2B22846FEF753
:1045B000C6FD761C641C202CF0DB6D1C4545E7DB3A
:1045C000FDF722FE0120FFF717FFE848E6494068A3
:1045D000BDE8F05FF4E62DE9F05FE24A116891F87A
:1045E0003001C407E248037803F0F00514D00570E9
:1045F00000264B7D0C7DDFF874A35B1CB046914612
:1046000004FB03F783460120FFF7F6FE2046DAF8A5
:104610000420D9F800100EE091F83E1101F00F01CE
:1046200029430170BDE8F09F32F91030B1F832C172
:104630006345F7DB401C8742F6DC0F2EF2D2761C76
:10464000F6B245EA060108F101088BF80010B8F14E
:10465000100FD8DBE6E710B54FF42E714FF4801041
:104660000AF0CDFDFDF7D0FDFFF7B5FFFFF714FF12
:10467000BC4ABF481268401D017892F8FB2701F040
:10468000F00102F00F0211430170BDE8104001205B
:1046900005F037B92DE9F0438DB000214FF6FF70DA
:1046A000ADF82C10DFF8CCC2ADF82800ADF804004E
:1046B000DFF8C082B04FDFF8AC92ADF80810ADF86B
:1046C0001800ADF80C10ADF81000ADF814100CF196
:1046D000140C0D460E460124B96804FA06F008428F
:1046E00013D0002D0ADBD9F80000007D801EA842FF
:1046F00004DB1CF805200BA90AA803E01CF8052020
:1047000002A901A8FFF7E8FD6D1C761C202EE3D35B
:1047100000252E464FEA090C796804FA06F0084293
:1047200013D0002D0ADBDCF80000407D801EA8427B
:1047300004DB18F8052003A906A803E018F80520F3
:1047400005A904A8FFF7C8FD6D1C761C202EE3D335
:104750008748BDF82C20801CBDF828100078024442
:1047600092B2ADF82C20BDF8043001440344ADF8FA
:104770000430BDF8083089B21844ADF808007C4810
:10478000ADF82810401CBDF8183000780344ADF88F
:104790001830BDF80C300344ADF80C30BDF81030C3
:1047A0000344ADF81030BDF814301844ADF81400CF
:1047B000042005F0E9F8BDF80C20BDF8181005201C
:1047C00005F0E2F8BDF80820BDF80410062005F059
:1047D000DBF8BDF81420BDF81010072005F0D4F860
:1047E0000DB0BDE8F0832DE9F04763485D4B002430
:1047F00046694568D3F800302246012140F6FF792A
:1048000001FA02F72F421FD036F91480B8F1000FD9
:1048100005D0C84507D1076847F0100712E00768C0
:1048200047F020070EE0B3F836C1B3F84171E24615
:10483000BC44C44503DBAAEB0707474503DD076813
:1048400047F040070760641C521C202AD8D300247C
:104850008769D0F80860224601FA02F535421DD07A
:1048600037F914502DB14D4507D1056845F01005B5
:1048700012E0056845F020050EE0B3F83AC1B3F840
:1048800043A10CEB0A08A84503DBACEB0A0CAC45D2
:1048900003DD056845F040050560641C521C202AB4
:1048A000DAD3BDE8F0872DE9F05F334C0020314FBB
:1048B000666801460346012202FA03F5354203D039
:1048C000FD5C854200D928465B1C202BF4D3294E81
:1048D000D4F808701436002302FA03F53D4203D0E1
:1048E000F55C8D4200D929465B1C202BF4D3DFF800
:1048F00080801C4D08F1030808F1010988F80000C8
:1049000089F800102A68A8F1020AA8F1010B92F8B0
:104910007A37DE077ED09B077CD502F28B72537DFF
:10492000947D157E03EB04239CB2D37DD67E03EBEE
:1049300005239DB2937E577F03EB06239EB2137F20
:10494000127803EB07239FB2520617D5631900EBC9
:1049500043009AF80020F31910449BF8002001EB63
:10496000430118E04C281000F4A70120B4381000CF
:10497000F6071000B8021000AC28100062195200AF
:1049800002EB40029AF800001044F219520002EBC8
:1049900041029BF800101144FEF785FAFE490968B0
:1049A00001F27B72B1F87B37834201D2A1F87B0719
:1049B00091F87A07400736D591F88B07400617D54E
:1049C000600040426B4291F87B1700EB43000144CA
:1049D0009AF80000091A88F80010700040427942E5
:1049E00000EB4100117801449BF80000081A38E000
:1049F0009AF8000063191844B1F87B17404201EBA4
:104A00004000C0F3470188F800109BF80000F1193E
:104A1000084400E008E01188404201EB4000C0F388
:104A2000470189F80010FDE5DC4D9AF800209BF85D
:104A300000302D6802440B44FF2645F080059A4261
:104A400009D2991A0844FF2802D888F80000E9E53D
:104A500088F800600AE09342E5D2D01A0844FF28A3
:104A600002D889F80000DDE589F800602560D9E505
:104A70002DE9F84FDFF82093C94DC948D9F8001047
:104A80001435DFF818B391F83011044649064FF099
:104A9000010A7DD534210AF0B2FBFFF704FFFDF7D0
:104AA00002FCFDF7F1FB042003264FF00008009004
:104AB0000220FFF7A1FCF00729D04FF0000E72464C
:104AC00070464F464FEA0B030AFA00F1D3F804C0D0
:104AD00011EA0C0F13D05969D7F800C031F9121040
:104AE000BCF838C1614509DA215CDDF800C04FF03F
:104AF000010E6144FF2900DDFF212154521C401C9E
:104B00002028E1D3BEF1000F01D126F00106B00745
:104B100029D54FF0000E724670464F464FEA0B0300
:104B20000AFA00F1D3F808C011EA0C0F13D0996902
:104B3000D7F800C031F91210BCF83CC1614509DA60
:104B4000295CDDF800C04FF0010E6144FF2900DD53
:104B5000FF212954521C401C2028E1D3BEF1000F34
:104B600001D126F0020656B1FFF79DFEFDF79BFB33
:104B7000FDF78AFB08F10108B8F1640F98DB032602
:104B8000002000900220FFF737FCF00722D000E061
:104B900053E0002739463846CC465A460AFA00F315
:104BA000D2F8048013EA080F0ED05369DCF80080B5
:104BB00033F91130B8F83881434504DD235C13B173
:104BC00001275B1E2354491C401C2028E6D30FB943
:104BD00026F00106B00721D5002739463846CC46D5
:104BE0004FEA0B020AFA00F3D2F8088013EA080F22
:104BF0000ED09369DCF8008033F91130B8F83C81AD
:104C0000434504DD2B5C13B101275B1E2B54491C6B
:104C1000401C2028E6D30FB926F00206002E0AD049
:104C2000FFF741FEFDF73FFBFDF72EFB0098401C10
:104C300000906428A6DBBDE8F88F7F2234210AF0BB
:104C4000B4FAFFF730FEFDF72EFBFDF71DFB402603
:104C50000327002000900220FFF7CEFBF80731D099
:104C60004FF00008434640464FEA0B010AFA00F2B3
:104C7000D1F804C012EA0C0F1CD04A6940F6FF7C40
:104C800032F91320624506DB012E04DD225C4FF071
:104C90000108921B0CE0D9F800C0BCF838C162458D
:104CA00007DA225C4FF001083244FF2A00DDFF22C0
:104CB00022545B1C401C2028D8D3B8F1000F01D12E
:104CC00027F00107B80731D54FF0000843464046AA
:104CD0004FEA0B010AFA00F2D1F808C012EA0C0FF1
:104CE0001CD08A6940F6FF7C32F91320624506DB4E
:104CF000012E04DD2A5C4FF00108921B0CE0D9F86C
:104D000000C0BCF83CC1624507DA2A5C4FF00108DC
:104D10003244FF2A00DDFF222A545B1C401C20285D
:104D2000D8D3B8F1000F01D127F002076FB1FFF718
:104D3000BAFDFDF7B8FAFDF7A7FA002E05DD0098D9
:104D40007610401C0090642885DB0326002000902C
:104D50000220FFF751FBF00727D0002739463846DD
:104D6000CC465A460AFA00F3D2F8048013EA080F38
:104D70000ED05369DCF8008033F91130B8F838816F
:104D8000434504DD235C13B101275B1E2354491CFA
:104D9000401C2028E6D305E04C281000AC28100069
:104DA000B80210000FB926F00106B00720D5002781
:104DB00039463846CC465A460AFA00F3D2F80880FB
:104DC00013EA080F0ED09369DCF8008033F9113034
:104DD000B8F83C81434504DD2B5C13B101275B1E11
:104DE0002B54491C401C2028E6D30FB926F002069C
:104DF000002E3FF420AFFFF756FDFDF754FAFDF704
:104E000043FA0098401C00906428A1DB13E72DE9C9
:104E1000F05FA54E0024A54D30684FF07F03224679
:104E200090F830118F0706D50124490601D42B7064
:104E300004E02A7002E090F83F11297090F83011D8
:104E4000DFF86C824F0709D544F00204480602D40B
:104E500088F8003006E088F8002003E090F8401160
:104E600088F80010002C77D0342192480AF0C7F956
:104E70008F49FF20891C0870491E0870FDF704FA4D
:104E8000FDF711FA3068DFF83092B24690F8300141
:104E9000400662D54FF0100B00260220FFF7ACFA57
:104EA000E00723D0D9E904230020014606E000BF33
:104EB00033F91170874200DD3846491C9142F7DB17
:104EC000DAF80010B1F83621824202DA2878401E62
:104ED00008E0B1F84B11814206DB28785844FF28DE
:104EE00000DDFF20287001E024F00104A0072AD58E
:104EF00000200146D9F80C70D9F8183006E000BF40
:104F000033F91120824200DD1046491CB942F7DB1B
:104F1000DAF80010B1F83A21824205DA98F8001068
:104F2000491E88F800100EE0B1F84B11814208DBF1
:104F300098F800005844FF2800DDFF2088F80000A2
:104F400001E024F00204002C06D0FFF7ACFCFDF7D2
:104F5000AAF9761C202EA0DB65E54026002702205A
:104F6000FFF74AFAE0071AD0D9E9042C00200146DD
:104F700006E000BF3CF91130834200DD1846491CB1
:104F80009142F7DBDAF80010B1F83611814203DA0A
:104F90002878A0EB060010E050B124F00104A0072F
:104FA00025D500200146D9F81830D9F80C200DE09D
:104FB00028783044FF2800DDFF202870EFE700BF8D
:104FC00033F911C0844500DD6046491C9142F7DB8E
:104FD000DAF80010B1F83A11814205DA98F80010B9
:104FE000891B88F8001002E070B124F00204002C44
:104FF000B2D0012E00DD7610FFF755FCFDF753F916
:105000007F1C202FABDB0EE598F800003044FF2812
:1050100000DDFF2088F80000E9E770B5264C00208D
:105020002060FEF70CF86060FEF734F8A06060685E
:10503000042140086060201DFDF71EFF206104214F
:1050400004F10800FDF718FFE0600220FFF7D4F933
:105050001A482169806800EB41026261E26802EB54
:10506000410100EB4100A061FFF7D1FE0E4D286821
:1050700090F83001800601D5FFF7FAFCFFF7B3FB8B
:10508000FFF708FBFDF70FF909482968C01C0278F3
:1050900091F8FB1762F3030101702068BDE87040CE
:1050A00040F0020004F02DBC4C281000F70710005F
:1050B000F8071000B8021000AC281000B438100037
:1050C00010B5014610229948FEF7A2F998484168A8
:1050D0008020FBF7CDFF002803D0BDE81040FBF790
:1050E00091B910BDF0B5934D06460C4628684FF0B7
:1050F000FF3193B090F8B10000F00F00401C8140E8
:10510000CF436846FEF7B4F901208DF800008DF812
:105110000140286800F5867001788DF8121044F07F
:1051200005018DF801100297ADF81060AFF26F0124
:10513000019141788DF8161080787C4D8DF817001C
:1051400003246846FCF70FFE00218020FBF710FFC8
:1051500000218020FBF73AFF2878002804D0FDF7D3
:1051600090FB641E002CECDC13B0F0BD2DE9F04781
:10517000704D4FF00009DFF8B481286800F57070B9
:105180000478467887781AE049462046FFF7AAFF58
:10519000D8F8040007F078FD0146286890F80B2144
:1051A00012F00F0000D1012012094A43B2FBF0F0C7
:1051B00082B22146302004F011FCE01984B2B442DE
:1051C000E2DDBDE8F0872DE9FF5F4FF6FF764FF097
:1051D000000A93460F46804634465546DFF8549100
:1051E0001CE000BF38F815005146FFF77BFF4F4821
:1051F000406807F049FDD9F8001091F80B2112F032
:105200000F0100D1012112094243B2FBF1F080B23B
:10521000A04202D238F8156004466D1CBD42E1DBA5
:10522000ABF8006003980480BDE8FF9F2DE9F041D2
:10523000404D04468846286888B000F1D20690F8B0
:10524000D10006AB00F00F01491C05AA3046FFF75C
:10525000BAFF2A6892F8D000800721D5BDF8146003
:105260000121ADF8006002F1F20500234FF4803C0B
:105270006F4607E0E8563044604502D227F8110037
:10528000491C5B1C92F8D100C0F30210401C9842EC
:10529000F0DC002904DD06AB05AA3846FFF793FFD2
:1052A000BDF814002080BDF81810A8F8001008B050
:1052B000BDE8F0812DE9FC411F4E00235A1E19461E
:1052C0003068FBF705FA1D4C01A968466588FFF7B1
:1052D000ADFF184F3868B0F8FA10BDF804008142ED
:1052E00001D9218000E02080BDF800006080306896
:1052F000FBF7A6F9BDF80000854207D0386890F8A2
:10530000D000400702D56088FEF735FE0C48012426
:10531000294604700B480470BDF80020092004F0F1
:1053200016FB09480470BDE8FC810000C438100079
:105330000C3810004C2810002438100000381000E1
:10534000622810008F281000A82810002DE9F047CF
:105350000178FE4C01B1217001461022FC48FEF795
:1053600057F8FC4B186890F8CD17CA07F84901D0D8
:10537000CD6800E08D68427D6068F74E42430020B2
:1053800014E000BF97F8F0125FEAC17C08D08907EB
:1053900006D597F8F17235F810107F1C794301E0BB
:1053A00035F810101718401C26F817101F68797D63
:1053B0008142E7DC60684FF0000200F101006060AC
:1053C000797D01FB00F71BE090F8F0C25FEACC7832
:1053D0000ED05FEA8C7C0BD501EB020C90F8F10249
:1053E00035F81CC0401C0CFB00FCB81826F810C097
:1053F000881807EB020C35F8100026F81C00521C28
:10540000186890F815C09445DEDC61684FF001081B
:1054100001F10101616090F8B12008EB121490F8DD
:10542000F022D50705D0950703D490F8F1522C440B
:10543000E4B2A14223DA90F87A27D20719D090F883
:10544000CD378AB2DB0701D0C1F34F0290F8BA031F
:1054500000F00F00B2FBF0F100FB1121BC484C380A
:105460000029417802D041F0020101E021F002015F
:105470004170BDE8F047B6484C38FCF774BCD10722
:105480002FD091072DD4B0F8F2A2002522E0407D64
:10549000B149684301EB40018946002015E000BF97
:1054A00094F8F142012231F91060641C06E000BF5B
:1054B00002FB070C521C31F91CC066449442F7DC15
:1054C000A6EB0A0229F81020401C1C68677D874261
:1054D000E6DC6D1C186890F8B11008EB1111A942B8
:1054E000D5DC9E4841688020FBF7C2FD002803D030
:1054F000BDE8F047FAF786BFBDE8F0872DE9FF5F0A
:10550000DFF84CB24FF6FF7400258A46A046ABF197
:105510004C0BA9468D4E5BE08D484C38FDF7A8FF3B
:105520008C4A116891F8CD07C00701D0102300E024
:1055300002238BF80030009830F81530ABF82C308F
:105540009BF8013043F004038BF80130AFF20323E2
:1055500001F2C931CBF804300A788BF83220CA78CE
:105560008BF834204A788BF8372089788BF83810FC
:105570000327C6F8049000BF754886F800904C38A1
:10558000FCF7F1FB00218020FBF7F2FC00218020DA
:10559000FBF71CFD307820B1FDF773F97F1E002F5B
:1055A000EADC6D4802F0E5FB6A49096891F8C82316
:1055B00012F00F0100D101211209424390B2B0FB59
:1055C000F1F0A04203D20099044631F815806D1C19
:1055D0005545A1DB0299A1F8008003980480BDE83D
:1055E000FF9F2DE9F04105465A4888468CB0006877
:1055F0000AAB00F2823C90F8812300F2A23490F8CA
:10560000800302F00F01C2F30216C0F3400709AA9B
:10561000491C6046FFF772FFDFB1BDF8243001215D
:105620000020ADF800304FF4803C6F46761C07E058
:1056300022561A44624502D227F81120491C401C08
:10564000B042F5DB012904DD0AAB09AA3846FFF7B1
:1056500055FFBDF824002880BDF82810A8F80010D8
:105660000CB0BDE8F0817CB53D4E00235A1E1946B2
:105670003068FBF72DF83B4C01A96846E588FFF739
:10568000B0FF34480168BDF80400B1F8AC23824291
:1056900001D9A28000E0A080BDF80000E080208158
:1056A000854205D091F88013490701D5FEF7B5FC76
:1056B0002D49012008702D4908702D4900200860EF
:1056C0002C4908703068FAF7BBFFBDF80020294666
:1056D0000A2004F03CF97CBD2DE9F047DFF8748026
:1056E000DFF86C900025D8F80000A9F14C0900F211
:1056F000C33004884688077950E015484C38FDF7D8
:10570000B7FED8F8000090F8CD07C00701D01021EF
:1057100000E0022189F80010A9F82C4099F8011046
:1057200041F0040189F80110AFF2DF31C9F804102B
:1057300006490020486006484C38FCF714FB00215D
:105740008020FBF715FC0021802015E0C828100000
:10575000203910004C281000B49801200C3810009B
:105760002438100000381000622810008F28100024
:10577000E8291000DE291000FBF728FC094802F098
:10578000F8FA0246962D03DA074820F815206D1C1A
:105790002146312004F022F9E01984B2B442ACDD94
:1057A000AAE60000B4980120B01A01202DE9F041CA
:1057B000174604460D46002609E0E00703D03146AF
:1057C000384604F042F8761C6D084FEA340454EA77
:1057D0000500F2D1BDE8F08130B5034600204FF05E
:1057E000FF32012505FA00F40C4202D0521C9A4205
:1057F00003D0401C2028F5D3002030BDF0B50E4664
:105800000125074605FA06F2FE4C0F2FD4E91510C4
:1058100065D2DFE807F064434B081064641921295E
:10582000323A54585C003046FFF7D6FF8540A06AF4
:105830000543A56253E001463046FFF7CDFF8540A2
:10584000206C054325644AE03046FFF7C5FF8540DC
:10585000E06A0543E56242E03046FFF7BDFF854060
:10586000206B054325633AE001463046FFF7B4FF5D
:105870008540A06C0543A56431E03046FFF7ACFFDE
:105880008540606B0543656329E001463046FFF7BC
:10589000A3FF8540E06C0543E56420E03046FFF758
:1058A0009BFF8540606A0543656218E0014630460B
:1058B000FFF792FF8540E06B0543E5630FE0A06BC7
:1058C0000243A2630BE0206D0243226507E001461C
:1058D0003046FFF781FF8540606C054365642068B2
:1058E000401C2060F0BD10B501461022C648FDF7EF
:1058F0008FFDC64841688020FBF7BAFB002803D023
:10590000BDE81040FAF77EBD10BDFDF78BBB10B5AA
:10591000FDF77AFB4008400010BD2DE9F0478946AD
:1059200005464FF0FF34FDF77DFBB64F00231946C7
:10593000D7F804604FF0010C0CFA01F2024200D0DB
:10594000641CAC4206D1B9F1010F0AD020EA02036F
:105950000E462021491C2029EED318467E60BDE862
:10596000F0871346F4E72DE9F047894605464FF0E6
:10597000FF34FFF7CCFFA34F024600207B680146AF
:105980004FF0010C0CFA01F6164200D0641CAC4238
:1059900006D1B9F1010F08D022EA06000B46122108
:1059A000491C1229EED37B60D9E73046F6E72DE992
:1059B000F04198B0044688466846FDF759FD13A8A3
:1059C000FCF759FEFFF7A3FF8E4F40087865FDF7FF
:1059D00029FB20268E4DB865012C0AD0022C22D03E
:1059E000032C26D0042C29D0052C30D0062C4ED0E8
:1059F00064E0FDF77FFB0290FDF782FB039001203E
:105A00008DF800000C20ADF8100040208DF8120039
:105A10008DF8166091208DF817000298400878657F
:105A20000398B8654AE0FFF772FF0990FDF7FAFAAC
:105A300014E0FDF7F7FA01210A9003E0FDF7F2FA0E
:105A400000210A904046FFF78EFF099007E0FFF71C
:105A50005EFF099001214046FFF75FFF0A908DF835
:105A60000060286800F55A7081788DF83210C1788E
:105A70008DF8371001788DF8381041788DF839108D
:105A80008188ADF82C100089ADF82E0016E0FFF7E4
:105A90003EFF0990FDF7C6FA0A908DF8006028686D
:105AA00000F2613081788DF83210C1788DF83710AE
:105AB00001788DF8381040788DF8390000209DF875
:105AC00001108DF8140021F030018DF8150041F01F
:105AD0004A018DF834008DF833008DF80110AFF2D3
:105AE000F91103260191012C13D0092C27D00A2C7F
:105AF00025D000BF8DF856008DF858008DF857005E
:105B0000022C13D0032C11D0042C0FD0052C0DD057
:105B100015E0296891F889178DF8500041F00301CC
:105B20008DF84C103C21ADF84E10E3E72868B0F832
:105B30006E13ADF85210B0F87203ADF8540013A80C
:105B4000FCF7BAFD304C6846FCF70DF900218020C7
:105B5000FBF70EFA00218020FBF738FA20780028A6
:105B600004D0FCF78EFE761E002EECDC18B031E679
:105B70002DE9FC5F00210120FFF719FF224847684B
:105B8000FDF7B8FA0190FDF7BBFA0090042101A8D7
:105B9000FDF772F9064604216846FDF76DF9844663
:105BA00000200546DFF85CB0DFF864A000905CE000
:105BB0004FF00008C1465C462846DBF85810FFF756
:105BC0000BFE014601208840A16C08424CD1012403
:105BD0003BE000BF04FB0C51DAF8000037F911205C
:105BE00090F86703B2EB001F2EDA08F10108B9F153
:105BF000000F00D1A146721E944225D1B8F1010FC9
:105C000022D107E0D0281000303910000C381000E5
:105C10004C281000ACF10102954204D1611E012014
:105C2000FFF7ECFD0EE007EB4101B1F90220B2EB0A
:105C3000001F05DB35B131F9021CB1EB001F01DAA1
:105C4000002000E002208046641CB442C2DBA6EBC8
:105C50000901414508D829460220FFF7CFFD012060
:105C60000099A840084300906D1C6545A0DB012504
:105C70003BE000BF4FF0000844462CE0DBF840302A
:105C8000DBF8482000201A4311D0D9462046DBF823
:105C90005810FFF7A1FD014601208840D9F84810AF
:105CA000084203D1D9F84010084000D0012005FB7C
:105CB0000C4137F91120DAF8001091F86713B2EBB4
:105CC000011F07DA30B901200099A040084201D134
:105CD00008F10108641C6445D0DBB8F1000F03D063
:105CE000691E0120FFF78AFD6D1CB542C2DBBDE8CD
:105CF000FC9F2DE9F041E34C00200546E24FDFF820
:105D00008C83A0611EE029460520FFF750FE216923
:105D10000120BE6800EB410C36F91C10D8F80000D9
:105D200090F87703B1EB001F03D929460E20FFF747
:105D300065FD36F91C00A169884202DD36F91C00B8
:105D4000A0616D1C60698542DDD343E52DE9F0411A
:105D500000210620FFF72BFECB480025CB4EC94C77
:105D600087680EE0E0683168284437F9100091F840
:105D70006513B0EB011F03DD29460A20FFF73EFD46
:105D80006D1C20698542EDDB00250EE0A0683168BE
:105D9000284437F9100091F86513B0EB011F03DDBB
:105DA00029460B20FFF72AFD6D1C60698542EDDB5B
:105DB00010E52DE9F041B34C00200646206237E0A3
:105DC00031460420FFF7F3FDAF48002587682BE03C
:105DD000FDF728F901462846FFF7FEFC01460120A1
:105DE0008840216C08421ED1A849A068284409684F
:105DF00007EB400030F9040C91F87813B0EB011F69
:105E000007D931460820FFF7F9FC29460920FFF79A
:105E1000F5FCA068216A284407EB400030F9040C27
:105E2000884200DD20626D1C60698542D0D3761CFB
:105E300020698642C4D3CDE42DE9F041914C002085
:105E40000546914FDFF84482E0611AE029460320BD
:105E5000FFF7ADFDBE68B6F90210D8F8000090F863
:105E60007603B1EB001F03D929460720FFF7C6FCD4
:105E7000B6F90200E169884202DDB6F90200E0618C
:105E80006D1C20698542E1D3A4E42DE9F041002195
:105E90000220FFF78CFD7C487C4D7A4C876828688F
:105EA00090F86003000713D500260EE0E06829682B
:105EB000304437F9100091F87413B0EB011F03D987
:105EC00031460320FFF79AFC761C20698642EDDB01
:105ED000286890F86003C00613D500260EE0A0687D
:105EE0002968304437F9100091F87513B0EB011FA1
:105EF00003D931460420FFF781FC761C6069864295
:105F0000EDDB67E42DE9FC41614E00235A1E194682
:105F10003068FAF7DDFB4FF48010411209F04DF9BB
:105F2000FCF7C1F9FCF7B0F9FCF76EF9554C00200D
:105F30002060FFF7ECFC0090FDF774F8019004215D
:105F40006846FCF799FF0546042101A8FCF794FF79
:105F5000014600EB4500C4E90205C4E904514B4D7C
:105F6000286890F86003010701D4C00601D5FFF747
:105F70008CFF286890F86003800601D5FFF75CFF6E
:105F8000286890F86003000601D5FFF712FF286823
:105F900090F86003C00701D0FFF7D8FE286890F89A
:105FA0006003400601D5FFF7A4FE286890F860035F
:105FB000800701D5FFF7DCFD206800285DD0D4E91B
:105FC0000A359D43E562606AD4E90F1C9843A843F3
:105FD0006062676C21EA0C01B943E163A16B226D39
:105FE0009943A943256B22EA0C02A943A163A16C42
:105FF000BA438A43AB43A362226501220021FFF723
:10600000D5FB02220021E06BFFF7D0FB0322002129
:10601000A06AFFF7CBFB04220021206CFFF7C6FB30
:1060200007220021E06AFFF7C1FB08220021206B54
:10603000FFF7BCFB09220021A06CFFF7B7FB0A2287
:106040000021606BFFF7B2FB0B220021E06CFFF731
:10605000ADFB0C220021A06BFFF7A8FB0D22002155
:10606000206DFFF7A3FB0E220021606CFFF79EFB63
:106070003068FAF7E5FABDE8FC810021084603F034
:10608000E4FBF5E7D0281000303910004C28100050
:10609000243810006B49002008707047694E0024B6
:1060A000694DDFF8A881DFF8A8A1DFF8A8B1347046
:1060B0004FF0FF39287880B10128FBD140F27D7084
:1060C0000021FAF755FFFBF70BF8C1071ED000219E
:1060D0000120FAF77BFF2C70ECE70227012100205A
:1060E000FDF70FF800213846FAF742FF0121084674
:1060F000FDF707F8FAF7F4FF8007DBD5002140F23F
:106100007F70FAF763FF01202870D3E7010714D5E9
:1061100000210820FAF75AFF002347464A4619464D
:10612000D8F80000FAF7D4FA00234A461946B869AD
:10613000FAF7CEFAFEF78FFA15E041071AD50021DB
:106140000420FAF743FF002347464A461946D8F889
:106150000000FAF7BDFA00234A461946B869FAF773
:10616000B7FAFEF75AFFB869FAF76AFA3868FAF729
:1061700067FA9FE7C10606D500211020FAF726FF2F
:10618000FFF798F896E7810606D500212020FAF758
:106190001DFFFFF768FA8DE7C10507D500214FF411
:1061A0008070FAF713FFFEF7E1FF83E7810507D55B
:1061B00000214FF40070FAF709FFFFF78DFA79E735
:1061C000410606D500214020FAF700FFFFF79AFEAE
:1061D00070E7400599D500214FF48060FAF7F6FE8C
:1061E0001D4804601D48076804603846FDF71AFE24
:1061F000B80701D500F0E3FBA7F57060BF3801D107
:1062000005200AE0F80701D0152006E017F0420F3C
:1062100005D0DAF8000040F0060003F072FB1048E9
:106220000460CAF80040DBF8000090F84904C10798
:1062300001D180079DD5307800289AD008F015FE4E
:10624000347037E7A52810002C29100024381000DE
:106250005C2810004C281000E42910005028100081
:1062600058281000FE4900200870FE490870FE49B9
:106270000870FE490870FE4908700121FD4A11703E
:10628000FD4A1170FD49FF2208614861888008704D
:10629000C861CA80FA4A086248621268B2F852318C
:1062A0008B81B2F854214A818862887001F020B84D
:1062B00030B50024234605E030F913508D4200DD4F
:1062C000641C5B1C9342F7DBED48006890F86101A9
:1062D000A04201D2012030BD002030BDF0B5002524
:1062E0002F462C46DDF814C009E000BF30F91460D9
:1062F000B54203DA964201DD3546E7B2641C8C42B2
:10630000F4DB25B18CF8007001201D60F0BD002089
:10631000F0BD30B585B0DA4C01A8009020680025AA
:1063200003ABB0F95221017DD648FFF7D7FF50B13A
:1063300023689DF8040093F88A2102F00F0181423E
:1063400019D81B7D14E002A80090206804ABB0F9B6
:106350005421417DCC48FFF7C1FF68B123689DF807
:10636000080093F88A2102F00F01814203D85B7D77
:10637000591A814200DA150905B0284630BDFEB52C
:10638000BF4801AB5022006890F88911B0F98771BD
:1063900001F00F060C09B0F9855102A90091017DA9
:1063A000B848FFF79BFF0198B84201DD3046FEBDBB
:1063B000A84201DA2046FEBD401B311B4843791B31
:1063C00090FBF1F02044FEBD30B5B048AC4D0478F0
:1063D000286890F85101800703D5FFF7D0FFA4EBA0
:1063E0000004286890F85101400702D5FFF791FF9B
:1063F0000444002C01DA002402E00F2C00DD0F24FD
:10640000204630BD30B564290CD00023642407E059
:1064100030F913504D4395FBF4F520F813505B1CF5
:106420009342F5DB30BD70B5002364250AE0CC5CF7
:10643000642C06D030F91360664396FBF5F420F81F
:1064400013405B1C9342F2DB70BD2DE9F047002541
:10645000894629462F462E46A8462B460DE000BF0A
:1064600030F913C039F913400CFB0C660CFB0477B0
:1064700004FB0488654421445B1C9342F0DB87FBEA
:10648000020485FB013CC71A86FB020385FB0565F8
:1064900064EB0C04B0EB060C63EB050688FB02030F
:1064A00081FB0121851A63EB01086421A7FB01032D
:1064B00004FB0131002207FB02113346624608F05B
:1064C0000BFE0246A2FB070301FB073102FB04118E
:1064D0002A46434608F000FE002C00DA4042BDE8A0
:1064E000F08730B547F6F873002405E030F9145012
:1064F000AB4200DD2B46641C9442F7DB002405E030
:1065000030F81450ED1A21F81450641C9442F7DB53
:1065100030BD70B503460020024601EBD17408E09F
:1065200003EB420633F91250B6F90260AD1B284462
:10653000521CB2EB640FF3DB621008E003EB420580
:1065400033F9124035F9025C641B2044521C8A4224
:10655000F4DB70BDF0B587B00746494C03A8009046
:1065600020689C468E461646017D002504AB0FFA36
:106570008CF27046FFF7B2FE01283BD102A80090D2
:10658000206805AB32B2417D3846FFF7A7FE0128EF
:1065900030D1DDE9041081424FF0640203DD504345
:1065A00090FBF1F102E0514391FBF0F1206890F88B
:1065B00092218A421EDD9DF8081019B990F89121A8
:1065C000D20716D0427D521E8A4203D190F8911113
:1065D00089070ED59DF80C1019B990F89121520732
:1065E00007D5027D521E8A4204D190F8910100071E
:1065F00000D4012507B02846F0BD2DE9FC41204C10
:1066000084460F4620680025164690F890114907E9
:1066100079D5009690F89311427D0B091C4960468C
:1066200001F02EFF0096206890F89311027D0B096F
:1066300017493846243101F023FF206890F8901163
:10664000090631D5407D43F6FF76CDE90060104A5A
:1066500033461049104602F06AF82068007D1BE0BE
:10666000712810008D2810008E281000722810004C
:10667000732810008F281000922810003029100075
:106680004C281000A02001207C200120932810001D
:10669000401C0120C2160120CDE90060FD4A3346AE
:1066A000FD49104602F043F8012700972068FB4996
:1066B000437DB0F89E21F748243802F04FF8064693
:1066C00000972068F449037DB0F89C21F14802F05E
:1066D00045F807462068EF49F04A437DEC31A1F5C3
:1066E000887001F09CFF2068EB4AED49037DE94882
:1066F00001F095FFEB490022EB48012E06D0026223
:10670000012F14D042622846BDE8FC81036A5B1C5D
:106710000362266896F8936106F00F069E42EFDA50
:1067200002620B68012543F040030B60E8E7436A0F
:106730005B1C4362246894F8934104F00F049C426C
:10674000E1DA42620868012540F040000860DAE7BB
:10675000F0B40446D5480B46802100680D4690F8F9
:10676000680110B10146C0F58075CF480089032843
:1067700005D22146F0BC52001846FCF749BE002065
:106780000FE000BF33F9106034F910704E4307FB7F
:106790000566F71706EB176646F30F2623F8106019
:1067A000401C9042EEDBF0BC7047F0B50024BF4DBA
:1067B0000FE030F8146031F81470012B0CD0F61B88
:1067C0002F6897F86D717F4206EBC70620F81460BA
:1067D000641C9442EDDBF0BD3E442F6897F86D7168
:1067E000F2E72DE9FC47B04D80460026288998B98C
:1067F0002422AA49AE48FCF70BFE4022A649AD4828
:10680000FCF706FEA3482421643008F0D6FCA1481A
:106810004021883008F0D1FC28890127A34C0328A7
:1068200002D2A548077014E013D92168B1F86B2192
:1068300082420ED94B7D97499D4A6431974801F0B9
:10684000EEFE206893499B4A037D8831924801F00F
:10685000E6FE206890F85011427D090710D590F8A7
:106860008D11CDE9001290F88B31944A8B49404646
:1068700001F05DFF20688749427D88398F4802E03A
:10688000844940468839FFF763FF2068834A90F8BF
:106890005011437D09078A4901D5884800E04046E8
:1068A00001F0BDFE20687D4A8549437D79488838DE
:1068B00001F0B5FE206890F85011C90610D5427D50
:1068C00090F896127E48FFF79DFD216891F85001DF
:1068D000C00605D54A7D01F51C717948FFF7A3FD77
:1068E0002268B2F85411B2F86901B2F86B41014460
:1068F0000BB229898C4201D2184403B2002004460D
:10690000DFF8C0C1DFF8B891527D1CE039F9108082
:10691000984515DD761C022E13D96878401C40B2CC
:106920006870002804DD68488CF800706C7007708F
:1069300047F6FF70814201D2491C2981BDE8FC87DE
:106940000026401C00B28242E0DC6C708CF80040F3
:10695000EEE7034610B50020024603E033F912408B
:10696000521C20448A42F9DB10BDF0B54F4C0F4653
:1069700000252168497DFFF7ECFF06462068017D70
:106980003846FFF7E6FF236801460024D3F89C72DF
:106990004548B74203D38F4201D3C4620DE0C16AB8
:1069A000491CC16293F89B228A4206DC3D490125BD
:1069B0000A6842F400520A60C4622846F0BD3B48AF
:1069C000006890F89011890606D5374901220A70AF
:1069D00090F895211209CA6190F8F002C00701D021
:1069E00002F09ABD70471CB52F490020098901B9F2
:1069F00001201021CDE900102C4C29490F232068DB
:106A00006431427DA1F1240001F05DFD244924227E
:106A10004031A1F18800FCF7FBFC214924226431BC
:106A2000A1F18800FCF7F4FC20681D49437DB0F912
:106A3000AE216431A1F1240001F0FFFD012800D056
:106A400000201CBD2DE9F041184C00231A46216896
:106A500018461E4E1E4F0D7D0EE000BF36F9101079
:106A600037F910C0B1EB0C0100D5494289B28B4215
:106A700001D20B4682B2401C8542EFDC5908092046
:106A800002F082FF236800210A460846114D124E8B
:106A90005C7D30E0641C0120E6160120C216012056
:106AA000741D01205C281000302910004C281000B3
:106AB000261701204A170120D42910007039100030
:106AC0007C200120732810008F28100034980120AA
:106AD00074980120EC9701201098012035F91030AE
:106AE00036F91070DB1B00D55B429BB2994201D294
:106AF000194682B2401C8442F0DCBDE8F0414908EE
:106B00000A2002F041BF70B5FF4A0020034640F260
:106B1000FF711268FD4DFE4C05E000BF25F8101016
:106B200024F81030401C567D8642F7DC0020F94CDA
:106B3000F94D04E024F8101025F81030401C167DA3
:106B40008642F7DC70BD2DE9F041F44C06460D4657
:106B5000A078012844D1A06A08B9FFF7D4FFEA4819
:106B60000022EA49DFF8A8C3076812E031F91230C1
:106B700036F91200834200DA184621F812003CF977
:106B8000120036F91230984200DC18462CF8120038
:106B9000521C787D9042E9DC0020DE4BDE4A12E098
:106BA00033F9106035F910108E4200DA314623F8BF
:106BB000101032F9106035F910108E4200DD3146A8
:106BC00022F81010401C397D8142E9DCA06A401C8B
:106BD000A062642804D3FFF735FF0020A070A062F4
:106BE000BDE8F0812DE9F34F85B0CD4C4FF0FF317A
:106BF0004FF0000A039120780125CA4ED14657462E
:106C0000D04601281ED0C048DFF81CB3006890F8B9
:106C10002020D2061CD590F82520C44803889A422B
:106C200016D2A0F80080DBF80010C14841F0220124
:106C3000CBF800104168A802FAF7E9F9357007B0FF
:106C4000BDE8F08F357000F053FB84F80080F6E764
:106C5000B84C00235A1E1946E068F9F739FD0023A5
:106C60005A1E19462069F9F733FDB348AB4C00783A
:106C700001287DD02089012805D9A348AF490068A3
:106C800090F880010870002020813278DDE905014C
:106C9000FFF7B3FC06469C48006890F87001400678
:106CA00006D5206A002802DC606A002800DD012782
:106CB000FFF78AFB01909B48DFF84C82A0490078DF
:106CC0000090D8F80000019B427D059801F0D8FBA8
:106CD00094489B49019B00780090D8F8000024312B
:106CE000027D069801F0CCFBD8F8000090F8501116
:106CF00009071CD590F88D110023427D8DE80E0008
:106D00008F4A90F88B318F49104601F0ACFCD8F8CF
:106D10000000002390F88E11027D8DE80E00884A55
:106D200090F88C3124328849104601F09CFC7D4952
:106D3000DFF8D48100200870D8F80000814A834928
:106D4000437D7F4801F06BFCD8F800007E4A804903
:106D5000037D7B48243001F062FCD8F8000090F8F5
:106D6000910100063ED57A497848FFF7FEFD00E024
:106D700002E0012834D035E06348006890F8510102
:106D8000C00605D5FFF72FFE72490128087011D003
:106D90003278DDE90501FFF730FC01280DD00598B8
:106DA000FFF71FFD634C2069F9F74AFCE068F9F72B
:106DB00047FC44E784F8018010E06748057084F8D8
:106DC00001803570DBF80010594841F04201CBF8E2
:106DD000001041684FF48060FAF719F93570E1E767
:106DE0004FF0010ADFF84C81D8F81000F9F728FCC1
:106DF000D8F80C00F9F724FCDFF80C81D8F8000073
:106E000090F8901109074FD54D49427DC8314F4840
:106E1000FFF767FBD8F800004949427DC83100F50B
:106E20007470FFF712FB6061D8F80000417D4448A0
:106E3000C830FFF76EFB8646A0616069009032287B
:106E40001CDD3F48D8F80020C830B0F90030B2F857
:106E500054118B4207DD92F815C000EB4C0C3CF945
:106E600002CC8C4509DC49428B4207DA527D00EBAB
:106E7000420030F9020C884200DA0127D8F80000FD
:106E8000009990F894218A420EDAB0F8AC2172454C
:106E90000ADA90F89001400601D54FF001092F4819
:106EA000016841F480710160D8F80000C44690F890
:106EB0005011C9060DD5427D90F896122348FFF770
:106EC000A1FADCF80000027D90F8DC122048FFF700
:106ED00099FADCF80000E04690F89011890743D554
:106EE000B0F85231B0F8542119491848FFF732FB75
:106EF000012805D181461948016841F400710160FB
:106F0000D8F800002CE000004C281000EC9701207D
:106F10001098012034980120749801203029100025
:106F2000922810008F2810005028100060281000B0
:106F30000C38100024381000632810007429100049
:106F4000DC1B0120C2160120E6160120703910005A
:106F50009439100072281000732810005C2810006B
:106F600090F89001800705D4D8F8000090F89011AF
:106F700009070ED5B9F1010F09D1B4F904000028B1
:106F80000CDB401E00B2A080002807DC0126D8F8E8
:106F9000000090F8950100F00F00A080D8F80010D4
:106FA000C44691F85001C0060DD54A7D01F51C710B
:106FB000BF48FFF738FADCF80010BE480A7D01F53B
:106FC0002871FFF730FADCF80000E04690F8501125
:106FD000090610D50095437DB74AB849B44801F079
:106FE000F5FA0095D8F80000B34AB549037DB148D9
:106FF00001F0ECFA0DE0407DAD494200AF48FCF7EE
:1070000007FAD8F80000AB49007D4200AC48FCF715
:10701000FFF9D8F8000090F89111C9062BD503A903
:107020000091427DB0F8AC31521E0021A04801F021
:1070300068FA012815D10398012805DBD8F800105B
:107040004A7D921E824211DAE0880127401E00B27A
:10705000E08000280FDA9B480126016841F4807126
:107060000160D8F8000090F8950101E091F89501D1
:1070700000F00F00E08092499048FFF764FDD8F8D7
:10708000000090F85111C9070DD0B0F95E21417D83
:107090008A4801F055FBD8F80000B0F95E21017D67
:1070A000874801F04DFBD8F8000090F850114907CF
:1070B00012D50095804A437D0A3A83497F4801F002
:1070C00085FA0095D8F800007B4A8049037D0A3A8A
:1070D0007B4801F07BFA0DE0407D784942007A4818
:1070E000FCF796F9D8F800007549007D4200774812
:1070F000FCF78EF9D8F8000094F800C0B0F85211EF
:10710000B0F85421BCF1010F07D0DFF8C4C19CF8DE
:1071100000C0BCF1010F0DD016E0B0F898C1BCF171
:10712000000F00D06146B0F89AC1BCF1000F0BD03F
:10713000624609E090F857C1A1EB0C0190F856C1E6
:1071400089B2A2EB0C0292B2DFF888C19CF800C0B1
:10715000BCF1000F07D090F8A3C1624490F8A4C11D
:1071600092B2614489B20FFA81F9A4F80C9011B27D
:107170006181427D5448FFF79BF88446D8F80000AF
:107180004946027D5148FFF793F85349DFF8509183
:10719000BCF1010F81F800C05049087001D10128ED
:1071A0000BD05049002089F80000087020690028A1
:1071B0001BDD401E20610CD017E0454889F80050C7
:1071C0000078012811D1D8F8000090F897012061CB
:1071D0000BE0D8F8000090F89001C00605D53948BA
:1071E000016841F08001016002E0BAF1010F0DD1A8
:1071F000DBF800103C4841F02201CBF80010416858
:107200004FF48060F9F703FF38480570012E0CD168
:10721000DBF80010344841F04201CBF8001041681F
:10722000B002F9F7F4FE31480570D8F80000454681
:1072300090F89011890624D52178012921D1E1699E
:10724000002915DD427DB0F954111F48FFF730F8D1
:1072500006462868027DB0F952111C48FFF728F84D
:1072600006B100B94FB1286890F895010009E061B6
:1072700099F80000012807D017E0E069401EE0619E
:10728000F6D100202070F3E72868B4F9041090F8D4
:10729000950100F00F00884207D1002F7FF4D7AC92
:1072A0000A49094800F05EFCC9E400F094FAC6E41B
:1072B00070391000943910006A291000D439100078
:1072C000F83910005C2810007C200120A02001204B
:1072D0008C281000752810008D2810008E281000B2
:1072E00071281000732810000C3810008F2810002F
:1072F000FD49002001220870FC498860C8600861CF
:107300004861886148708A70F94A1070F94A0870BB
:107310001070C8708880C8807047F7490A68B2F852
:107320006411814201DB00207047B2F8662182427D
:1073300001DCFF207047521A401AC0EB002090FB7E
:10734000F2F0704730B5EC4A00241268937EDD07F6
:1073500092F882310BD0834217DC158BEB1A8342F3
:1073600013DB92F8830188420FDCD28A0AE0834261
:107370000BDCD58AEB1A834207DB92F88301884243
:1073800003DC128B101A884200DA0124204630BD3B
:107390002DE9FE4314460D460646072B08D0D34878
:1073A000092B016906D0316041692960806910604C
:1073B000BDE8FE833288ADF802202A88ADF80020AF
:1073C0002768ADF806108146808AADF8040001AA4E
:1073D000694602A806F09EFE02A806F093FEDFF8BA
:1073E00018830346D8F800C09CF87401BCF87621D5
:1073F00000F00F01BCF878C1000952430CFB0CFCF3
:1074000093420BDD634501DB084607E09B1A411AF6
:107410004B43ACEB020193FBF1F1401ABDF9023092
:10742000C0F11002D9F810C0534300FB0C331B0904
:107430003360BDF900305343D9F8142000FB02300B
:1074400000092860D8F800001022D9F8181090F828
:107450007501A2EB10127A43000900FB0120001114
:107460002060A5E75FF0000200EB82035B6840F854
:107470002230521C052AF7DB416170472DE9F04F9D
:10748000002793B080463E463D46FFF7EBFF0021C4
:1074900058F821000744484300FB0155491C0644A5
:1074A0000629F5DB914C09971C3460680A90A068A6
:1074B000CDE90B0620690D906069CDE90E05E06904
:1074C0001090206A119009A8FBF7F8FC83460391FD
:1074D0002068CDE90907A0680B90E068CDE90C06AB
:1074E00060690E90A069CDE90F05206A119009A886
:1074F000FBF7E4FC8146206809906068CDE90A0743
:10750000E0680C902069CDE90D06A0690F90E06954
:10751000CDE910058A4609A8FBF7D0FC0326A9FB94
:1075200006570A460AFB06710926A0FB0637002407
:1075300009FB041402FB0672002100FB0120EA187B
:107540004441039912EB0B0061414FF47562002333
:1075500007F0C2FDC8F80C0013B0BDE8F08F30B5DD
:10756000654A01241268937EDD0792F87A310BD0C8
:10757000834217DC158BEB1A834213DB92F87B01F5
:1075800088420FDCD28A0AE083420BDCD58AEB1AF0
:10759000834207DB92F87B01884203DC128B101ACE
:1075A000884200DA0024204630BD2DE9F0418AB03F
:1075B0001C460694DFF84081CDE900120546D8F854
:1075C00000000026494C90F8700137460B46C00772
:1075D00028D0082D26D094F90300062819DB11B213
:1075E00018B2FFF7BCFF00284448009909D0FFF704
:1075F00045FF0090414801991830FFF73FFF019087
:1076000010E0FFF72FFF3D4801991830FFF72AFFE0
:1076100008E0401C394940B2E07041F82030183190
:1076200041F820202B4606AA01A96846FFF7B0FEC4
:10763000072D02D0092D08D02EE000982061019876
:10764000606106980126A06127E0D8F8001091F843
:107650007001400720D522690098101A00D54042D9
:1076600091F87C3198420BDA63690198181A00D5B9
:10767000404291F87DC1604502DACDE9002300E087
:107680000126A2690698101A00D5404291F87E1191
:10769000884201DA069200E00126D8F80000C446CC
:1076A0004FF0000890F87001000641D5082D3FD03A
:1076B000019801B2009800B2FFF744FE0746012886
:1076C00036D1DCF8000090F87011090730D4072D8E
:1076D00018D00B49097841B390F8A601401CA0606E
:1076E00000200AB0BDE8F0818C2810007429100039
:1076F00071281000732810004C2810004039100029
:1077000075281000FB4A82F8008090F89001C007AD
:10771000E6D0F948016841F022010160F74841686C
:107720004FF48060F9F773FCDAE790F87301D5E75E
:1077300046B100982061019A6261069EA661012F00
:1077400002D030E00120CCE7DCF8001091F8703175
:107750001B0728D58B7EDB0791F882310FD083423F
:1077600000DD0093088BC01A009B984200DA00905D
:1077700091F88301904200DD0190C98A0EE08342B6
:1077800000DD0093C88AC01A009B984200DA00907E
:1077900091F88301904200DD0190098B081A01994C
:1077A000884200DA0190CDF814800098ADF81600F8
:1077B0000198CDF81080ADF8140043468DF81050B4
:1077C0003046FFF7AAFD8DF812008DF8133004A89B
:1077D00001F064FFB6E7CA4810B50178C9480068EF
:1077E00049B190F9A611C3480278C748012A05D0CB
:1077F0000021C1600DE090F97311F4E78268521C1A
:1078000082608A4208D300231A4619460820FFF7EF
:10781000CCFEBDE810406BE510BDF0B50746DDF8C5
:1078200014E037F912404FF0FF30744501DA0024BC
:1078300000E01046012517E0561B07D437F916C0A3
:10784000F44503DDA44501DD304664465619A1F137
:10785000010C664507DC37F916C0F44503DDA44585
:1078600001DD304664466D1C9D42E5DDF0BDF0B59E
:1078700000240125A1F101060BE0571B02D430F9C9
:1078800017703C445719B74202DC30F917703C447A
:107890006D1C9D42F1DD012A02DB891E8A4200DD5A
:1078A000640030F912002044F0BD2DE9F047954DF9
:1078B00014469A462E6830F91420814602FB04F0E3
:1078C0000123A1F1010196F862C117E0E51A08D47D
:1078D00039F91570B6F85E81474502DB07FB0500F4
:1078E0003A44E5188D4208DC39F91570B6F85E8126
:1078F000474502DB07FB05003A445B1CB3EB1C1F4A
:10790000E4DD4A4380FB0A01D31707F0E5FB00B230
:10791000BDE8F0872DE9F04F8FB00C468246174640
:1079200099460026182108A8189D07F068FC2DB973
:107930007448006890F8620100F00F057A1B07EBAD
:10794000050300D50022651EAB4200DD631E08A9B9
:107950005046FBF721FB6D484FB1AF4232D1694928
:10796000096891F85111890613D54E466EE06549B4
:10797000096891F85111890668D4BAF904100160B8
:10798000BAF900104160BAF902104B460122816039
:1079900010E00AEB440100EB84000C3831F9062DAD
:1079A0008260B1F904204260B1F902107F1C4B469D
:1079B0003AB20160611E554802F0AEFC99FBF5F148
:1079C000461A43E0DDE90CB0B0F1000841DADDE928
:1079D000082352EA03003CD0DDE90A01019104903A
:1079E000002936DB4748066896F85001400611D555
:1079F0005846414607F070FB002800DA404296F8EE
:107A00006311884206DA4B463A4621465046FFF754
:107A10004CFF1AE01BEB0B01A1FB052448EB08000F
:107A200000FB0540EB1701FB030304980199464254
:107A3000A6FB0907002464EB010404FB09714FEA6B
:107A4000E97506FB051107F047FB064630460FB007
:107A500083E5B8F1000FD6DADDE908010843D2D09A
:107A60000B980028CFDBF1E738B5264D049C2D6834
:107A700095F85051AD0603D50094FFF74BFF38BD84
:107A800001B0BDE8304010E72DE9F04700249A46E8
:107A9000CE1E81462346A44627462546022A03DBFE
:107AA000B24201DC104633E70020491E08E000BF67
:107AB00039F91080B8F1000F01DDC4447F1C401C6F
:107AC0008842F5DB9CFBF7F7022A21DA10460DE02D
:107AD00039F91060BE4203DA3CB90446002304E0E1
:107AE0001CB19E4201DD33460546401C8842EFDB57
:107AF00022E000008C281000502810000C381000E4
:107B0000752810004C28100074291000F83E100051
:107B1000B24211DD10460DE039F91010B94203DA16
:107B20003CB90446002304E01CB1994201DD0B4638
:107B30000546401E0228EFDC534500DA154628466C
:107B4000E6E630B5044630F911300020491C06E065
:107B500034F911509D4201DD2B460846491C9142E3
:107B6000F6DB30BD2DE9F34F6D4C85B0226892F8FD
:107B70008431567D03F00F056F4206EB470606F091
:107B8000FF0B167D1A0900EB45005342059006EBEA
:107B9000430301EB4200DBB203931A460021069037
:107BA000FFF7CFFF05465A4600210598FFF7C9FFAA
:107BB000064620685B4F90F87001800607D5B7F93C
:107BC00000302A4603990698FFF75EFF05462068B5
:107BD000DFF854A190F87001C00607D5BAF900305B
:107BE000324659460598FFF74FFF0646DFF83C91AD
:107BF000DFF83C8199F80000012828D1206890F82E
:107C00006001010723D0010921D0B7F900100091CC
:107C100000F00F03B8F9042003990698FFF7FDFD63
:107C20000746BAF9000000902068B8F906205946C6
:107C300090F8600103090598FFF7EFFD002F01DBC5
:107C4000002802DAFFF7C7FD01E03D4606462FB2E5
:107C500032B2A8F80470A8F8062000260096206822
:107C60005946B0F918300598FFF7FEFE00960290CD
:107C700020683A460399B0F916300698FFF7F4FEEB
:107C80000190206890F87001800704D5022202A9B3
:107C900001A803F03DFF02A901A8FBF777FC01232F
:107CA0002A4603990698FFF7E2FD0346214800782B
:107CB0000028206816D090F9A52198F800004146C8
:107CC000401E40B288F80000002806DB206890F8CB
:107CD0007F01104442B2FF20087099F80000CD687F
:107CE00018B104E090F97221E7E76D1CCD60954270
:107CF00013D340F2FF12CA60C8F8086030B10920FF
:107D0000DDE90112FFF751FC28B106E0012089F8F6
:107D100000000720F4E7FFF75EFD012007B01CE438
:107D20004C2810003C2910003A2910008C28100023
:107D30007429100075281000E548E64A0068B0F87C
:107D4000AC139180E44990F8B10308817047E2498F
:107D50000020DF4A8880C880C86048801268DF4BF6
:107D600092F85C2112091A7008610870DC490870E9
:107D700070472DE9F04395B0814602AF482138465F
:107D800007F03DFAD2480123016891F8B1204C7DFB
:107D900091F8A01103EB1216890715D5002580462E
:107DA00010E000BFD8F8001005FB04F009EB40001C
:107DB0004A7D91F88B31CDE900324946024600F008
:107DC000B6FC6D1CB542EDDB002010E000FB04F2B8
:107DD000002109E002EB010C57F8215039F91C3061
:107DE0002B4447F82130491CA142F3DB401CB04230
:107DF000ECDB002007E000BF57F8201091FBF6F104
:107E000047F82010401CA042F6DB00200121A4F11D
:107E1000010517E04FF0000C63460BE003FB04186C
:107E200039F9182057F82180B2EB080200D55242E8
:107E300094445B1CB342F1DB9CFBF6F2824200DD12
:107E40001046491CA942E5DBB0F5803F04DB4FF644
:107E5000FF7015B0BDE8F08380B2FAE730B59C49F9
:107E60009E4B096891F85021920725D59C4A1278BB
:107E70004AB191F8A74104F00F022509B1F8A841D1
:107E8000B1F8AA1107E001F5AC710C7904F00F020A
:107E900025090C884988A04201DC1A7030BD88424F
:107EA00001DB1D7030BD001BAD1A6843091B90FB40
:107EB000F1F01044187030BD91F85C0100F00F0033
:107EC000F8E72DE9F041824D296891F88023B1F857
:107ED000AC33D4077F4A3ED091F8AF4304B90124B4
:107EE000968891F8AEC3F71A07FB0CF797FBF4F4EA
:107EF000B1F8AA7337442744774CB8420BDD794870
:107F00000026E66041682020F9F781F8E6802868BD
:107F100090F8B10306E0864202D9714D2D7825B163
:107F200091F8B1032081BDE8F0816F4909780029FB
:107F3000F9D1B4F90810002901DD491E21812189F8
:107F40000029F0D1B11E814200DA01468B4200DDEA
:107F500019469180E7E79380E5E75D4A10B514681C
:107F60000021B4F8A121824204D294F8B000800725
:107F700000D5012158485A4B0278914211D1197805
:107F800091420AD0584C2478224307D00169491EF7
:107F90000161002901DC0078187010BD01700169D1
:107FA000F7E739B194F8B22002610170002AF4DCDD
:107FB000197010BD94F8B320F6E7454910B509686B
:107FC00091F8B010CA06444918D5484A14780A46B0
:107FD000D388C3EB03125200012C05D0C41A002C25
:107FE0000CDC414C247824B102EB4000C0F34F106C
:107FF00004E0C3EB83121044C0F38F10C88080B23A
:1080000010BD10B5FFF7B5FEFFF7D7FF324CA080CB
:10801000FFF7A3FFA088FFF721FFA088BDE810406D
:108020004FE7F0B431490B782B494A88B3B1322A73
:1080300001D2521C4A80264A0125136893F8B140A8
:108040005B7D05EB1415CC6894FBF5F605FB164437
:10805000274E634306EB430700230CE0012AEAD9CD
:10806000521E4A800022CA60E5E700BF30F813C004
:1080700027F813C05B1CD2F800C09CF815C09C45C3
:10808000F4DCCB685B1CCB60136893F8CD77FF07FB
:1080900007D05B7D641C5F00634306EB4304002351
:1080A00007E0C8680CE0FE1830F8166024F813608A
:1080B0005B1C1668767D9E42F5DCC868401CC86073
:1080C000A84202DBF0BC0A489BE7F0BC7047000006
:1080D0004C28100000381000B4291000932810001C
:1080E000752810000C38100071281000632810004B
:1080F0003C1E0120CA490020886048600860C949C8
:108100000870704710B500230BE000BF30F9134032
:10811000002C00DA64428C4201DD012010BD5B1CA2
:108120001BB29342F2DB002010BD70B5BE4CBF4ABB
:10813000BF492068437DBF4800F071FA2068BE4AFD
:10814000BE49037DBE4800F06AFA2068427DB0F95E
:108150009812B748FFF7D6FF05462068027DB0F9B0
:108160009812B648FFF7CEFF0022AD49012803D090
:10817000012D01D00A6070BD0868401C08602368AA
:1081800093F89A328342F6DCAE48036843F4805396
:108190000360AD480A60016841F022010160AB480C
:1081A0004168BDE870404FF48060F8F730BF70B5AB
:1081B0000546002003460BE035F9134031F9136002
:1081C000A41B00D5644224B2A04200DA20465B1C06
:1081D0009342F1DB70BD2DE9F05F9D4800784007C8
:1081E00078D59C48904E8E4C01783068002731B38A
:1081F0006760A76090F82C10B0F82F90B0F833505B
:108200004FEA111A01F00F0B427D93499348FFF793
:10821000CEFF804630689249027D9248FFF7C7FF43
:108220003268804BB2F854C1B8EB5C0F04DCB2F892
:108230005211B0EB510F1EDD012018701CE0616877
:10824000491C616090F82A20B1EB121F00DD6760C5
:10825000A16802F00F02491CA1608A4200DAA760FF
:1082600010F82B1FB0F80290C5884FEA111A01F0E0
:108270000F0B2B38C8E71F70774F794B0020B6469D
:108280004CE0794A00211278012A09D0774A32F964
:1082900010C037F9102094450DDAA2683AB11CE0FD
:1082A000724937F8102031F81010891A01E0CBF12B
:1082B000000109B211E0D4F80480B8F1000F0CD12C
:1082C000ACEB02020FFA8AF14A4506DDAA4202DD52
:1082D00029B202E082E00FFA89F196F88023520772
:1082E00016D500220CE000BFDFF848C102EBC2083F
:1082F0000CEB880C521C3CF8108088442CF8108041
:1083000096F880834FF0010C0CEB981C9445EBDC45
:1083100037F81020114427F81010401CDEF80060D8
:108320007246717D8142ACDC002048E04E4E002157
:108330003678012E09D04E4E36F910C033F9106050
:10834000B4450DDAA6683EB11BE0494933F8106028
:1083500031F81010891B01E0CBF1000109B210E0E7
:10836000D4F80480B8F1000F0BD1ACEB06060FFA7D
:108370008AF14E4505DDAE4201DD29B201E00FFA7A
:1083800089F197F88063760713D500264FF0010E28
:1083900009E0DFF8ACC00CEB861C761C3CF81080C2
:1083A00088442CF8108097F880830EEB981CB44515
:1083B000EFDC33F81060314423F81010401C1768CC
:1083C000397D8142B2DC97F89101000606D597F815
:1083D0008003400702D5BDE8F05FA6E6BDE8F09F48
:1083E000114810B5006890F82000C10716D0214947
:1083F0000978002912D12049097809B180060DD5E4
:108400001E4C00235A1E1946E068F8F761F9FFF781
:10841000E2FEE068BDE81040F8F712B910BD0000B8
:10842000C8291000A72810004C2810001A18012095
:10843000703910008A1701203E190120943910006C
:108440003E1801205C281000502810000C38100045
:10845000D829100063281000C2160120DC1B01205F
:10846000E6160120001C0120D4291000E219012089
:10847000061A012066281000712810002438100008
:10848000F0B40C4601460498C3F11006012801D04F
:10849000002014E02046F0BC5200FAF7B9BF00BF3C
:1084A00034F9105031F910705D4307FB0655EF1792
:1084B00005EB177545F30F1524F81050401C90423A
:1084C000EEDBF0BC7047F0B40C460146DDE9046019
:1084D000F51A012801D0002010E02046F0BC52001F
:1084E000FAF796BF34F9107031F910C05F430CFBF6
:1084F000057797FBF6F724F81070401C9042F1DBEB
:10850000DFE7F0B50646002004460546521C059FED
:108510000AE000BF36F911C09C4504DDA44502DD28
:1085200064460D460120491C9142F3DB3D60F0BDDD
:10853000F0B54FF0000C67466646654664460EE0AF
:1085400031F914E0BEF1000F03DDF44406F1010639
:1085500003E002DA774405F1010504F101049442D5
:10856000EEDB9CFBF6F697FBF5F70024DFF844C240
:1085700029E08BB131F91450002D13DD30F814507F
:1085800035442DB220F81450DCF800E0BEF858E471
:10859000754517DD354413E030F8145031F814E018
:1085A00075440DE00EDA30F814503D442DB220F839
:1085B0001450DCF800E0BEF85CE4754502DA3D4496
:1085C00020F81450641C9442D3DBF0BD2DE9F04335
:1085D00091460022DDF81CC018E000252E462C46EE
:1085E00002EB0407BF1E08D49F4206DA30F9178059
:1085F00039F9147008FB07553E44641C052CEFDB69
:10860000BCF1010F06D021F81250521C9A42E4DB53
:10861000BDE8F08395FBF6F421F81240F5E770B55C
:10862000002407E032F8145030F81460AD1B21F834
:108630001450641C9C42F5DB70BDF0B500252C463F
:1086400009E000BF31F9146030F91470F61B96424E
:1086500000DD6D1C641C9C42F4DB022D01D901205D
:10866000F0BD0020F0BD2DE9F04F8946DDE90A6735
:10867000012447F6F8719A464D429346A4460023DA
:10868000DDF824E018E000BF30F8132039F813803B
:10869000D21BA8EB020212B2914200DD11469542B4
:1086A00000DA1546002A02DA4FF0000402E001DD8C
:1086B0004FF0000C03F10103B342E5DB54EA0C0276
:1086C00006D0012C01D02CB108E0BCF1010F05D17E
:1086D000002103E0BCF1010F00D1294600252C4602
:1086E0002A4611E030F8123039F812C0DB1B0B4477
:1086F000ACEB03031BB2534505DACEF1000C634526
:1087000001DD1D44641C521CB242EBDB95FBF4F20C
:108710000A44002107E000BF30F81130DB1B13448E
:108720002BF81130491CB142F6DBBDE8F08F7EB565
:108730000026DDE907458DE87000FFF794FF7EBD58
:1087400030B500231C4606E030F91350954201DA9B
:1087500020F813405B1C8B42F6DB30BD2DE9F04363
:1087600000252E462C46DDF81C9017E031F91470D8
:1087700030F914C007EB0208C44505DDBCEB070760
:1087800000D57F423E4408E0A7EB0208C44504DA66
:10879000BCEB070700D57F423D44641C9C42E5DBEF
:1087A000B9F1000F00D10025B54201D201202FE719
:1087B00000202DE74C28100010B500210420F8F708
:1087C00005FC6448644A00685168414006D0506026
:1087D000480703D5BDE81040FDF744BD10BD70B596
:1087E0000546480713D55D4C00235A1E19462069DB
:1087F000F7F76EFF5A492846FAF727FC59492846E9
:10880000FAF749FC2069BDE87040F7F719BF70BD61
:108810002DE9F04150480021534D017053492C6817
:108820000C423AD04068044051480078002834D1C6
:108830004A4E0023CA171946B069F7F749FF214687
:108840004C48FFF7CCFF4C484C4F006890F8A01103
:10885000C90709D0287800060CD43878052809D033
:108860004448FFF7DEFB05E090F85C01444900F066
:108870000F000870B069F7F7E3FE600703D53949C8
:108880003748FEF7AFF93878052802D12868002864
:1088900003DABDE8F041FFF7A3BDBDE8F0812E4942
:1088A00010B500204860FFF725FCFDF7DBFCFFF763
:1088B0004EFABDE81040FFF73FBA274C002767701B
:1088C000FFF7EDFF4FF6FF780126607850B30128DF
:1088D000FBD100213520F8F74BFBF8F701FC0546EA
:1088E000C00706D000214046F8F770FBFFF7D7FF1E
:1088F0006770680705D500210420F8F767FBFFF7CC
:1089000087FFE80605D500211020F8F75FFBFFF789
:1089100053FFA806D9D500212020F8F757FB1948A6
:108920000670D2E704210020FAF7EBFB00210220B9
:10893000F8F71EFB04210120FAF7E3FBF8F7D0FB60
:108940008007C2D500214046F8F740FBFFF7A7FF9C
:108950006670BAE78C2A1000D42910002438100061
:10896000E2190120061A0120882810003C0200802C
:1089700066281000C08D01204C281000942810009B
:1089800093281000322910002DE9FC47894607463C
:10899000FAF755FB0090FAF77DFB01900421684639
:1089A000FAF76AFA0446042101A8FAF765FA2044A6
:1089B000F74C4600F749E068F74D704301EB400083
:1089C00029687200B1F8F2823946FAF721FD286869
:1089D000E16890F8F102884202D10120A07002E023
:1089E000A078012819D1EB4F002014E02A6801215A
:1089F00037F9103092F8F122521C05E006FB010C09
:108A0000491C37F91CC063448A42F7DCA3EB080217
:108A100029F81020401CB042E8DB286890F8F112D9
:108A2000E068814201D3401C00E00020E060A078B3
:108A3000BDE8FC872DE9FC4115460E460746FAF7CE
:108A4000FEFA0090FAF726FB0190009804214008F6
:108A500000906846FAF710FA0446042101A8FAF7D4
:108A60000BFA00EB440C07EB440207EB4C03014606
:108A700006EB440706EB4C06002006E032F810C077
:108A80000CFB05FC27F810C0401CA042F6DB0020C0
:108A900006E000BF33F810206A4326F81020401C7F
:108AA0008842F7DBBDE8FC812DE9FC471546894685
:108AB0000646FAF7C4FA0090FAF7ECFA019004219E
:108AC0006846FAF7D9F90446042101A8FAF7D4F95F
:108AD0000146304606EB440305EB4407002207E05D
:108AE00030F802CB33F8028B521CC44427F802CB77
:108AF000A242F5DB01EB440206EB840006EB4203E5
:108B000005EB4206002207E030F8027B33F802CB87
:108B1000521C674426F8027B8A42F5DB4846294608
:108B2000002204E030F8023B21F8023B521CA24232
:108B3000F8DB09EB440005EB8402002105E000BFEF
:108B400030F8023B22F8023B491CA142F8DB6FE7F8
:108B50002DE9F0438946904909684C7D0B7D641CE2
:108B6000012116E04A1C01FB03F55A4300EB4506C0
:108B700000EB420709EB4505002207E036F812C07A
:108B800037F81280C44425F812C0521C9A42F5DB13
:108B9000491CA142E6DBBDE8F08370B505467E487E
:108BA0000C46006890F88C17C9060AD5007D294646
:108BB00042002046FAF72CFC21462846BDE87040CA
:108BC000C6E721462846BDE87040FAF746BC724821
:108BD000006890F829010106704802D50188491CF7
:108BE00001E06B498988018070472DE9F0476A4CA4
:108BF0006B480027216802783E4691F8C810BA46B3
:108C0000CB0717D08B0715D5664B1B78C1F38205B0
:108C1000012101FA05F52B4201D0017002E0514615
:108C200080F800A0C8B2824204D001280ED0CD2026
:108C300000F067FE574DDFF85881103D287838B1B5
:108C4000F9F71FFEC8F81CA0BDE8F087CC20EFE7BD
:108C5000FFF7BDFF206890F81801400701D5F9F72C
:108C600047FD514800780128ECD0DFF840910023FF
:108C70005A1E1946D9F81800F7F72AFD98F81C0073
:108C8000C00715D04A496868FFF787FF2168484F39
:108C90000B7D4A7D18465343B1F96E21454901EBDE
:108CA000400107EB4000FFF7C8FC88F801000127EE
:108CB000B8F81C0010F4DE7F46D0206890F8CD078D
:108CC000C00705D0D5E902013B4AFFF7EDFE03E0FE
:108CD0003949A868FAF7A5FB98F81C004546000634
:108CE00007D52068344990F8CC270846521CFFF776
:108CF000A1FE2068314990F8F002C0072E4802D04A
:108D0000FFF742FE01E0FAF78CFB206890F8F012C2
:108D1000C90701D0AE7800E0012690F84914890710
:108D200012D5427D254D012305EB42002449FFF772
:108D3000FFFB206801232349027D407D02EB4000B8
:108D400005EB4000FFF7F4FB1F49D8F81C00086052
:108D5000D9F81800F7F774FC1C4C012F03D104203C
:108D6000E168F8F754F9012E7FF46CAF1849B1F9B6
:108D70000000002806DD401E00B2088010B90D205A
:108D800000F0BFFD04202169F8F741F95AE700001F
:108D9000DC291000483A10004C2810009C281000D4
:108DA000762810004B000020942810002438100072
:108DB0004089012042000120303E1000C08D01207A
:108DC000888E0120AC8E0120882810000C381000FD
:108DD0009028100010B501461022FD48FAF718FB44
:108DE000FC4881680220F8F743F9002803D0BDE869
:108DF0001040F7F707BB10BD70B594B00446684645
:108E0000FAF736FBF448F54BF549C461E2072CD07C
:108E10009DF8002042F001058DF800500A6892F894
:108E20007A67F60707D0EF4E3678012E03D145F06A
:108E300080058DF8005092F82051ED0715D0EA4DCD
:108E40002D7895B91D78032D0FD0002C0DDB02F283
:108E5000211255788DF8125015788DF817509278A8
:108E60008DF8132044F48062C26114F49E7F4FF0A9
:108E7000000545D00A6892F8A061F6070DD092F877
:108E8000CD67F60709D01B78052B12D09DF800306E
:108E900043F010038DF8003002E01B78052B08D05A
:108EA00092F87A27D2079DF8002025D042F00602DA
:108EB00024E0002C1BDA92F87A37DB079DF80030AB
:108EC00002D043F0060301E043F020038DF80030A8
:108ED00092F87037DB0703D092F873278DF83620AD
:108EE0008DF83450C26942F08002C26108E09DF8FA
:108EF000003043F00203E9E742F020028DF8002041
:108F0000E2051CD5B94A1278012A03D0B84A127872
:108F1000012A14D1096891F8B02112070FD58DF8F4
:108F2000345091F8CD17C90705D09DF8001021F0F5
:108F300010018DF80010C16941F08001C1619DF8F8
:108F4000000010F0B60F05D09DF8010040F00400BD
:108F50008DF80100AFF2831001906846F8F703FF27
:108F600014B070BD00EB80004FF6FF7101EA4000C5
:108F7000F8F7B6B9994810B50178994805290068FD
:108F800007D09C490978012906D090F81A4134B1DC
:108F900006E090F81D41FAE790F81B41F7E714242A
:108FA000F8F786FA002801DD04EB8404204610BDA2
:108FB000F0B58B49054600200A6892F82040E10789
:108FC0003FD086490B788449052B1CD092F8393064
:108FD000894E36782EB1670603D492F84974FF079C
:108FE00030D0864F3F780FB1A4062BD58C68641C17
:108FF0008C609C4225DD0020886092F85011012091
:10900000C90718D108E00E7892F83A30032EDFD263
:10901000761C0E708B60DBE792F8021259B992F859
:10902000E012C90707D192F86012C90703D192F87C
:10903000B011C90702D00EB940F23D10284040F0EF
:109040000040F0BD5A428A60F0BD2DE9F04FDFF8D4
:109050008CA1614C002368499AF800C0A0690A7885
:10906000E1461E469846C50719460DD05F4D2F783C
:10907000634D012F06D06778012F03D012B92F78E6
:10908000012F01D129700126450601D502B1012623
:10909000420709D5594A1278012A03D0594A127851
:1090A000012A01D14FF001084E4F574D574A012E6A
:1090B0000ED04B4ED646BCF1030F36680ED04FF0A3
:1090C000010ABCF1020F15D0BCF1050F47D049E0F1
:1090D000616121612970117039705AE02161297034
:1090E00011706269521C626196F85D31934250DAE8
:1090F000616149E0DFF818C19CF800C0BCF1010FC4
:1091000027D0DFF810C19CF800C0BCF1010F20D0BF
:10911000DFF804C19CF800C0BCF1010F19D096F82B
:1091200018C15FEA8C7C1DD56161D4F810C00CF1C8
:10913000010CE346C4F810C096F819C10CEBCC083A
:1091400008EB0C18BBEB880F0CD3216185F800A04D
:1091500023E06161216129701170397002E0B8F17A
:10916000010F0CD0B9F1020F0ED0B9F1050F14D0D8
:109170008EF800A0034023622A783AB356E061617A
:10918000216129701170397002238EF800303F235D
:10919000F0E703238AF80030ECE74FF0050C8EF877
:1091A00000C010F00C0F3DD01E235FEA807C35D04C
:1091B00092F800C0BCF1010F30D196F81861F606A4
:1091C0002CD511701B2387F800A0D3E72DE00000F9
:1091D000383A10000C381000DC29100094281000D8
:1091E0004C28100065281000A62810006D281000DB
:1091F000702810006A2810006628100071281000DE
:1092000072281000732810006328100064281000D2
:109210008D2810008E281000A728100082F800A0CA
:109220003970A7E71F231170A4E72170FFF7C0FE74
:10923000216A08432062BDE8F08F2DE9F041CE4E4F
:1092400000235A1E19463068F7F742FAFFF7FDFE71
:10925000CA49086800280ADDC94A12783AB9401E8E
:10926000086004D1C74841690220F7F7D0FEC64C18
:10927000C64F206890F87A07C00707D0C448007826
:10928000032803D0388B10F49E7F03D1FFF772FEC2
:10929000FFF768FE2068BF4D90F8F007C00708D0C0
:1092A000286830B100212020F7F762FE00202860F6
:1092B0000CE0386AFFF7A0FD00210220F7F758FE06
:1092C00000210220F7F782FEFFF78FFC3068F7F7E6
:1092D000B7F9206890F8F007800701D501202860D1
:1092E000BDE8F08110B500210120F7F76FFEBDE861
:1092F0001040A2E7F8F704B82DE9F05F00273946DF
:109300000420F7F763FEA448DFF880820668D8F8E7
:10931000181091EA06054CD0DFF880A2DFF880B281
:10932000DFF8809235423C4626D029BB9E48012773
:10933000002104604FF6FF70F7F748FEC8F81C40A4
:10934000C8F82040C8F81040C8F81440C8F80840D1
:109350008AF8004089F800408B498BF8004088F873
:109360000140096891F82911890705D58F48A8F8A7
:10937000044004808E480480042D05D1C8F80C40B8
:1093800088F8024089F80040814D4046C8F81860CE
:109390008EB10221012F19D02A78052A09D1046142
:1093A000C8F814408AF8004089F800408BF8004063
:1093B0002970BDE8F09FF7F7A3FF01202870BDE8F2
:1093C000F05F00214FF6FF70F7F700BEF00702D004
:1093D0000320287000E02970BDE8F05F2DE710B58C
:1093E00000211020F7F7F2FD6948017801290CD01F
:1093F0000521017065490020684A48610861012122
:109400001170684908706649087010BD10B50021D8
:109410000820F7F7DBFD5E490878052813D15B4A81
:1094200000205E4B5061106118705E4B18705C4BF1
:1094300018709069C20701D0032003E010F02C0FD0
:1094400002D00220087010BD8005FCD50420F9E789
:1094500010B500215D20F7F78BFDF7F741FE0107FE
:1094600002D5BDE81040D1E7C10602D5BDE81040E5
:10947000B5E7410609D4410702D5BDE810403BE7F6
:10948000C00702D0BDE810402CE710BD10B5022186
:109490000020F9F736FE00210420F7F769FD0221CC
:1094A0000120F9F72EFEF7F71BFE400702D5BDE8B5
:1094B000104021E710BD35490020354C8861C86156
:1094C000012208622270354A086148611070354AED
:1094D000384B10701E221A80314A10704870C860D4
:1094E0008870354908703549087007E020780128F0
:1094F00004D00528FAD8FFF7ABFFF7E7FFF7C6FF60
:10950000F4E7224900204861086124490870254990
:1095100008702349087070471C480021C1608170A1
:10952000704710B5F8F753FF18490020C86110BD07
:1095300010B5F7F7E5FE134881680120F7F798FDAD
:10954000002803D0BDE81040F6F75CBF10BD80B224
:10955000F7F7F0BEF7F7FEBE10B5F7F7FBFE0B48C6
:109560008188491C8180BDE810400120EFE7064852
:10957000006890F81C01F5E424381000882A1000D7
:10958000662810000C3810004C281000DC29100050
:1095900094281000782810008C2A100063281000EE
:1095A0006528100064281000882810009C281000EE
:1095B0009E28100090281000A8281000A92810004C
:1095C00070B5FF4C002305465A1E1946A068F7F7F0
:1095D0007FF8002807D02846F7F774FFA068BDE899
:1095E0007040F7F72DB870BDF64B10B51B680246FA
:1095F00001201C8B944200D20020DA8A8A4200D2D9
:10960000002010BDF7F75EBF1CB50021009101914D
:1096100002789DF8001062F303018DF80010427883
:1096200062F307118DF800104289BDF8011062F352
:109630000B01ADF801100289BDF8021062F30F11A1
:10964000ADF8021082798DF80420C2798DF80520DA
:1096500002798DF806208078090900F0FE008DF867
:109660000700BDF80100C0F30B00FFF7BDFF0128A4
:1096700002D16846FFF7A4FF1CBD1CB50020009076
:10968000019002208DF80000CF480068C007400E0E
:109690008DF807006846FFF793FF1CBD1CB500213D
:1096A0000091019101788DF8001041788DF801103A
:1096B000C188C1F307118DF802108188C1F3071129
:1096C0008DF80310017901F00F018DF804108279F3
:1096D00041EA02118DF8041081788DF80510C178E7
:1096E00001F00F018DF80610B7490968C907490E46
:1096F0008DF80710B0F90410B0F90600FFF774FFF9
:10970000012802D16846FFF75BFF1CBD1CB5002095
:1097100000900190AB4800684178827810208DF865
:1097200000004006437A8DF80130A84B1B788DF875
:10973000023043891B0A8DF8033040898DF80400FC
:10974000A1488DF805108DF806200068C007400E6E
:109750008DF807006846FFF733FF1CBD1CB50020DD
:109760000090019011208DF8000097480068C00714
:10977000400E8DF807006846FFF722FF1CBD2DE95B
:10978000FC410646002000900190122015460C4630
:109790008DF800004FF008571EE0200A8DF80100F8
:1097A000C4F30B008DF80240315C30448DF8031097
:1097B00041788DF8041081788DF80510C0788DF807
:1097C0000600D7F8E001C007400E8DF80700684694
:1097D000FFF7F6FE241D2D1F002DDEDCBDE8FC8109
:1097E0001CB50022019200920F228DF800208DF806
:1097F00001008DF80610402073498DF80700012004
:1098000008606846F7F75EFE1CBD1CB50023009398
:109810000193DB238DF800308DF801008DF80210E4
:10982000100E8DF80300100C8DF80400100A8DF84E
:10983000050065488DF806200068C007400E8DF8C9
:1098400007006846FFF7BCFE1CBD1CB50022009255
:1098500001920F228DF8002005228DF801208DF84D
:10986000020059488DF803100068C007400E8DF8BB
:1098700007006846FFF7A4FE1CBD7CB500250095D7
:1098800019208DF8000040070195417A8DF80110EC
:109890004E4909788DF802104189090A8DF80310A4
:1098A0004089484E8DF80400474C306841788DF867
:1098B000051080788DF806002068C007400E8DF8EE
:1098C00007006846FFF77CFE00951A2001958DF889
:1098D0000000306800F5FC6001788DF801104178D7
:1098E0008DF8021081788DF80310C0788DF804008F
:1098F0002068C007400E8DF807006846FFF760FE3D
:109900007CBD1CB52F49096891F82911490603D47B
:1099100000F00F010C2919D10021009101911621AD
:109920008DF800108DF80100010A8DF80210010C6D
:10993000000E8DF8040024488DF803100068C0075D
:10994000400E8DF807006846FFF73AFE1CBD1CB5B7
:1099500000230093019316238DF800308DF8010049
:10996000080A8DF80200100A8DF8040016488DF8D8
:1099700003108DF805200068C007400E8DF8070021
:109980006846FFF71DFE1CBD1CB500230093019324
:1099900016238DF800300B238DF801308DF802006E
:1099A000080A8DF804008DF80520100A8DF80600CD
:1099B00005488DF803100068C007400E08E000005D
:1099C000243810004C281000E0010022A4281000C8
:1099D0008DF807006846FFF7F3FD1CBD1CB500239A
:1099E00000938DF80000080A8DF802000193100A18
:1099F0008DF8050006488DF803108DF806200068E4
:109A0000C007400E8DF807006846FFF7D9FD1CBD62
:109A1000E00100229748006890F82A0100F0070052
:109A2000801C00EB8000C000F7F76FBC2DE9F04709
:109A3000914D286850B3DFF8448200235A1E19461E
:109A4000D8F81400F6F744FE00240127286807FA26
:109A500004F6304213D004EB440005EB800999F87A
:109A6000040005280BD104218548F9F705FAC1B295
:109A700009F10400FFF7C8FD2868B0432860641CA2
:109A80000A2CE3D3D8F81400F6F7DAFD7C48001F5F
:109A90004068002802D0BDE8F047BBE7BDE8F0878A
:109AA000F7F743BC2DE9F05F754DDFF8D0A12D1F0E
:109AB0000023D5F804805A1E1946DAF81400F6F788
:109AC00007FEDFF8B0914FF0005BD9F8000090F886
:109AD0002901800702D500218BF805100027664870
:109AE0000126BE400168314239D007EB470200EB46
:109AF00082042279032A09D0042A07D0052A2ED10C
:109B0000D9F8002092F82921D20628D4B143016067
:109B10002079032802D0042804D018E0686806439E
:109B20006E6014E0D9F8000090F82A0100060BD509
:109B30000520207104215248F9F79EF9C1B2201D79
:109B4000FFF762FD042020716868B043686004215B
:109B50004B48F9F791F9C1B2201DFFF755FD7F1C65
:109B60000A2FBCD3D9F800004C4690F82901800791
:109B700002D580218BF80510DAF81400F6F760FDA5
:109B8000206890F82901C0060ED56868B8F1000F6A
:109B900005D0002808D1BDE8F05FF7F7C6BB002864
:109BA00002D0BDE8F05F35E7BDE8F09F3449002002
:109BB000091F48607C21304805F021BB304D00264C
:109BC0002D1F2E70F7F7B1FB287840B30128FBD189
:109BD00007200021F7F7CCF9F7F782FA044640078F
:109BE00006D500210420F7F7F1F9F7F79EFB2E7058
:109BF000A00705D500210220F7F7E8F9FFF752FF8B
:109C0000E007E1D000210120F7F7E0F919480068EA
:109C100090F82901C006D7D5FFF708FFD4E7002147
:109C200008240846F9F76DFA00212046F7F7A0F955
:109C300000210120F9F765FAF7F752FA0007C3D5BA
:109C4000FFF7B4FFF7F771FB00210F20F7F7BEF91C
:109C500001202870B8E710B5F7F767FB09480168DD
:109C60000120F7F705FA002803D0BDE81040F6F709
:109C7000C9BB10BD4C2810008437100024381000D8
:109C8000042A10000C3810002DE9FF5F7A481023D9
:109C90000026016891F86704020900F00F00CDE981
:109CA0000220B1F868040090B1F86A04019091F8BC
:109CB00023204C7DA3EB121A704B4FEA121B087D38
:109CC0001A68641C521C1A6091F866544443B2EB43
:109CD000151F00DD1E605A6805F00F05521C5A6002
:109CE000954200DA5E60DFF898C1DFF89891664F20
:109CF00074E000BF91F82020520632D437F910806A
:109D0000B1F926603CF9102008EB0605954264DBAA
:109D1000B1F92860A8EB060595425EDC08FB0BF55F
:109D200002FB0A524FEAE27502EB157242F30F1E74
:109D300091F8D020520711D5AEEB08020FFA82F845
:109D40005FF0000202EBC20609EBC615521C35F8A3
:109D50001060042A464425F81060F3DB27F810E071
:109D60003BE037F910E0B1F926603CF910500EEBFA
:109D70000602AA4231DBB1F92860AEEB0602AA4224
:109D80002BDC0022754504DA5D688DB9039A5242D6
:109D90000BE01E6866B9029A009EA5EB0E0512B292
:109DA000B54205DD019A954201DD12B200E032B202
:109DB00091F8D0506D070DD55FF0000505EBC50893
:109DC00009EBC8166D1C36F81080042D904426F857
:109DD0001080F3DB724427F81020401CA04289DB7E
:109DE00091F8200000070CD52748F9F7C4F9274956
:109DF000274A086004B00146BDE8F05F2248F9F741
:109E00000BBABDE8FF9F10B51B4C206890F84904C1
:109E1000C00703D0F9F7B4FF012817D0206890F8E5
:109E20002000C10727D01B49097809B1400622D577
:109E3000194C00235A1E1946E068F6F749FCFFF753
:109E400023FFE068BDE81040F6F7FABB134801684D
:109E500041F0050101601248016841F020010160F4
:109E600010490120087010484168BDE810404FF4C7
:109E70008060F7F7CCB810BD4C281000082A1000FD
:109E800040890120C20401204200012084281000E2
:109E90006437100066281000243810005028100085
:109EA00058281000542810000C381000FE490020DB
:109EB0000870704700E010460A5C8242FBD1704790
:109EC00070B500250E4603462C4606E0194620468E
:109ED000FFF7F0FF1855641CE4B2B442F6D3002239
:109EE0000AE0985C904203D19D546D1CEDB201E0F4
:109EF000185C9854521CD2B2B242F2D3284670BDBC
:109F000038B1884202D20B4601461846884200D03A
:109F10001154084670472DE9FF4F99B00120049075
:109F2000E24819689A460068067D477D41B19AF873
:109F300002109AF800905046B14205D2491C04E044
:109F40004FF000094D4608E0314645789AF8030085
:109F5000CEB2B84200D2471CFFB2002007A9085475
:109F6000401C2D28FAD3199905EB051001EB400C84
:109F7000681C67E01998E34608EB081100EB410CF8
:109F800009F101045AE000BF0CEB040015900068D1
:109F900010B31CF8040000B31598002310F8010C4E
:109FA00000B103461BF8041021B107AA1846FFF7B9
:109FB000A7FF03461A9800280BEB04000ED015905B
:109FC00010F8011C21B107AA1846FFF799FF0346B4
:109FD00015984178D9B91FE0E41C2EE0189010F8CC
:109FE000011C59B115981BF8042010F8010C1043FE
:109FF00004D007AA1846FFF783FF03461898417854
:10A0000051B115981BF804204078104304D007AADA
:10A010001846FFF775FF034613B10CF804300CE047
:10A0200004982D2806D20CF804000498401CC0B2F5
:10A03000049002E0401E0CF80400641CB442A3D952
:10A0400008F101008046B84294D907A80499FFF7A7
:10A0500037FF804641001B9805F0AFF800204FF60F
:10A06000FF7202E04AF82020401C4045FAD33BE052
:10A07000199905EB051001EB400022304C46059084
:10A080002FE00598011901204058A8B3487838B34B
:10A0900007AA105C48701B991B9A0AEB800B31F8D9
:10A0A0001010491C22F810109BF800102046F8F7F9
:10A0B000F6FE8BF800009BF801102846F8F7EFFE3B
:10A0C0008BF801009BF802102046F8F7ECFE8BF8A5
:10A0D00002009BF803102846F8F7E5FE8BF8030012
:10A0E000641CB442CDD36D1CBD42C1D3A8F10100A4
:10A0F0001DB0C0B2BDE8F08FFFE7E41CF0E72DE92A
:10A10000F043994655784FF0010C1BE005EB051321
:10A1100000EB430622360023147897780CE000BF4A
:10A1200006EB040898F90180884503D10CFA04F87D
:10A1300048EA0303641CE4B2A742F1D249F825308F
:10A140006D1CEDB2D378AB42E0D2BDE8F083F0B540
:10A15000554B0026554D1C7894B0012C11D11E7022
:10A160000B78002B5AD04B78002B57D02B688F7868
:10A170001C7D641EA74251D05B7DCC785B1E9C4247
:10A180004CD000234FEA0D0444F823605B1C142BD1
:10A19000FAD34B7891F803C01BE000BF50F823704E
:10A1A000B7B17E0846EA47063E4354F8237037436A
:10A1B00044F8237004EB8307D7F804E04EEA060E58
:10A1C000C7F804E0D7F808E04EEA060EC7F808E042
:10A1D0005B1C9C45E2D2002304EB8306766840F8C2
:10A1E00023605B1C122BF7D3012A17D1087808B122
:10A1F000401E0870487808B1401E48702A68887868
:10A20000127D521E904201DA401C88702A68C8787C
:10A21000527D521E904201DA401CC87014B0F0BD4D
:10A220002DE9F0478246107D012873D14C781F4EEE
:10A2300001234FF003096AE030685AF82450027D88
:10A24000601C42431A48006800EB42000A7811E0A3
:10A2500003FA02F72F420DD000EB420730F91280CB
:10A2600037F902CCB7F90270C444BC449CFBF9F73F
:10A2700020F812708F78521C9742E9DC0A785AB3A2
:10A2800003FA02F72F420DD000EB420730F912809B
:10A2900037F902CCB7F90270C444BC449CFBF9F70F
:10A2A00020F812708A7805E0102A10004C2810005F
:10A2B0008028100037683F7D974203FA02F707EACB
:10A2C000050714D117B300EB420530F9127035F9C8
:10A2D000025C3D446D1017E015F0010FE2D0B0F9BB
:10A2E0000020B0F902703A4452100280DAE76FB1F0
:10A2F00000EB420530F912C035F9027CB5F9025085
:10A3000067442F4497FBF9F520F81250641CC87875
:10A31000A04291DABDE8F0872DE9F05F9B4600236B
:10A320000D46144619464FF4803A012A01DA0022FC
:10A3300003E000EB840252F8042C50F82490AC4265
:10A3400001DB002002E000EB84004068824202DD75
:10A350000346114602E001DA13460146A0EB020271
:10A360004FF4803CA2FB0C084FEAE27707FB0C8716
:10A370004FF0000602FB06764944C3F1000201EBF0
:10A3800042024FEAE273314604F0A6FE4FF48036F3
:10A39000A4FB063CE7170A4607FB06C6002104FBA0
:10A3A0000161181851412A46EB1704F095FE024648
:10A3B000A2FB0B0501FB0B514FEAEB7402FB0411EE
:10A3C0005246002304F088FE00B2BDE8F09F2DE95C
:10A3D000FF5F002704463D463E468821F748DDF8EA
:10A3E0003C9004F00CFFDFF8D8E36078DFF8D4B3DA
:10A3F000DEF8003031E021782BE000BF93F814C084
:10A40000421C02FB0C1C9246DBF8002032F91C2097
:10A41000BA420CDDDFF8A4C36D1CADB25CF820C0FD
:10A4200016440CEB0208DFF894C34CF8208099F82E
:10A430001420012A0CD11A7DDFF88CC302FB0AF22A
:10A440000CEB010A12F80AC04CF0800802F80A80EE
:10A45000491CA2788A42D1DA401C94F803808045D6
:10A46000C9DA00210A46607808E0DFF850C35CF8DA
:10A4700020C08C4501D961460246401C8045F4DA73
:10A48000597DF046491E12B2CC48029BFFF744FFAB
:10A490000E9908608821C94804F0B1FE2078C74AA7
:10A4A000DBF800A0D8F800C015E061780FE000BF2D
:10A4B0009CF814804B1C03FB08083AF91830BB4287
:10A4C00004DD52F82080434442F82030491CE378F0
:10A4D0008B42EDDA401CA1788142E6DA00231F4668
:10A4E000207806E052F820409C4201D923460746D6
:10A4F000401C8142F6DA9CF814103AB2491EAF486B
:10A50000019BFFF709FF03990860C9F80860A9F8E3
:10A510000450BDE8FF9F2DE9F74FA94E8C46002758
:10A5200031681446127DB1F868A084B03D463846C3
:10A53000B94612B1012A03D012E0B1F8C8A10FE068
:10A5400091F8A02052070BD502A8CDE90004B1F97B
:10A550001820B1F9161003AB6046FFF738FF6DE025
:10A560009CF8011039E0049A52F821B09CF80010D0
:10A5700003912BE00121914011EA0B0F24D03168A7
:10A580000B7D02999E4601F1010808FB03218D4BCA
:10A590001B6833F91110514506DD531C03FB010004
:10A5A00008FB01990D447F1C217D01295DD0864B5C
:10A5B00000290EFB08F1134411F803805ED048F027
:10A5C000200800BF01F80380521C03929CF802107F
:10A5D000039A9142CEDA0299491C02919CF8032019
:10A5E0008A42C0DA3268411B9246D28A4FEAE17C45
:10A5F000A1FB02080CFB02824FF0000B01FB0B21B8
:10A600009AF81420521E6A43D31704F065FD039094
:10A61000A9EB05013268CB179146128BA1FB02080A
:10A6200003FB028201FB0B2199F81520521E6A439D
:10A63000D31704F051FD0290A560A780207D00286B
:10A64000306890F880001CD0C00604D5002202A912
:10A6500003A801F05DFA02A903A8F8F797FF039891
:10A6600060800298208007B044E5574B0EFB08F14C
:10A67000134411F8038048F08008A3E748F040082D
:10A68000A0E78006E7D50122E1E72DE9F04F4C4C29
:10A690004C4B834600204A784FF0010AD4F80090D2
:10A6A000CE78D3F8008015E05BF822700B78541C4C
:10A6B0008D780CE00AFA03FC1CEA070F06D099F823
:10A6C00014C004FB0C3C38F91CC060445B1C9D4268
:10A6D000F0DA521C9642E7DA0CE52DE9F0438146A8
:10A6E0005078079E23E000BF354B00EB0014354D3A
:10A6F0001B6809EB440422341B7D401C2D68434336
:10A7000005EB430513784FF0000C0CE0E71897F8C1
:10A710000180884505D135F91380B04501DC87F803
:10A7200001C05B1C1BB297789F42EFDA00B2D3786E
:10A730008342D9DA09E52DE9F0410746107D204D25
:10A7400014460E46022807D12968E08891F8661061
:10A75000884201D9032020750422314604F11000FB
:10A76000F8F756FE31463846FFF78FFFE0600122CA
:10A7700031463846FFF7EBFC286890F88C07C00696
:10A7800004D5224631463846FFF74AFD2246314677
:10A790003846FFF7C0FE2046BDE8F04103F057BA47
:10A7A00030B595B01C4615466B46FFF7A8FC22460F
:10A7B00029466846FFF7BFFF15B030BDF83E1000D0
:10A7C0004C28100080281000349D01202DE9FF4FF7
:10A7D00086468A4600204FF6FF755378D67826E0E5
:10A7E00003EB03140EEB440C14780CF1220CFE491D
:10A7F000DFF8F8B39778D1F8009014E00CEB04017F
:10A8000091F80180D0450CD199F81480591C01FBB6
:10A8100008483BF81810884200D208468D4200D9FB
:10A820000D46641C24B2A742E8DA5B1C1BB29E42B0
:10A83000D6DA039908800D990D8004B05AE42DE909
:10A84000F04F9B46824653782AE000BFE84D03EB69
:10A8500003100AEB4004AD68223405EB40052235B5
:10A860001078E14FDFF884C34FF0010913E0261898
:10A8700076788E420DD13E6896F814805E1C06FBF9
:10A8800008063CF916605E4503DD05EB000888F814
:10A890000190401C00B296788642E8DA5B1C1BB23D
:10A8A000D0789842D2DA25E42DE9F047CE4F82469F
:10A8B000C8B03868DDF840811E4690F8705046A850
:10A8C00000908946144645AB5046FFF77FFF307D28
:10A8D00030B9C84800780128386829D090F8CE519E
:10A8E000BDF81411BDF818016422091A6943B1FBBF
:10A8F000F2F1BF4F0D184FF42A71B86804F05DFCF7
:10A90000ABB2224649465046FFF799FF20680190B6
:10A9100001AB2EAA0121B868FFF7FDFA0546012810
:10A9200020D901240DF1B80A0DF10409B84615E04B
:10A9300090F86E57D4E700BF3AF81400F08009EBA6
:10A9400084073146384601F091F933463A462146AC
:10A95000D8F80800FFF724FF641CE4B2AC42EBD93E
:10A9600048B0D7E43346224649465046CDF80080E9
:10A97000FFF7B3FE3346224649465046FFF710FF25
:10A98000EEE72DE9F04F9C4D974E14782D78927894
:10A990003768012D03D097F871501CB103E097F888
:10A9A000C950FAE7012497F814809446A8F10107EA
:10A9B000BA4202D1ACF10102D2B203EB031C00EBAC
:10A9C0004C078B4822375B1C806808FB03F800EBC0
:10A9D0004C0C86480CF1220C00EB48034FE0381970
:10A9E0004078884249D1DFF8148233F91400B8F96D
:10A9F0000080404541DD03EB4409284439F902BC9D
:10AA00004FF0000A584503DAB9F90280404534DBBB
:10AA1000012C10D0D6F8008098F81480A8F1020814
:10AA2000A04512D139F9048C404521DAB9F90280E8
:10AA3000404522DB1CE0B3F90200B3F90080284452
:10AA4000404515DAB3F90680F2E7584505DAB9F959
:10AA50000480404501DA4FF0010A39F9048C404581
:10AA600003DAB9F90280404507DBBAF1000F04D1DF
:10AA70000CEB0408012088F80100641CE4B2944245
:10AA8000ADD929E62DE9F74F97B05478D778002053
:10AA900013905948DFF850A115460178DAF8000004
:10AAA000012905D07130067890F8019014B107E0C3
:10AAB000C930F8E7DDE9170101240023FFF761FF42
:10AAC000DAF80010E878497D491E884207D1401E17
:10AAD000C7B2CBB2DDE917012A46FFF752FF0AE100
:10AAE000179904EB041001EB40034149223304F1B0
:10AAF000020C896804F1010E01EB400022300B903A
:10AB0000DAF80000611E007D00FB01F2374900FB0E
:10AB10000CFC01EB4202069200FB04F201EB420244
:10AB2000099200FB0EF201EB4C0B04F1030C00FB4D
:10AB30000CF001EB4000079001EB42022878D4E0D2
:10AB4000191891F801C018998C457CD12B4932F91C
:10AB500010C0B1F900108C4575DD0021DDF82480AE
:10AB600011910CEB060138F91080CDF83880414581
:10AB700007DA3BF91080414503DA4FF00108CDF8C0
:10AB80004480E8B3DAF80080CDF8588098F8148053
:10AB9000CDF85480A8F10108804531D002EB40087F
:10ABA000CDF8288038F9028CCDF82080414509DAAB
:10ABB000DDF82880B8F90280414503DA4FF001083A
:10ABC000CDF84480DDF82480CC4408EB4008CDF873
:10ABD000488038F9028CC44517DA0BEB4008B8F905
:10ABE0000280C44511DA0CE04C281000F4A70120C3
:10ABF000102A1000A628100076281000522A1000F3
:10AC00005EE04FF00108CDF84480DDF84880B8F9E7
:10AC10000280C44505DA0BEB400838F9028CC445C4
:10AC200061DBDDF844C0BCF1000F5CD1DDF858C039
:10AC30009CF815C0ACF1020CA4450FD0DDF838C06B
:10AC400061450BDA00E03DE0DDF81CC03CF910C0C6
:10AC5000614503DA4FF0010CCDF844C0012C0DD052
:10AC6000DDF818C03CF910C0614507DA3BF910C0A7
:10AC7000614503DA4FF0010CCDF844C0012822D021
:10AC8000DDF854C0ACF1020C84450DD0DDF820C0D5
:10AC9000614509DADDF828C0BCF904C0614503DA72
:10ACA0004FF0010CCDF844C0DDF828C03CF904CCCD
:10ACB000614505DADDF828C0BCF902C0614512DB48
:10ACC000119951B10FE0B2F90210B2F900C031444C
:10ACD0006145F5DAB2F906C0F0E70B994FF0010CC7
:10ACE000014481F801C0401CC0B2A9788142BFF480
:10ACF00027AF0EF0FF04BC427FF6F2AE13981AB0F5
:10AD0000EAE42DE9FF4FFD4C0E460746C5B0154657
:10AD10004FF42A71A06804F050FA2A4631463846AA
:10AD2000FFF7B0FE29686E460091B8BB33462DAAE6
:10AD30000021A068FFF7EFF8074601282FD902F09D
:10AD4000F1FF0125DFF8B8830DF1B409AA4618E038
:10AD5000D8F8001039F8150091F8751088420FD90D
:10AD600084F800A04899C88006EB8500834648997E
:10AD700000F07CFFE9B25A46489BA068FFF710FD3F
:10AD80006D1CBD42E4DDD8F8000090F84004800757
:10AD900002D4002002F0CBFF49B09DE4FFE7321D52
:10ADA0000121489BA068FFF7FBFCF5E72DE9F04F78
:10ADB0008246D34800259146D0F800602A462B46AB
:10ADC00009EB0300401E21D4747D84421EDDCD4C6E
:10ADD000377D00F10100246807FB00F004EB400818
:10ADE00003EB430C4FF000000AEB4C0B01EB0004AB
:10ADF000641E08D4A74206DD3BF910C038F91440A0
:10AE0000624404FB0C55401C0328EFDB5B1C032B46
:10AE1000D6DB02B9012295FBF2F05DE42DE9FF4F8C
:10AE200084B00C4601464078DDF844B000B1401EC5
:10AE3000B34F00F0FF09C8783E68727D551EA842E6
:10AE400001DA401C00E0501EC5B2087800B1401E77
:10AE500000F0FF0A307D8978421E914201DA481CD9
:10AE600000E0401EC6B2B4F9120009F101010290DF
:10AE70006CE0DFF88C824F1CD8F80000007D00FBEE
:10AE800007F248430BEB420203EB4000CDE9002000
:10AE90000AF1010057E09A49096891F814E007FBAC
:10AEA0000E0103EB4101B1F9022006998A4245DD0A
:10AEB0000199B4F9008001EB40010022B1F900C012
:10AEC0000CFB0822B1F902C0B4F902800CFB082285
:10AED000B1F904C0B4F9048001EB4E010CFB082267
:10AEE0000392B1F900C0B4F906800CFB0822B1F955
:10AEF00002C0B4F908800CFB0822B1F904C0B4F90F
:10AF00000A8001EB4E010CFB0822B1F900C0B4F934
:10AF10000C800CFB0822B1F902C0B4F90E80B1F923
:10AF200004100CFB0822B4F910C001FB0C21029A9A
:10AF300091FBF2F1009A22F8101002E0009921F83A
:10AF40001020401C00B2B042A5DB39B2A94290DB10
:10AF50004F4615E0017D781C41430BEB4108009002
:10AF60003A4651462046FFF721FF28F81A003A4694
:10AF700031462046FFF71AFF28F81600009807B25E
:10AF80005F48AF420068E5DD007D691C41430BEB83
:10AF90004101009109F1010148430BEB400857467C
:10AFA00010E04A4639462046FFF700FF28F8170010
:10AFB0002A4639462046FFF7F9FE009921F8170086
:10AFC0007F1C3FB2B742ECDD08B06CE42DE9F74FCF
:10AFD0008646507800B1401E494ED178C0B23568DF
:10AFE0006B7D5C1EA14201DA491C00E0591ECCB207
:10AFF000117801B1491ECBB291782A7DB246551E17
:10B00000A94201DA4A1C00E0521ED5B22DE000BF71
:10B01000DAF80010421CDFF8F4B0097D5143394AD8
:10B02000126802EB4106384A02EB410700EB0012BE
:10B030000EEB42022232194614E000BF37F911C06C
:10B0400002EB010926F811C099F80180B8F1000F50
:10B0500007D1BBF90080C44503DDDDF804C089F8E1
:10B0600001C0491CA942E9DD401CA042D0DDBDE879
:10B07000FE8FF8B50E46264907460698097815460C
:10B08000022916D21F4A93F814C01F4913681C4A9C
:10B09000BCF1000F14680DD094F84020920608D53A
:10B0A000012806D10091B4F958201A492846FFF723
:10B0B000B5FEF8BD94F8C0018206FAD54006F8D571
:10B0C0000091B4F9C42114492846FFF7A7FE2A4687
:10B0D00031463846BDE8F84078E738B51C7DFCB10C
:10B0E000074C246894F86040E5071BD00B4C00BF68
:10B0F000B4F900400094FFF7D7FB38BD102A1000C8
:10B100004C28100080281000F4A701204A2A1000C3
:10B110007428100026F6000012F60000522A1000D3
:10B12000F94CE5E7A407E8D501B0BDE83040E8E513
:10B130002DE9F0478146F5488A4600230168184604
:10B1400001250E7D4F7D1DE000EB001409EB44044A
:10B150002234194612E000BF52F8208005FA01FCA3
:10B1600018EA0C0F08D004EB010898F801C0BCF1F4
:10B17000000F01D188F801A0491CC9B2B142EBD33C
:10B18000401CC0B2B842DFD3BDE8F087F0B55478B8
:10B19000002613E004EB041300EB4305223513787B
:10B1A00007E0EF1897F801C08C4500D17E705B1C5A
:10B1B0001BB297789F42F4DA641C24B2D378A3427E
:10B1C000E8DAF0BDD24A10B5127801243AB9CF4A74
:10B1D000126892F86020120718D5012916D18178DB
:10B1E0000278891A01D5C1F1000101F10101CAB249
:10B1F000C1784078081A00D54042401CC1B21046C0
:10B20000F7F74DFEC0B2012800D10024204610BD42
:10B210002DE9F04FBD4BBF4C8A4683460120517843
:10B22000D778D4F800901D6822E000BF01EB01142C
:10B230000BEB440422341378967815E004EB030CEE
:10B240009CF80180D0450DD195F8148001F1010CD6
:10B250000CFB083839F918C0B5F8D281E04501DA9D
:10B26000002003E05B1C1BB29E42E7DA491C09B2D6
:10B270008F42DBDA05E430B5A44CA74A2468B2F962
:10B280000030A64A34F9A85FB2F90020B4F90240B0
:10B2900029B9A349B1F90030A249B1F90020A0426F
:10B2A00001DD104630BDA84201DA184630BD201A33
:10B2B000D11A4843611B90FBF1F0101A00B230BD67
:10B2C0002DE9FF4F1078B5B09B46174600B1401EE0
:10B2D0008E4BC0B231901A68B878117D8C1EA04296
:10B2E00001DD481E00E0401CC4B2787800B1401E69
:10B2F000C0B20090507DF978821E914201DD401E5F
:10B3000000E0481CC0B200262890B24618210EA8C2
:10B3100003F075FFB046DDE93501C146454614AB83
:10B320003A46FEF7ECFE387840B97878C8B17748ED
:10B33000F9780068407D401E814212D07349BA7886
:10B3400008688646007D2990401E824201D17B78A4
:10B350003BB182420DD19EF81500FA78401E824220
:10B3600007D16A480068B0F8AA00801CABF81F003B
:10B3700069E0684A0098136814E02999421C514317
:10B3800003EB410C07B2319909E000BF3CF91120F1
:10B39000424503DD90460FFA81F93D46491CA14222
:10B3A000F4DD401C28998842E7DDAC1E03A9AD1CE2
:10B3B00020E000BF9EF81400621C504303EB4007DE
:10B3C000002021F81600A9F10200021D08E000BFCC
:10B3D00031F816C037F81080401CC44421F816C05C
:10B3E0009042F5DD31F81620761C02EB0A000FFAC8
:10B3F00080FA641CAC42DDDD042300220EA903A800
:10B40000F7F7CAFDDDE91201DDE90E2303F064FE62
:10B410004FF47A71484390FBFAF0404204B2ABF823
:10B420001F4001212046FFF726FF3849096891F89F
:10B43000F017090603D53C4A369922F81140BBF8AB
:10B440001C10814202DD012039B0E6E40020FBE758
:10B450002DE9F043994680460020537823E000BF51
:10B4600003EB031408EB4406284C2A4F22362468C9
:10B470005D1C3F68247D6C4307EB440C14780EE0A0
:10B4800037197F788F4208D13CF91470874204DD68
:10B49000A9F802403846A9F80030641CE4B2977855
:10B4A000A742EDD2EBB2D4789C42D9D2BDE8F0836A
:10B4B0002DE9FF4F83B01878109C92461E46A0706D
:10B4C000987820705878E070D87860704FF0000B52
:10B4D0005F785EE0039907EB071001EB400101F193
:10B4E0002209049901EB400000F122080748006896
:10B4F000017D781C414301900648006800EB410043
:10B500000090357840E00000562A10004C281000CA
:10B510007428100080281000522A1000542A1000AD
:10B520004C2A10004E2A1000F4A7012009EB050058
:10B530004178514522D1009830F915101198814277
:10B540001CDD0BF101001FFA80FB21782846F7F77C
:10B55000A6FC207061783846F7F7A1FC6070A178EE
:10B560002846F7F7A0FCA070E1783846F7F79BFC77
:10B57000E07008EB050080F801A003E008EB05008F
:10B58000002141706D1C2DB2B078A842CEDA01982E
:10B5900007B2F078B8429DDA584607B03DE4FE495C
:10B5A0000278096822B10A7D8378521E934208D13D
:10B5B000427822B1C278487D401E824201D10120EA
:10B5C00070470020704730B5054695B0F24800231B
:10B5D0008DF8503002680C46107D401E8DF85200E8
:10B5E0008DF85130507D6B46401E8DF8530014AAE3
:10B5F0002846FEF784FD002214A96846FEF7A7FD41
:10B600006A4621462846FFF793FD15B030BD2DE967
:10B61000F14FDCB003205390E048E14CDE4D006870
:10B620004FF0000800F52A71C4E90101296891F87A
:10B630006020D30701D1920701D54FF00108D94A04
:10B640001278012A13D091F8C011C1F3C0018946C4
:10B650004FF0000B0CAB39AA0121CDF830B0FEF74A
:10B660005AFC2B68074601201A7DA24618E091F883
:10B670006217C1F34001EAE7012100EB0014DFF893
:10B6800028E309E0DAF8046001EB440C16F80CC07A
:10B690000EF802C0521C491C1E7D8E42F2DA401C7C
:10B6A000597D8142E8DAC149012481F800B0F3E113
:10B6B000E1B239A88DF82A1030F81400ADF8120064
:10B6C0000CA800EB8402509259ABDAF80400FFF7A3
:10B6D000BFFEADF82800ADF82BB006468AF800B0E2
:10B6E000BDF9660158B1BDF9642142B129680B7DED
:10B6F0005B1E984203D0487D401E824201D101204A
:10B7000000E000205690286890F8A010C9070CD0DF
:10B71000A4490978002908D1A54A90F8A7101288F1
:10B720009142A449097801D211B17CE002297AD270
:10B7300001218DF8201090F8A41052919D490978AC
:10B74000012905D190F8BC205299114489B2529137
:10B750005699012964D090F8A50051909648E2B21C
:10B76000B0F900105BA8CDE90001509BDAE90101B6
:10B77000FFF79EFE8C49ADF8120008558F4901EB8A
:10B78000440188824E81529988424CD9519988420D
:10B7900049D88948B0F90000864244DD286890F80D
:10B7A000A000800713D5E1B203AB5BAADAF808006A
:10B7B000FFF786FD01280AD0286890F8A010090735
:10B7C00031D590F8AD107E48007881422BD27D496A
:10B7D0007B4A012008701078401CC1B211702868A3
:10B7E00090F8AD308B4202D290F8AE0010705198B4
:10B7F000E1B2C0B253900220ADF82200ADF82400AF
:10B800008DF821B003AB5BAA5646DAF80800FEF7C4
:10B81000C7FFE1B25BAAB068FFF7B8FC3BE102E00A
:10B8200090F8A60099E756995098FFF7CBFC0128AD
:10B83000F4D16548B0F900108E4272DD012F19D1A4
:10B8400039AA32F814302A6892F89D20934211D90F
:10B8500056490120E3B2087003A800905B485646A1
:10B86000509ADAF80410006800F01CFA04208DF8F1
:10B8700020000AE15BA8CDE90001DAF80410E2B289
:10B88000509B0846FFF714FE0DF1E40C2CF8140051
:10B89000ADF81200286890F865604648007848B115
:10B8A0005098FFF77CFE012828683BD090F8BD0037
:10B8B000304486B239A830F81400B0426BD94149FF
:10B8C0000120E3B208703949564608703C4880F8B8
:10B8D00000B003A800903D48509ADAF804100068C0
:10B8E00000F0E0F939A82A6830F8141092F86700DF
:10B8F000814225D202208DF82000BDF82630B2F812
:10B900006E204046934200D20020539A91420CD3BD
:10B9100058B10090E1B203AB509A7068FFF7A9FBF1
:10B92000ACE011E090F87600C2E72748E1B203AB43
:10B93000B0F900000090509A7068FEF7CEFEA4E0C7
:10B9400004208DF82000F0E7286890F8C011C9079E
:10B9500021D01F490968F1B11E490978D9B98DF87C
:10B9600020B090F8C0015E46400705D5E1B20CAAB0
:10B97000DAF80400FFF727FE0A4847F6FF7200785E
:10B98000012832D0569801281348007831D0012878
:10B99000286837D022E077E04C2810007C2810007F
:10B9A000102A1000A6281000349D01206E281000D7
:10B9B0001E2A100074281000542A1000F4A7012039
:10B9C0006F2810006D281000522A100080281000E7
:10B9D0009C010022672810006828100090F8CB0115
:10B9E00031490978012910D014E0286890F86307DC
:10B9F000F6E70128286802D090F8CD01F0E790F82A
:10BA0000CC01EDE790F8CA01EAE7296891F8D9116D
:10BA1000084480B239A931F8141081423BD99142CF
:10BA200039D85C990220E3B208702048067003A858
:10BA300000901F485646509ADAF80410006800F04B
:10BA400031F9CDF80090E1B203AB509A7068FFF77E
:10BA500010FB286890F8C00180070CD515480078C5
:10BA6000012808D1E1B2509A7068FFF7D1FB012894
:10BA700001D111490870B9F1000F06D0E1B203AB52
:10BA8000509A7068FFF729FB05E0E1B203AB509ACA
:10BA90007068FEF785FE641CBC427FF609AE5DB09F
:10BAA000BDE8F08F70470000742810006F28100068
:10BAB0008028100068281000482A1000F0B50024E3
:10BAC000491E05680BE000BF32F91470AF4205DC77
:10BAD00002EB4406B6F90270AF4202DA641C8C42F3
:10BAE000F2DB8C4213D032F9146003EB440133F9DA
:10BAF0001430B1F9021002EB4402AD1BC91AB2F9BD
:10BB000002206943921B91FBF2F119440160F0BDE0
:10BB1000F0B50E461D494FF0000C1300096864464D
:10BB2000624604D0012B09D0022B0ED018E091F808
:10BB300071C491F8704401F272410CE091F871C641
:10BB400091F8704601F2726105E091F871C591F8C3
:10BB5000704501F272510A460CEB04013E2914DCD7
:10BB600002EB4C0303EB4C0505EB4407BCF1010F62
:10BB700002DD6146FFF7A2FF012C06DD3B462A46A7
:10BB800021463046BDE8F04098E7F0BD4C28100053
:10BB90004FF47A72504390FBF1F17D4810B5814229
:10BBA00001DAC01110BD42F6A640814201DD5A20E3
:10BBB00010BD784A002000BF32F910308B4205DCFE
:10BBC00002EB4003B3F902308B4202DA401C4528F5
:10BBD000F2D332F9104000EB800302EB4000091B66
:10BBE000B0F90200553B001B01EB810191FBF0F025
:10BBF000184410BD30B50D460446FFF7C9FF00EBF1
:10BC0000D0704010002D02D00DDD34B130BD002CBD
:10BC100003D005DD4FF02D0030BD4FF0000030BDEA
:10BC20004FF05A0030BD002C03D005DD00F15A0062
:10BC300030BD6FF0590030BDA0F15A0030BD10B5D5
:10BC40008C1A00D56442002800DA404204EB400020
:10BC500011440A18081A521040104FF47A714843E0
:10BC600090FBF2F0C0F57A70588310BD30B5827841
:10BC70000378CD88D21AC3784078521C1B1A5B1CFB
:10BC800005FB02F0D4185D4340006A00B0FBF4F0FD
:10BC9000B2FBF4F2904202D9C8820A8330BDCA8254
:10BCA000088330BD2DE9FF4F1646002284B01046B0
:10BCB0001546964693469246747896F8039036E079
:10BCC000059904EB041301EB43012231039133780E
:10BCD000029396F802C027E0039919444F78079918
:10BCE0008F4220D12C4909680F7D611C01FB073769
:10BCF000049901EB4701A9EB0407B1F902107F1C7D
:10BD0000CDE9001702995F1A00997F1C0A44794314
:10BD100001FB07BB019F084401FB07EE0099794333
:10BD200001FB07AA0D445B1C9C45D5DA641CA145A8
:10BD3000C6DA4FF47A71414391FBF2F14FF47A7312
:10BD40006B4393FBF2F201FB05F44FF47A7394FB1F
:10BD5000F3F7414391FBF3F1AEEB0704ABEB0107C3
:10BD60006A4392FBF3F1AAEB01056000791BFFF730
:10BD700041FF11992A46487539462046119BFFF725
:10BD80005EFF119908B03046BDE8F04F6EE7000045
:10BD90005AD3FFFFCCF500004C281000F7490020D3
:10BDA0000870F7490870F74908707047F64930B4D1
:10BDB0000020F64A087001211170F549FB4AFC4C3D
:10BDC0000870F449FB4D0870F3490870F349087096
:10BDD000F3490870F3490870F34948708860C860F7
:10BDE0001268B2F862302380B2F8A1402C80F24D84
:10BDF000B2F8C6212A80F14D2B80F14B1C80F14B0B
:10BE00001A80F14A10804860087030BCC6E72DE9FE
:10BE1000FF4F81B0E54A4FF00109CDF8009012685C
:10BE20009B464D4692F815C0137D0CF1010C62E063
:10BE30004FF0000A47F6F8725442D646564619E0CB
:10BE400005FB036730F8178031F81770A7EB080778
:10BE50003FB2BA4200DD3A46BC4200DA3C46002F0F
:10BE600002DA4FF0000903E002DD4FF0000700970F
:10BE700006F101069E42E3DB009F59EA070608D05F
:10BE8000B9F1010F03D0B9F1000F04D006E0012F82
:10BE900004D1002202E0012F00D12246002412E04A
:10BEA00005FB034630F8167031F816601744F61B90
:10BEB00036B25E4506DACBF10007BE4202DDB2447F
:10BEC0000EF1010E641C9C42EADBBEF1000F01DDA5
:10BED0009AFBFEFA0AEB0204002209E005FB0326A6
:10BEE000DDF80C8030F81670521C274428F81670C4
:10BEF0009A42F3DB6D1C65459ADB05B0BDE8F08F17
:10BF00002DE9F041C2F1100742B1012B06D0AF4B31
:10BF10001C78A64B012C05D000244DE0BDE8F04173
:10BF2000F7F79BBA002518E000240FE0367D05FBEB
:10BF30000646641C31F916C030F916E00CFB02FC11
:10BF40000EFB07CC4CF30F1C21F816C01E6896F8A8
:10BF500062C7B4EBDC0FE9DD6D1C1C68647D641CFA
:10BF6000AC42E1DA00200127994D11E092F86227F6
:10BF700007EBD20207E000BF00FB0424521C35F897
:10BF8000146021F814601C68247D9442F4DC401C89
:10BF90001A68547D641C8442E8DABDE8F08100BF71
:10BFA00031F9145030F91460554306FB075545F339
:10BFB0000F1521F81450641C1E68757D367D6D1CAC
:10BFC0007543A542ECDCE8E7F0B5784D00278446E0
:10BFD0002D6801203C466E7D2D7D06F1010606FB95
:10BFE00005F60BE03CF9145031F914E0B5EB0E0501
:10BFF00000D56D429D4200DD7F1C641CA642F1DC31
:10C00000974200DD0020F0BD2DE9F04389466F49DD
:10C0100000252C460A786549012A0B6806D0B3F83A
:10C0200053675A7D197D521C4A4312E0B3F8596791
:10C03000F7E700BF39F9117030F911C007EB0608B6
:10C04000C44505DDBCEB070700D57F423D44641CB9
:10C05000491C8A42EEDC544865B193F83610A1427F
:10C0600008D2C16811B10120BDE8F0830121C1608F
:10C070000020F9E70021FAE72DE9F047824653480E
:10C080004A4C8946017800260125206890460129FE
:10C0900036D090F8371000BF01F00F0190F8200063
:10C0A00001EB81014FEA4107000720D54A48494A80
:10C0B00001685046F7F7B0F84848464902680B68EF
:10C0C000D1F804C0D21A4368A3EB0C031A44836866
:10C0D000D1F808C0C068C968A3EB0C03401A2168F6
:10C0E0001A441044B1F87810814200DA0025206823
:10C0F00090F8200080070FD53948007818B10BE080
:10C1000090F85B17C8E72048007828B949465046A0
:10C11000FFF77AFF00B100252348002142789AB149
:10C1200088F800108268521C8260236893F83730C8
:10C130001B0903EB8303B2EB430F02DD8160417007
:10C1400001263046BDE8F0871DB1816088F80050B7
:10C15000F7E78268531C8360BA42F7DD0122427020
:10C160008160226892F837201209EFD141700126D0
:10C17000ECE7F0B5012464250C484DE06828100078
:10C18000482A100067281000662810006228100056
:10C19000702810006D2810006F2810006E28100005
:10C1A0006B2810006C2810001C2A10004C2810006E
:10C1B0004C2A10004E2A1000502A1000522A10005B
:10C1C000542A1000562A10004A2A1000A6281000EF
:10C1D00042000120743710008428100064371000DA
:10C1E00074281000377D674331F9176006FB02FCA5
:10C1F0009CFBF5FE764421F817600668367D04FB4B
:10C20000066601EB4607641C37F9026D06FB02FC6B
:10C210009CFBF5FC66443E800668777D7F1CA74248
:10C22000E0DC002218E0A61831F9164004FB03F701
:10C2300097FBF5F73C4421F816400468667D247DA1
:10C2400006FB0426521C31F9164004FB03F797FB4A
:10C25000F5F73C4421F816400468247D9442E2DC62
:10C26000F0BD70B5F94B1B685C7D1B7D641C5C43A5
:10C2700008E000BF32F8135030F81360AD1B21F80E
:10C2800013505B1CA342F5DB70BD2DE9F05FEF4856
:10C29000EF4B01681B78B1F9A120B1F96200012BC5
:10C2A0000AD0B1F9C631EB4C2578E84C012D246851
:10C2B00094F8C0A103D012E0B1F96437F3E7E64C7B
:10C2C000246864B1B1F96C00B1F99E205FEA8A7408
:10C2D00005D5E24C2478012C01D1B1F96A00E04C7B
:10C2E0002478012C2ED0022C06D3B1F8BE200AB13E
:10C2F000B1F9BE0002461346DFF868E3DA4C0546A2
:10C30000AEF800202080D94CDFF868C3DFF868B3AE
:10C31000238091F864601C46801B06B291F8A3004C
:10C32000101A07B291F8C301181AD14B00B2814616
:10C330001F80ACF80060ABF80000D04800780128FE
:10C340000DD03CE091F8BA40224491F8BB4012B2C3
:10C35000204491F8DA4100B223441BB2CCE791F8B3
:10C36000CC004FF0640C00FB05F8B8FBFCF845442A
:10C37000DFF8F482A8F8005000FB02F8B8FBFCF8E4
:10C3800000FB04F5B5FBFCF54244AEF80020B74ACB
:10C390002C44148000FB06F4B4FBFCF4B54A34448E
:10C3A000148000FB07F2B2FBFCF200FB09F0B0FBCB
:10C3B000FCF43A441A8004EB0900ABF8000091F851
:10C3C000A000C00706D1A8480188AA48AEF800100E
:10C3D000008818805FEACA7002D09F48006830B9B0
:10C3E000A248BEF8001001801988ABF80010A148DF
:10C3F000BBF90020B0F90010B3F90000F6F757FDC3
:10C400009F490880BDE8F09F904A10B51268537D9F
:10C41000127D5B1C534306E030F912408C4201DD73
:10C42000012010BD521C9A42F6DB002010BD2DE900
:10C43000F047804693488946002400684FF4AA617B
:10C44000054602F0BAFE814A1068037D01200646C7
:10C4500016E000BF00EB001105EB4107012108E0E9
:10C4600039F913C05B1CC44502DD641C7E54A4B2C0
:10C47000491CD2F800C09CF814C08C45F0DA401C6E
:10C480001168497D8142E5DA20465BE6F0B56F4EE2
:10C4900033685D7D1B7D6D1C5D430024274608E0ED
:10C4A00030F913C0944502DA21F8137000E0641CDF
:10C4B0005B1CAB42F4DB3068B0F89B00A04201DDAE
:10C4C0000020F0BD0120F0BDF0B500255F4C26E056
:10C4D00000220123767D0EE003FB075C30F91CC0CF
:10C4E000BCF1000F04DD0AB1944503DA624601E0B5
:10C4F0000022731C5B1C9E42EEDA002A0EDD012333
:10C5000008E0367D03FB065630F81670BF1A21F896
:10C5100016705B1C2668777D9F42F2DA6D1C2668D8
:10C52000377DAF42D4DCF0BD2DE9F043474B814667
:10C530001868467D057D761C002028E01A6892F870
:10C540005C20642A06D9643A02FB00F494FBF5F4FB
:10C55000141B04E0C2F16402424392FBF5F464341C
:10C5600001224FF064080FE01F683F7D02FB0707C0
:10C5700039F917C0BCF1000F05DD0CFB04FC9CFB76
:10C58000F8FC21F817C0521CB242EDDB401CA84257
:10C59000D4DB69E52DE9F0472C4B81468A461868C3
:10C5A000447D057D641C01202DE01E6896F85D1019
:10C5B000642907D96439421E777D4A4392FBF7F21A
:10C5C0008A1A06E0C1F16401421E5143727D91FB5B
:10C5D000F2F2317D6432414309EB41060AEB410737
:10C5E00000214FF064080BE036F911C0BCF1000FD8
:10C5F00005DD0CFB02FC9CFBF8FC27F811C0491C74
:10C60000A942F1DB401CA042CFDB9BE530B50F48CF
:10C6100040F2FF751C4B00681C4C417D007D491C9D
:10C620004143002205E000BF23F8105024F81020F9
:10C63000401C8842F8DB30BD2DE9F00F0348002391
:10C640001C46066899460121777D3EE04C28100083
:10C65000A6281000682810009C010022482A10001B
:10C66000742810004E2A10004C2A1000502A100086
:10C67000542A1000522A1000562A10007628100062
:10C680004A2A10007C281000EC8E01206C930120B7
:10C690000020DFF8E8A2DFF8E882357D12E000BF75
:10C6A00001FB05023AF912C038F91220BCEB020274
:10C6B00000D5524292B2934203D2134684B21FFA7B
:10C6C00081F9401C8542EBDC491C8F42E0DA44EAE8
:10C6D0000920BDE8F00F590882B20820FDF754B9CF
:10C6E0002DE9F041A74C0546207801282BD1606840
:10C6F00008B9FFF78BFFA448A04BA14E0168487D05
:10C70000097D401C484312E033F9117035F91120BE
:10C71000974200DA3A4623F8112036F9117035F9BC
:10C720001120974200DD3A4626F81120491C81422B
:10C73000EADB6068401C6060642804D3FFF77CFF7C
:10C7400000202070606028E42DE9FE4F06468F48E7
:10C750000027007810B18E49012008708D4C00230D
:10C760005A1E1946E068F3F7B3FFFFF78EFD8B48BA
:10C77000894D8B4902682B783046FFF7C1FB0026B4
:10C780002E7002AA87498648FFF776FC05469DF879
:10C790000800DFF81482DFF814A250B3DFF8E89144
:10C7A000DFF80CB2D9F8000090F8400080070FD5F0
:10C7B0008048BBF90010B0F900207F48B0F90000B4
:10C7C000F6F775FB764A03B276491046FFF71FFB72
:10C7D0007A4D744A72482968FFF743FDE068F3F721
:10C7E0002FFFD9F800004C4690F88110C90711D0EE
:10C7F00017E0E068F3F724FF012D0AD1D8F8001004
:10C80000A80241F00501C8F80010DAF80410F4F7A6
:10C81000FEFBB0E090F89A20296813460846FFF71F
:10C82000A8FC206890F84000400703D52968084616
:10C83000FFF74AFE206890F84000000703D52968FA
:10C840000846FFF7A7FE206890F84000C00603D511
:10C8500029680846FFF768FE2868FFF741FF20684F
:10C8600090F86010490718D52968B0F96820084683
:10C87000FFF70CFE012810D1206890F860008006B8
:10C880000BD5D8F800104FF4806041F00501C8F8CE
:10C890000010DAF80410F4F7BAFB494800780228CF
:10C8A00019D048492868F6F7D8FDDFF81C914548AB
:10C8B000B9F90010FFF7A8FDDFF810C1DFF810810B
:10C8C000444D9CF800108CF8006088F80060E9B1D5
:10C8D00001283BD01CE0206890F840104906E4D5C0
:10C8E0008DF804608DF80560017D491E8DF80610F5
:10C8F000417D491E8DF8071032490091B0F95A2048
:10C90000354901A82B68FEF789FACEE701280ED039
:10C910003249087808B1401E0870206890F8AD20B0
:10C920002F4801788A4225D2491E017023E0BBF9C5
:10C9300000102448FFF768FD8CF800002E80206866
:10C9400090F82901000701D5FCF797FE254801273B
:10C9500088F8007001681B48F6F77FFD1949B9F99E
:10C960000000FFF764FD074948802988814202D210
:10C97000288000E006703846BDE8FE8FEC8E01206E
:10C980006C9301201C2A10004C281000A6281000CF
:10C99000682810002438100062281000342A100083
:10C9A00074A3012042000120502810000C38100010
:10C9B0004C2A1000502A10004E2A10007C2810002B
:10C9C00074281000F4A701204A2A10006D281000D6
:10C9D000702810006028100012F600006728100070
:10C9E0006F28100080281000FE48FF4A006830F8C9
:10C9F000FA1F1180FD49C079C8807047FB480021AB
:10CA0000F84A41808180C160126892F8432012097F
:10CA1000826001610170F648017070472DE9F041B4
:10CA2000F04DF14A2E6896F8D010B6F8FA30C907E2
:10CA300041D096F8FF4004B90124118896F8FEC051
:10CA4000CF1A07FB0CF797FBF4F4B6F8FC700F4411
:10CA50002744E64CB8420EDDE6480026E660416811
:10CA60001020F4F7D4FAE44901200870A680286861
:10CA700090F8010106E0814202D9DD4D2D7825B103
:10CA800096F80101E080BDE8F081DC4D2D78002DA5
:10CA9000F9D1B4F90650002D01DD6D1EE580E48862
:10CAA000002CF0D1891E814200DA01468B4200DD64
:10CAB00019461180E7E71380E5E7F0B5C949CB4E89
:10CAC000096891F84020D20770D0C94A1478CC4A3E
:10CAD0001278ACB1012A09D091F84330B1F84A700C
:10CAE00003F00F021D09B1F8483015E091F84D3000
:10CAF000B1F8547003F00F021D09B1F852300BE089
:10CB0000012A1AD011F8423F03F00F024FEA131521
:10CB10004B888F88A1F1420191F820C15FEACC7C5B
:10CB200016D0DFF8E0C2BCF800C05FEA4C5C0FD55D
:10CB300091F8252154B112090AE011F84C3F03F095
:10CB40000F021D094B888F884C39E5E702F00F0270
:10CB5000984201DCB260F0BDB84201DBB560F0BDC7
:10CB6000B1F95C47B1F95EC7B1F9601744EA0C0E40
:10CB70005EEA010E11D04443444342F210720CFBB2
:10CB800000FC94FBF2F39CFBF2F04FF47A7291FB01
:10CB9000F2F118440844B060F0BDC01AA91A484325
:10CBA000F91A90FBF1F01044F5E7FFE70020F2E7F7
:10CBB00010B58C4A944C002112682478B2F8B43035
:10CBC000012C01D1B2F85637B2F8B840844205D2F0
:10CBD00092F8B040240701D5032110E0B2F8B64026
:10CBE000844205D292F8B040640701D5022106E0E4
:10CBF000984204D992F8B000800700D501217B4803
:10CC00007B4C0378994211D1217899420AD07B4A12
:10CC10001278134307D00169491E0161002901DC24
:10CC20000078207010BD01700169F7E759B1022941
:10CC300001D1012B07D092F8B22002610170002AC5
:10CC4000F0DC217010BD92F8B320F6E76549096861
:10CC500091F8B010CA0665490DD58A88831A002B51
:10CC600009DC664B1B784BB1C2EB0212520002EB9F
:10CC70004000C0F34F10888080B27047C2EB821230
:10CC80001044C0F38F10F6E72DE9F043554E0546EA
:10CC9000A3B03768802197F8B10000F00F04641C3E
:10CCA00002A802F0ACFA97F86004C00714D000277D
:10CCB00010E03168087DB1F96334CDE9003000FB44
:10CCC00007F2B1F9613405EB420002462946FBF751
:10CCD0002EFD7F1CA742ECDB30680023814602A9B1
:10CCE000007D10E000FB03F6002209E006EB020CD9
:10CCF00051F8227035F91CC0674441F82270521C6B
:10CD00009042F3DC5B1CA342ECDB002207E000BF97
:10CD100051F8223093FBF4F341F82230521C904238
:10CD2000F6DC002213462AE000273E460DE000BF55
:10CD300006FB003C51F8238035F91CC0BCEB080C05
:10CD400001D5CCF1000C6744761CA642F0DB97FBC2
:10CD5000F4F699F82071FF070DD02A4F3F887F0520
:10CD600009D599F824714FEA171C0CFB06FC07F053
:10CD70000F069CFBF6F6964200DD32465B1C98429D
:10CD8000D2DCB2F5803F04DB4FF6FF7023B0BDE884
:10CD9000F08390B2FAE710B5FFF776FFFFF756FF82
:10CDA000124C4FF00051020A60804A738873FFF7FB
:10CDB000FFFE6088FFF781FE6088BDE810402DE629
:10CDC000F0B4084A116891F8B130097D03F00F04FE
:10CDD000064B641CDD6895FBF4F604FB16556943AD
:10CDE0000A4D15E04C281000003810002C2A1000C5
:10CDF000742810000C381000A92810006D281000AD
:10CE00006828100088281000A6281000749F0120B0
:10CE100005EB4105002104E030F8116025F81160B0
:10CE2000491C1668367D8E42F6DCD868401CD860F6
:10CE3000A04202DBF0BC0248ADE7F0BC7047000046
:10CE4000749F012031B56846FEF7E1FB954C2078D0
:10CE5000022805D19DF80000012801D100F05FFFF4
:10CE60009DF80000207000F0DBFE38BD10B5FEF725
:10CE700019FEBDE8104000F0C3BE10B5FEF796FFE6
:10CE8000FDF714F800F0A4FEFFF7B8FD8649002076
:10CE900008608649086010BD824900204860ECE7C0
:10CEA00010B50024FFF750FC012801D098B101E033
:10CEB000FFF7C8FF7E480124007850B17D4901206A
:10CEC00008707D48006890F8F002C00701D0FCF7B8
:10CED00023FB204610BDFFF7C9FFFAE72DE9F04715
:10CEE000764F774900263868084273D0724C206824
:10CEF00090F82901800703D572487349008808809B
:10CF0000DFF8C8A100235A1E1946DAF81800F3F713
:10CF1000DFFB6449387809790840C0072ED02068C3
:10CF20006B4D4FF0000890F86010C90632D5DFF85D
:10CF3000A49199F80010C9B967490978B1B1B0F85E
:10CF40007D3090F87C2065496548FFF73DF868B969
:10CF5000206890F87F0028706248017841F0010154
:10CF600001706149012089F800000870287898B1A3
:10CF7000401E287059495A48F6F76FFA3868002859
:10CF800002DA3046FCF73FFFDAF81800BDE8F04758
:10CF9000F3F756BB85F800802068454690F8B0004E
:10CFA000C00702D04E48FFF70BFF5048007828B169
:10CFB0000128DFD14E4800780028DBD14D480178A8
:10CFC00009B10570D6E74C494548FFF769FF0646A9
:10CFD000D0E7FFE7BDE8F08710B500210420F3F7A4
:10CFE000F5FF46482F4900684C6844400AD0486025
:10CFF000E00701D0FFF741FF600603D5BDE8104010
:10D00000FEF7CCBE10BD274C00276770FFF7ECFC85
:10D010000126607860B30128FBD140F28510002121
:10D02000F3F7A6FFF4F75CF80546C00706D0002129
:10D030000120F3F7CBFF6770FFF72EFF680705D5D8
:10D0400000210420F3F7C2FFFFF748FF280605D5AB
:10D0500000218020F3F7BAFFFFF7BEFFE805D8D51F
:10D0600000214FF48070F3F7B1FF25480670D0E738
:10D07000022503210020F6F744F800212846F3F7A3
:10D0800077FF03210120F6F73CF8F4F729F8800731
:10D09000BFD5FFF701FF002140F28710F3F796FF9D
:10D0A0006670B6E7402A1000082A10000C2A10000B
:10D0B00066281000922810004C28100088281000C4
:10D0C000030000809C2810009E28100024381000C7
:10D0D0006B281000622810007428100074AC012026
:10D0E000408901206C281000A82810006328100037
:10D0F00064281000A9281000C08D01208C2A10007F
:10D100001C2A1000F948002101704160704710B5D9
:10D11000027F817F531A9B1C042B05D9437FC47F58
:10D120001B1B5B1C022B0FD9F14B1B7873B12AB16F
:10D13000F04A1268127D521E914207D1417FC07F92
:10D14000081A401C022801D8012010BD002010BD83
:10D150002DE9F84F446805462004DFF89CB3000C25
:10D1600015D000220A2790461046012606FA00F143
:10D170000C421CD0C0EBC00101EB410105EB810169
:10D180000C3191F82030012B06D00A2712E0002044
:10D190008BF80000BDE8F88FB1F808C0CB6893FBAE
:10D1A000FCF3934203DD91F807801A460746401CC2
:10D1B0000A28DBDBDFF83CA3DFF830934FF0000CEC
:10D1C000686806FA0CF108420CD0CCEBCC0000EBFE
:10D1D000400005EB80040C3494F82000012802D0B4
:10D1E00006287ED0AEE0022084F82000207948B1E5
:10D1F000BF48007890B3DAF80000674590F8C000A7
:10D2000033D119E0BD480078012808D0BC48007827
:10D210000128DAF800002AD090F8CF0129E0B448BC
:10D2200000780028B748007809D0C0B1DAF80000CB
:10D23000674590F8550718D100F00F0019E030B19C
:10D24000DAF80000674590F85807F5D00DE0DAF8F5
:10D250000000674590F8D001EED006E018E0DAF85B
:10D260000000674590F8D801E6D0000901E090F889
:10D27000D401E0702046FFF74AFF01281ED06178F4
:10D28000D9F8042006FA01F08243C9F8042059E0D5
:10D29000674502D0E179414504D1DAF8000090F801
:10D2A0008200C9E7984800780128DAF8000002D027
:10D2B00090F88200D9E790F8CD00D6E7DAF80000C0
:10D2C000E17890F8830000F00F000844E070617886
:10D2D000D9F8042006FA01F01043C9F8040031E03F
:10D2E000FFE7072084F82000814800780028DAF85A
:10D2F00000003ED090F8C100844A00F00F00E070BA
:10D30000DAF80010127891F8AD30934206D291F815
:10D310008510E27801F00F011144E170DAF8001095
:10D32000626A91F88500B2EB101F0BDD91F8841052
:10D3300001F00F0200F00F01E0780A44824201D9A7
:10D340000844E0700CF1010CBCF10A0FFFF638AF95
:10D350005FF00007686806FA07F108427DD0C7EB66
:10D36000C70000EB400005EB80040C34E07818B1F6
:10D3700058E090F88400BFE794F82000022804D019
:10D38000072830D008284AD04CE0032084F8200039
:10D390009BF80010491C8BF80010207950B9DFF879
:10D3A0005C8198F8000018B94FF48670FCF7A9FA70
:10D3B00088F8006056480078012833D12079022887
:10D3C00030D1DFF8388198F80000012802D10C2014
:10D3D000FCF797FA4F49052008704F49002088F85C
:10D3E000000008701EE0DAF8000090F880000006E7
:10D3F00005D56946204601F0B3F9012809D0092076
:10D4000084F820009BF8000060B1401E8BF80000FB
:10D4100008E02046009900F025FE0820F0E70920EA
:10D4200084F820006178B04606FA01F0D9F80410BB
:10D43000CC4608421AD02046FFF769FEB0B9DAF8A8
:10D440000000E17890F8830000F00F00081A00282F
:10D4500000DC0020E070607800E00BE008FA00F8E3
:10D46000DCF8040020EA0800CCF80400E07808B1F9
:10D47000401EE0707F1C0A2FFFF66CAF8AE6F0B505
:10D4800000211C4C012500BF426805FA01F31A4235
:10D4900021D0C1EBC10202EB420200EB82020C324E
:10D4A00092F82030022B16D1144ED3783678012E04
:10D4B00015D0134E3678012E26682FD096F8CF71EE
:10D4C00096F8826006F00F06BE1B9B1B1BB2002B5A
:10D4D00000DC0023D370491C0A29D5DBF0BD266887
:10D4E00096F8D07107F00F07EAE70000582A1000FD
:10D4F000742810004C2810006628100068281000BE
:10D5000069281000A6281000762810006F28100047
:10D510006D28100067281000482A100096F8D47172
:10D52000CEE7000070472DE9F04F002789B03E4656
:10D530003D463B46C3F10502002900EB820264D060
:10D54000B2F9002017445A4302FB03555B1C1644F2
:10D55000062BEFDBF74C009760680190A068CDE9DF
:10D560000206206904906069CDE90505E06907902D
:10D57000206A08906846F5F7A1FC82462068CDE94C
:10D580000007A0680290E068CDE903066069059095
:10D59000A069CDE90605206A08908B466846F5F734
:10D5A0008DFC8046206800906068CDE90107E06846
:10D5B00003902069CDE90406A0690690E069CDE9F1
:10D5C000070589466846F5F779FC0326A8FB064758
:10D5D0000B4609FB0671002508FB05110925A0FB78
:10D5E000056703FB0573002200FB0230A3194141CC
:10D5F00013EB0A0041EB0B014FF47562002301F0BD
:10D600006BFD09B000B2BDE8F08FB2F9022099E7D6
:10D6100070B5054600243A3021460646FFF783FFE1
:10D6200060F31F4401213046FFF77DFF014620468D
:10D6300061F30F00C5F8420070BDBF490A68B2F837
:10D640002B11814201D300207047B2F82D21824274
:10D6500001D8FF207047521A401AC0EB0020B0FBDF
:10D66000F2F0C0B2704738B5B2F90230B2F900201A
:10D670005B4302FB02340A460146684600F04AFD5D
:10D68000684600F03FFDA04201D9002038BD0120CE
:10D6900038BDF0B5A84C0022236893F887502B07BB
:10D6A00001D12B091DD0B0F93060B1F90230F31A65
:10D6B00000D55B4205F00F07BB4200D90122B0F94B
:10D6C0002E70B1F90030FB1A00D55B42B3EB151F89
:10D6D00001D942F0020232B1012A09D0022A09D04E
:10D6E00009E00020F0BDD0F82E0008600120F0BD58
:10D6F0000F8000E04E80D30715D0B1F90230B0F9A9
:10D700003050AB4207DD256895F8875005F00F05CE
:10D71000A3EB050306E006DA256895F8875005F0C7
:10D720000F052B444B80920712D5B1F90020B0F9B8
:10D730002E309A4205DD236893F88730A2EB13124E
:10D7400005E005DA236893F8873002EB13120A80AC
:10D750000968C0F82E10C4E72DE9F843764E0D464F
:10D76000044690F82010012730684FF00009032983
:10D770000DD0B4F93480002104F13A0C04F12E03E9
:10D78000B8F1000F1EDD90F8982032B10AE090F851
:10D790008900A086A4F8329068E090F89980B8F1EA
:10D7A000000F0BD0ADF8022090F89900ADF8000002
:10D7B0006A4661461846FFF756FF0146A08E401E96
:10D7C000A08626E0B4F93220002A0EDD90F8800011
:10D7D00040071ED529462046FFF75BFF014601287A
:10D7E00017D1608E401E608613E090F8862022B923
:10D7F00090F89780B8F1000F0BD0ADF8022090F8A8
:10D800009700ADF800006A4661461846FFF72BFF07
:10D81000014694F82000052806D0042804D00728E3
:10D820002AD0092828D029E041B1306890F880003A
:10D8300080071FD5D4F82E0028601FE0608E78B9CD
:10D84000B5F90200B4F93010084440106880B5F909
:10D850000000B4F92E100844401028802868A06207
:10D86000A4F83490306890F8880060862868C4F87E
:10D870002E0003E0002701E00129DBD03846BDE897
:10D88000F8832DE9F843044690F8200016460F4629
:10D8900003281CD004F13E02111FDFF8A080264DA2
:10D8A000052816D0082814D0072812D00928E6D158
:10D8B000684600F02FFC684600F024FC014698F80A
:10D8C00000000028286863D0B0F8C40062E008684F
:10D8D0005AE0684600F01EFC684600F013FC8446DF
:10D8E00098F8000048B12B6813F8C20F00F00F0140
:10D8F0005A88000952439B880EE0207998B101288C
:10D90000286814D090F88A002B6800F00F010009F5
:10D9100033F88C2F5B8852435B43944519DD9C455B
:10D920000EDB084615E0286890F8D101ECE790F886
:10D93000AC00E9E7602A10004C28100074281000A1
:10D94000ACEB020C411A0CFB01FC991A9CFBF1F1A7
:10D95000401AA16A3B68C0F11002414303FB021068
:10D960006FF0F02101EA101038602868338890F8D1
:10D970008B0000F00F01A08DC1F11002484303FBA2
:10D980000200000930803868A0623088A08576E700
:10D99000B0F88C0040438142F9DCA06A3860A08D69
:10D9A00030806CE72DE9FC47DFF80CA2DFF80C8231
:10D9B000074600264FF00109786809FA06F5284263
:10D9C0007DD0C6EBC60000EB400007EB80040C34B2
:10D9D00094F82000032807D0052805D0042803D098
:10D9E000082801D009286AD1D4F83A000090A08A0A
:10D9F000ADF80400D8F8000090F88000400603D588
:10DA00002046FFF705FE0090D8F8000090F880004F
:10DA1000000704D501AA69462046FFF732FFD8F86F
:10DA2000000090F88000C00706D001AA6946204691
:10DA3000FFF792FE002842D094F8200003280ED170
:10DA4000D8F8000090F82901410705D4C00706D096
:10DA50005B480078012802D1D4F836000090DAF84B
:10DA60000010584B2943CAF8001022791B78504601
:10DA70001A4305D194F82020092A01D0A943016056
:10DA800006EB46010AEB810594F820002D1D0328C2
:10DA90004FD0052853D0042851D008284FD0042057
:10DAA000B5F90A20BDF902108A4216D1B5F908105D
:10DAB000BDF90020914210D1D8F8001000E059E0E3
:10DAC00091F88010890708D5297901F07F02A178A3
:10DAD000B2EB510F01D1891CA170A17849082971BD
:10DAE0002279032A02D341F0800129710099A960AB
:10DAF00028702078687020796871D8F80000228931
:10DB0000434690F82F010109514300F00F00B1FB8B
:10DB1000F0F0A870E08AFFF790FDA871207EE87110
:10DB20001A68BDF80410B2F89000884209D30020AA
:10DB300013E02146384600F0D5F80320B0E7052071
:10DB4000AEE7B2F892208A4201D83F2005E0121ACF
:10DB5000081AC0EB801090FBF2F0E87094F82000F7
:10DB6000092807D12146384600F0B1F82146384649
:10DB700000F0CBF8761C0A2EFFF61EAFBDE8FC873E
:10DB800070B5114C002305465A1E19466069F2F71C
:10DB90009FFD2846FFF706FF6069F2F751FD064832
:10DBA0000068002806D009480168BDE870400220DE
:10DBB000F3F72DBA70BD0000843710004C28100018
:10DBC000A628100068281000243810000C38100017
:10DBD00010B54FF455715C4801F011FB4FF4F8712A
:10DBE0005A4801F00CFB5A490020087000F0B6F8C2
:10DBF000FFF788FA00F00CFABDE81040FFF792BC7E
:10DC000010B500F0F9F9504800F003FA4E48FFF75C
:10DC10009FFA4D48FFF7B4FF4C490020087010BD33
:10DC200010B54A4C207878B12146474800F020FDD5
:10DC3000454800F094F84448FFF78AFA4248FFF755
:10DC40009FFF0020207010BDBDE81040D8E770B5E0
:10DC50003E4C22780F2A25D23E490978012915D158
:10DC60003D49B0F902300968B1F86657AB4219DB9B
:10DC7000B1F86857AB4215DCB0F90030B1F86A571B
:10DC8000AB420FDBB1F86C178B420BDC02EB42119D
:10DC90000B195B1C014621221846F5F7B9FB2078C9
:10DCA000401C207070BD10B5034600205968012249
:10DCB00002FA00F4214206D0401C40B20A28F7DBE9
:10DCC0004FF0FF3010BD82401143596010BD10B5B8
:10DCD0004C7801234268A3409A434260002081F8B7
:10DCE000200010BD30B500220368012404FA02F5BB
:10DCF0002B4205D0521C0A2AF8DBFF20087030BDE9
:10DD00009440234303600A7030BD10B50C780123A2
:10DD10000268A3409A430260FF20087010BD0A48C1
:10DD2000FFF7ADBB09480A490078087070470A49F7
:10DD3000096891F86110C90705D0024604480178C6
:10DD4000024800F0AFB87047803F1000D442100086
:10DD5000842A1000A62810004C28100070472DE9D6
:10DD6000F041002506460127706807FA05F10842D0
:10DD700036D0C5EBC50000EB400006EB80040C3448
:10DD800094F82000012801D0022829D12079022806
:10DD900003D0012805D0E0B122E0B4F8050097498E
:10DDA0001AE0984996480968B0F9000091F8A01067
:10DDB000890705D5B4F91A000021FDF75CFA00B215
:10DDC000B4F8051081420BDA21463046FFF77FFF99
:10DDD00006E0B4F805008C49B1F900108842F3DB85
:10DDE0006D1C2DB20A2DBFDBBDE8F0812DE9F04797
:10DDF0000446914254D007D901EB0200A0EB020186
:10DE0000CAB2A0EB0200C1B201EB411000EB040169
:10DE100002EB421001F1010100EB0409CB88B9F8D3
:10DE2000075009F101002B44CB808B88B9F80550CD
:10DE30002B448B80CB68D9F80D502B44CB608D6878
:10DE40000B680068D9F809704FEA234C4FEA204864
:10DE500005FB0CFC07FB08CC05EB07069CFBF6FC5E
:10DE60006CF31F430FFA83FC05FB0CF500B207FBB4
:10DE7000005090FBF6F060F30F030B608E6020788B
:10DE8000A0F10101914208D000EB401001192039A6
:10DE900009F101002122F5F7BBFA2078401E20701D
:10DEA000BDE8F0872DE9FC5F074658480C46002581
:10DEB000017854480129006807D090F8730000BF2A
:10DEC00000FB00FA4FF0010990E090F8CB00F7E773
:10DED00009FA04F02646009065E0009A09FA06F077
:10DEE000494610425ED006EB46103844D0F8012077
:10DEF00020464BE0B04248D000EB40133B44D3F8FF
:10DF000001304FEA234CACEB224CA3EB02030FFA97
:10DF10008CFC1BB26CF31F4563F30F059B46394B1A
:10DF2000E6461B6893F861C0CDF804C05FEA8C7CBC
:10DF30000BD593F874800BFB08FC4FF064089CFB36
:10DF4000F8F808EB0B0C6CF30F05DDF804C05FEA82
:10DF50004C7C0AD593F874300EFB03FC64239CFBC5
:10DF6000F3FC0CEB0E0363F31F454FEA254C0CFB4F
:10DF70000CFC2BB203FB03C3534506D2DDF800C0F3
:10DF800001FA00F343EA0C030093401C3B78834200
:10DF9000B0DC04216846F4F76FFF012802D1009835
:10DFA00040000090761C3878B04296DC0421684628
:10DFB000F4F762FF01281DD0009A484600FA04F1E8
:10DFC000114203D03E78C846761E0CE0641CF5E78B
:10DFD000009908FA06F0084204D0F2B2E1B23846DD
:10DFE000FFF704FF761EA642F2DC641C3878A042DC
:10DFF0003FF76EAFBDE8FC9F704700004C2A100051
:10E000004E2A10004C281000502A100076281000CC
:10E0100070472DE9F0410024012605465FF0060710
:10E02000686806FA04F1084217D0C4EBC40000EB9C
:10E03000400005EB80010C3191F82000032806D048
:10E04000042804D0052802D0022803D005E081F876
:10E05000207002E02846FFF73AFE641C0A2CDFD34A
:10E06000BDE8F08110B5052200EB8203521E53F883
:10E07000364F12F0FF025C60F6D1C0F83A1010BDC6
:10E080005FF0000200EB8203521CD2B2C3F83A10D8
:10E09000062AF7D3704730B504464270087D2071D8
:10E0A000C868E06088682061C888208188886081AD
:10E0B000487DA0700D460869E061E88AE082288BFF
:10E0C0002083B5F81F006083A88BA4F80500A87F03
:10E0D000E071A889A082012B07D029682046FFF7AC
:10E0E000C1FF606A401C606230BD012084F82000DE
:10E0F00029682046FFF7C4FF002060622868C4F842
:10E10000360030BDB0F90010B0F90200494300FB01
:10E110000010704710B553884C881B1B4380128831
:10E120000988511A018010BD2DE9FF4F4FF00408F6
:10E130008946526808EBC004411E4FF0060C1D468C
:10E140000CEBC000DDE90D3A14441044B4F9004072
:10E15000B0F9007000E0491E08EBC1001044B0F9AE
:10E160000000A04201D00029F5DA08EBC1001044FC
:10E17000B0F90000A0427DD10CEBC1001044B0F911
:10E180000060491E0CEBC1001044B0F90000B04221
:10E1900001D00029F5DA0CEBC1001044B0F9000001
:10E1A000B0427DD108EBC1001044B0F900C0C4EB0F
:10E1B000C40000EB4000CCEBCC0103EB800001EB92
:10E1C000410103EB810107EB471303EB0A02D0F88F
:10E1D0004600D1F84610D2F8012006EB4613009213
:10E1E00003EB0A024FEA204BD2F8012001920BEB1D
:10E1F00021420FFA80FA09B20AEB01004310BDF97F
:10E200000200BDF90610BDF9048008444010BDF9B4
:10E210000010A0EB620041445844C3EB6101ADF82B
:10E220000E000AEB0100ADF80C006A4603A902A833
:10E23000FFF770FF02A8FFF765FF804601AA03A958
:10E2400002A8FFF767FF02A8FFF75CFF804527D908
:10E25000002000E0401C05EBC001B1F90410A14210
:10E2600001D04845F6D305EBC001B1F90420A24224
:10E2700016D100E014E0CE80002100E0491C05EB3F
:10E28000C102B2F90420624501D04945F6D305EB3D
:10E29000C101B1F90420624504D005EBC000C7807C
:10E2A000BDE8FF8FCF80FBE7F0B5002118E04A1CE6
:10E2B00012E0436803EBC10603EBC2043568236830
:10E2C0009D4208DD6768256075686560446804EBF9
:10E2D000C10423606760521C03689342E9DC491C57
:10E2E00002688A42E3DCF0BD70B5D0E9004506263D
:10E2F00006EBC40635442A800425426805EBC405B4
:10E300002A441180416801EBC401641C0B60046065
:10E3100070BDF0B5B1F90240B2F9025004FB05F648
:10E32000002E2ADDB1F90060B2F900707E43002EA4
:10E3300023DD64435D4394FBF5F424B24480B2F9D9
:10E340000020B1F900105A43494391FBF2F10AB29F
:10E3500078230280782C00DD4380B0F902406FF012
:10E3600077018C4200DA4180782A00DD0380B0F921
:10E3700000208A4200DA0180F0BD00214180FAE7E6
:10E380002DE9FF4FADF27C5D81464FF6FF70CDF871
:10E390000C050020CDF86C050DF21450CDF81C05CD
:10E3A0004830CDF874050020CDF8140502A80024EB
:10E3B0000E460DF5AB6B0DF5AD6AA046CDF8180510
:10E3C000FE480178012903D1CDF86C1500210170B8
:10E3D00000270120D9F80410B84001427DD0C7EBD6
:10E3E000C70000EB4001F64809EB8105DDF86C251C
:10E3F00001680C35012AB1F8940001D1B1F8CE00C2
:10E4000005F13A024043CDF8100591F896C00DF29F
:10E410004C53111D06C30DF5AB60FFF77BFE0DF5E8
:10E42000AB60FFF76FFE0CFB0CFC0CFB00FCDDF897
:10E430001005844502DDCDF820C501E0CDF82005AA
:10E44000E0480178012905D16FF00041CDF8201591
:10E45000002101704FF0000C52E000BF0CEB4C109B
:10E460003044401C01900DF24C5006C80830FFF7B4
:10E4700051FE05F142010DF26450DDF84C25FFF725
:10E4800049FEDDF87405B0F902006430C82806D8EA
:10E49000DDF87405B0F900006430C82801D9012303
:10E4A00000E003230DF25C510DF26452081FFFF7E8
:10E4B00030FFA88FBBF802100844AAF80200688F4A
:10E4C000BBF800100144AAF800100DF5AD610DF580
:10E4D000AB60019AFFF71EFE00E014E00DF5AB60A3
:10E4E000FFF710FEDDF820150346884206DA0FFA22
:10E4F0008CF239B2DDF81C05FFF7F6FE0CF1010CC9
:10E5000030786045AADC7F1C0A2FFFF662AFDDF889
:10E51000140500287ED0DDF81C05FFF7C5FE00219C
:10E520000DF2245E0DF5976B4FF0040A3BE000BF3F
:10E53000DDF818050AEBC1020244B2F900300622E8
:10E5400002EBC10210440122B0F900C0DDF88405DD
:10E55000056802FA03F005421FD1DDF8887502FA5A
:10E560000CF23F68174218D1DDF8847505433D6011
:10E57000DDF888552D681543DDF8882515600BEB0F
:10E58000C402641C9380A2F806C0DDF80C2510427A
:10E5900003D14EF8281008F10108DDF80C2582435C
:10E5A000491CCDF80C25DDF814058842C0DC754601
:10E5B000B8F1000F56D0CDE90096A8F101080DF58D
:10E5C000976355F828002146DDF81C25FFF7ACFDC0
:10E5D000EEE7641E0BEBC401B1F90400B1F90610BB
:10E5E000C0EBC00202EB420309EB83050C3501EBE3
:10E5F0004111314495F82020491C032A03D0042AF4
:10E6000001D0052A17D12A79022A14D10A7D022ABB
:10E6100011D000E028E06C4B8A8BB3F900309A42AD
:10E6200009DADDF884150A6801218140DDF88405E6
:10E630008A43026016E095F9012000232846FFF77F
:10E640002AFD95F82000032806D0042807D00728C3
:10E6500005D0052806D102E085F820A002E00520BB
:10E6600085F82000002CB4D10DF28C5DBDE8F08F50
:10E670002DE9FC41064640680F4650B1002001904C
:10E68000009001AB6A463046FFF77AFE0025012470
:10E690003CE0002415E000BFC4EBC40000EB4000E8
:10E6A00006EB80050C353046FFF7FDFA021E07DB4E
:10E6B00002EB4210C119491C01232846FFF7EBFC6D
:10E6C000641C3878A042E7DCBDE8FC81019904FABB
:10E6D00005F0084219D13046FFF7E5FAB0F1000C19
:10E6E00013DB05EB4510C119CCEBCC0000EB40006F
:10E6F00006EB8000491C0C3001236246FFF7CBFC7F
:10E70000009904FA0CF0084300906D1C3878A84278
:10E71000DCDC00255FF00607716804FA05F00142B1
:10E720001AD00099084217D1C5EBC50000EB400094
:10E7300006EB80010C3191F82000032806D0042854
:10E7400004D0052802D0022803D005E081F820700B
:10E7500002E03046FFF7BBFA6D1C0A2DDCDBB3E7A5
:10E760002DE9F84300F13A020D4604469146111D89
:10E770006846FFF7CFFC6846FFF7C4FC0746BDF8C4
:10E78000020010B90120ADF80200BDF900004FF4FD
:10E790007A714843BDF90210A28F90FBF1F0114449
:10E7A0000AB26A80618FBDF80030054E1944298095
:10E7B00033684FF47A7CB3F8188007E0A82810007B
:10E7C0004C2810006C281000522A100000214245ED
:10E7D00006DDB3F918206A80B4F93C30D21A05E09E
:10E7E000002A09DA6980B4F93C205242424392FB84
:10E7F000FCF2638F1A442A803368B5F90020B3F81D
:10E8000016C0624506DDB3F916102980B4F93A2026
:10E81000891A05E0002A0BDA2980B4F93A10494236
:10E820004FF47A72514391FBF0F0A18F0844688055
:10E830004A4629466846FFF76DFC6846FFF762FCCA
:10E840003168642391F852277A43B2FBF3F2BA1A83
:10E85000904216D9B5F9022091F8510782420DDD98
:10E860000B8B181A904209DDB5F9002091F850077A
:10E87000824203DDC98A081A904202DC0120BDE809
:10E88000F8830020FBE7000012490868124A10686C
:10E8900000280CD14FF4FA7300BF401C9842FBD300
:10E8A0000860106820B1086820F004000860704714
:10E8B00030BF7047094810B50168491C016008481D
:10E8C000006820B10120F4F73CFE30BF10BDBDE868
:10E8D0001040D9E710ED00E0AC1A0120A02810008C
:10E8E00084010022F9490020486088600860F849E6
:10E8F000086070472DE9F0474FF00857D7F88401BA
:10E9000000286DD105210120F4F7FBFBEF4D4FF0FE
:10E910000009DFF8C083C5F80490C5F80890EE4CF4
:10E92000C5F80090C8F8009002206168F2F76FFB0C
:10E930000220E168F2F76BFB08202168F2F767FB21
:10E9400002202169F2F763FBE44E306890F8290158
:10E95000800702D50120FAF7FAFDFAF7FFFE3068CA
:10E9600090F88003000703D520206168F2F74FFB81
:10E97000306890F8511109072FD590F85001C00761
:10E980002BD06868410728D4D54A1E2140F00400E6
:10E990001180D4490A6842F020020A606860D8F801
:10E9A0000010D14841F022010125C8F8001005707F
:10E9B000A8026168F2F72BFB0420A168F2F727FB9D
:10E9C00010202169F2F723FBC7F89051C0494FF698
:10E9D000E850C1F80090F2F771FC0120C7F88401FB
:10E9E000BDE8F08770B54FF00856D6F884010028CE
:10E9F00031D0BA48006890F82901800701D5FAF7AC
:10EA0000A9FDB4480025B44C056001206168F2F707
:10EA1000FEFAAE4845600420A168F2F7F8FA10202B
:10EA20002169F2F7F4FA8020E168F2F7F0FA0120A8
:10EA3000E168F2F7ECFA04202168F2F7E8FA012025
:10EA40002169F2F7E4FAC6F88451BDE87040052167
:10EA50000020F4F756BB70BD70B59C4D6A68D007B6
:10EA60002BD19C48A14B016841F0050101601C6855
:10EA700044F020041C60994B1B6893F8B031DB070D
:10EA800005D012F40B7F02D141F04201016096489B
:10EA90000126914C0670B0026168F2F7B8FA686816
:10EAA00040F0010068600420A168F2F7B0FA80200D
:10EAB000E168F2F7ACFA8E4806608E4900200870D3
:10EAC00070BD824810B50079C00701D1FFF7C4FFBF
:10EAD00088490120087010BD7C4910B54868C207FC
:10EAE0000ED020F001007C4C48600420A168F2F7B1
:10EAF0008EFA8020E168F2F78AFA7D4900200860EA
:10EB000010BD764810B5006890F8C001C00712D05B
:10EB10006E49486842060ED5774B002220F040002F
:10EB20001A706D4C48600420A168F2F770FA8020DA
:10EB3000E168F2F76CFA6E4900201031086010BDF0
:10EB4000664810B5006890F86207C00707D06B4CA4
:10EB50002078012803D1FFF7D4FF0020207010BDDA
:10EB60005E4810B5006890F8C001C00716D0624931
:10EB7000002008705549486842060FD440F0400014
:10EB8000554C48600420A168F2F741FA8020E16802
:10EB9000F2F73DFA564901201031086010BD4F4888
:10EBA00010B5006890F86207C00707D0534C207872
:10EBB000002803D1FFF7D4FF0120207010BD10B54D
:10EBC0004FF00854D4F88401002807D042488168E7
:10EBD0000820F2F71CFA0120C4F8880110BD10B516
:10EBE0004FF00854D4F88401002807D03A488168CF
:10EBF0001020F2F70CFA0020C4F8880110BDF2F7DB
:10EC00001FBC364810B5006890F85001C00711D0FD
:10EC10002E480021016041684A070BD521F004010C
:10EC20002D4C41600420A168F2F7F1F91020216910
:10EC3000F2F7EDF92E490020091D086010BD70B5EE
:10EC4000264D286890F85001C0073DD01F48426803
:10EC5000510730D42A490B78014689682BB141F01D
:10EC6000040181600521016025E01D4C1E2342F056
:10EC7000040223801B4B21F0040101261C6844F090
:10EC800020041C60C0E901211248134C016841F0C6
:10EC90002201016014480670B0026168F2F7B7F90A
:10ECA0000420A168F2F7B3F910202169F2F7AFF957
:10ECB0000F48001D0660286890F85101000703D531
:10ECC000BDE87040F2F708BB70BD0000882A100054
:10ECD00098281000502810000C3810004C28100004
:10ECE000902810005C2810005428100058281000AC
:10ECF0008C0100226A28100069281000A628100044
:10ED0000662810007047704770477047704770471B
:10ED1000724810B5006890F8C001C00715D070495E
:10ED2000012008706F49486842060ED440F0400048
:10ED30006D4C48600420A168F2F769F98020E16811
:10ED4000F2F765F969490120086010BDF2F75ABB76
:10ED50006448007900070ED4654840F6BF72016828
:10ED6000114301606349012008705F4841684FF416
:10ED70008060F2F74CB970475F4840F6A2520168D4
:10ED800041F0100101605B4901200870584801689A
:10ED900011430160544841684FF48060F2F737B97D
:10EDA000514841680820F2F732B94F4841680420C1
:10EDB000F2F72DB94C4841681020F2F728B94A48BB
:10EDC00041682020F2F723B9474841684020F2F714
:10EDD0001EB94248006890F8C800C00705D04749EE
:10EDE00001200870CC20FAF78CBD70474349002001
:10EDF0000870CD20FAF785BD70470A46B0F5805FF0
:10EE0000014602DA3548006801E04FF48010FAF755
:10EE1000B6BCF0B54FF40064B0F5805F02D22F4B62
:10EE20001D6803E0A0F580504FF48015002303E037
:10EE3000D65C1F185B1CEE558B4201DAA342F7DB50
:10EE4000F0BD10B5254C40F2FF112068F2F75EF9D5
:10EE500022684FF40071C2F8FC071046F2F7D9FCA3
:10EE6000BDE810400320FAF74CBD10B54FF48014F4
:10EE700040F2FF112046F2F749F921490860C91212
:10EE80002046F2F7D6FCBDE810400420FAF739BD61
:10EE9000FAF7F3BC144881682020F2F7B8B812489A
:10EEA00041684FF48070F2F7B2B80F4841684FF4F0
:10EEB0000070F2F7ACB810B50B4C4FF48070E168FD
:10EEC000F2F7A5F82169BDE810402020F2F79FB8BD
:10EED0000448007A400700D5B1E670474C2810007E
:10EEE00069281000882A10000C3810009C010022AC
:10EEF00050281000542810005C28100076281000BC
:10EF0000FC07100070B504462F480D46202C02DD8A
:10EF10002021016000E0046020212C4800F04DF920
:10EF200000222A4802E0A95C8154521CA242FADB6A
:10EF3000274841690120F2F79BF8002803D0BDE87B
:10EF40007040F1F75FBA70BD032804DD0888897846
:10EF500040BAFFF752BF7047032806DDC31E08887A
:10EF60008A1C40BA1946FFF754BF70471749164824
:10EF70000B780068A3F190021F2A03D8154850F8B7
:10EF800022000047B02B07D0B22B07D0FB2B07D0B5
:10EF9000FC2B07D1FFF769BF491CDDE7491CD3E70C
:10EFA000FFF74FBF70470C4910B50868401C086058
:10EFB00042F21071884205D9FFF723FEBDE81040E8
:10EFC000F2F78AB910BD0000942A1000C444100062
:10EFD0000C3810003CF6000098281000FFF782FC67
:10EFE0001148F2F734FAFAF791FB05210020F4F703
:10EFF00088F803200021F1F7BBFFF2F771F804460F
:10F00000C00707D000210120F1F7E0FFFFF7AEFFB6
:10F01000F2F749FAA007ECD500210220F1F7D6FF5C
:10F02000FFF756FFE5E70000E5EE000070B5064685
:10F0300000F03AF9056806F10B0020F00704B4422D
:10F040009CBF002070BD2B466A68BAB11068A04210
:10F0500010D304F1080188423CBF5068586007D3C0
:10F060005168101941601168091B016058601460F3
:10F07000101D70BD13465268002AE7D1214628466C
:10F0800000F01AF90028DED170BD70B50446051FE6
:10F0900000F00AF90068002C14BF446870BD002C11
:10F0A00018BFA54284BF20466468F8D801680A18D2
:10F0B000AA4218BF456003D12A6805461144016081
:10F0C00028684119A1421CBF6C6070BD616869600D
:10F0D00021680844286070BD10B54C1084EA5304C0
:10F0E00004D54042C1F1000138BF491E1B4204D57E
:10F0F0005242C3F1000338BF5B1E00F027F914F041
:10F10000804F04D04042C1F1000138BF491E14F0C5
:10F11000004F04D05242C3F1000338BF5B1E10BD44
:10F12000032A40F2308010F0030C00F0158011F833
:10F13000013BBCF1020F624498BF11F801CB00F80B
:10F14000013B38BF11F8013BA2F1040298BF00F85F
:10F1500001CB38BF00F8013B11F0030300F06D81D3
:10F16000083AC0F0088051F8043B083A51F804CB43
:10F17000A0E80810F5E7121D5CBF51F8043B40F809
:10F18000043BAFF30080D20724BF11F8013B11F814
:10F1900001CB48BF11F8012B24BF00F8013B00F858
:10F1A00001CB48BF00F8012B704702F0FF0343EA90
:10F1B000032242EA024200F002B84FF000020429A2
:10F1C000C0F0128010F0030C00F01B80CCF1040C96
:10F1D000BCF1020F18BF00F8012BA8BF20F8022BCA
:10F1E000A1EB0C0100F00DB85FEAC17C24BF00F870
:10F1F000012B00F8012B48BF00F8012B70474FF09E
:10F20000000200B5134694469646203922BFA0E876
:10F210000C50A0E80C50B1F12001BFF4F7AF090782
:10F2200028BFA0E80C5048BF0CC05DF804EB890073
:10F2300028BF40F8042B08BF704748BF20F8022BB6
:10F2400011F0804F18BF00F8012B704710B504462D
:10F2500010F0030F08BF11F0030F40F015804FF0BE
:10F26000013E121FC0F20E8051F8043BA3EB0E0CBE
:10F270002CEA030C1CEACE1C08BF40F8043BF0D07B
:10F28000A1F1040102F10402521E08DB11F8013B56
:10F29000002B00F8013BF7D11146FFF78EFF204607
:10F2A00010BD70477047704700487047EC4410002D
:10F2B000704770477047704738B504460A460020CB
:10F2C0006946AFF30080002808BF38BD02460099A8
:10F2D000204600F0E4F8012038BD012000F0F9B824
:10F2E000F8B5AFF30080054600200C46102000BFA3
:10F2F0000646A819A0420DD9324669460020AFF350
:10F300000080070008BF00F0E4F80098A04218BF92
:10F310000546C419FFF7C8FF05600746F01D20F039
:10F3200007004619284600F00AF8B44208BFF8BDA5
:10F33000A21B31463868BDE8F84000F0B0B80021A3
:10F340000160C0E9011070471020704753EA020CB9
:10F3500000F069802DE9F04B4FF00006002B1FBF35
:10F36000B3FA83F503FA05F424FA05F65E4012BFFA
:10F370001643B2FA82F502FA05F4C5F120051EBF64
:10F3800022FA05FC44EA0C04203556EA044C4FEA04
:10F39000144418BF641C4FF000084FF0000990425D
:10F3A00071EB030C39D3002919BFB1FA81F701FAC7
:10F3B00007F6B0FA80F700FA07F6C7F120071EBF7C
:10F3C00020FA07FC46EA0C062037B6FBF4FCA7EB54
:10F3D0000507103F07F01F0BCBF120060CFA0BFBC3
:10F3E0002CFA06F644BFB3460026202FA4BF5E4683
:10F3F0004FF0000B5BEA060C08BF4FF0010B19EB56
:10F400000B09ABFB027C48EB0608C01B06FB02CCD9
:10F410000BFB03CC71EB0C01C1E70B4602464146E6
:10F420004846BDE8F08B13B54FF000004FF00001E7
:10F43000AFF30080BDE81C40704710B5203AC0F023
:10F440000B80B1E81850203AA0E81850B1E81850E5
:10F45000A0E81850BFF4F5AF5FEA027C24BFB1E822
:10F460001850A0E8185044BF18C918C0BDE8104093
:10F470005FEA827C24BF51F8043B40F8043B08BF9C
:10F480007047D20728BF31F8023B48BF11F8012B63
:10F4900028BF20F8023B48BF00F8012B7047034605
:10F4A00040688C46002818BF814284BF03464068EC
:10F4B000F8D818681844884207D00CF1030020F0EF
:10F4C0000700001D411A521A0146081D0A60FFF785
:10F4D000DCBD10B500F010F8BDE8104000F007B832
:10F4E00070470446AFF300802046F0F76BFE00281B
:10F4F00001D000F029B8704710B5012805D00021CF
:10F5000003A000F027F8012010BD09A1F8E70000D2
:10F5100053494752544D454D3A204F7574206F66FC
:10F520002068656170206D656D6F72790000000064
:10F530003A2048656170206D656D6F727920636F48
:10F54000727275707465640001491820ABBEFEE7E5
:10F550002600020070B505460C460A2000E06D1C2E
:10F5600000F011F835B128780028F8D102E0641CC9
:10F5700000F009F814B120780028F8D1BDE87040F7
:10F580000A20AFF3008008B569468DF8000003201B
:10F59000ABBE08BDB71D0000D11D0000E91D000075
:10F5A000011E00001D1E0000351E00004D1E000043
:10F5B000631E000000000000B71D0000BB1D00001E
:10F5C000011E0000351E00004D1E00001D1E000023
:10F5D000D11D0000E91D0000631E000000010102B2
:10F5E0000102020301020203020303045AD3D9E910
:10F5F0006CF145F59FF73CF96CFA58FB18FCB9FC27
:10F6000044FDBFFD2EFE94FEF4FE50FFA9FF000056
:10F610005700B0000C016C01D2014102BC0247034B
:10F62000E803A8049405C4066108BB0A940E2716D3
:10F63000A62C0100020001000200040002000100EB
:10F64000020001001000FFFFFFFFFFFFFFFF14009B
:10F65000FFFFFFFFFFFFFFFF0C000000C5E90000F8
:10F66000D5E80000D9ED000039EA0000E3EB000026
:10F670001FEC000021EB00007FEB00009FEB00007F
:10F68000BFEB0000EDEC0000EFEC0000A3EA00008F
:10F69000F1EC0000E3EA000041EB0000DFEB0000CA
:10F6A0002DED000031ED000081ED00008BED00003C
:10F6B00095ED00009FED0000A9ED0000B3ED000006
:10F6C00059ED000071EE0000CDED000097EE000056
:10F6D00075EE00007FEE00008BEE0000DCF600000F
:10F6E00000281000980200000001000014F700003C
:10F6F000982A1000AC1A00005C0100001AAA01014F
:10F700002C1AFF0101125305FA0214F802FD01162A
:10F71000FFFFFEFF0A25FEFFFFFF12011A02040190
:10F720001E3206320F9A37089AE10803AED3030956
:10F7300036D00000000000000000000000000000C3
:10F7400000000000000000000000000000000000B9
:10F7500000000000000000000000000000000000A9
:10F760000000000000000000000000000000000099
:10F770000000000000000000000000000000000089
:10F780000000000000000000000000000000000079
:10F790000000000000000000000000000000000069
:10F7A0000000000000000000000000000000000059
:10F7B0000000000000000000000000000000000049
:10F7C0000000000000000000000000000000000039
:10F7D0000000000000000000000000000000000029
:10F7E0000000000000000000000000000000000019
:10F7F0000000000000000000000000000000000009
:10F8000000000000000000000000000000000000F8
:10F81000000000000000000000000000626AEA2D05
:10F82000A5972600FFFFFF3F00000000FFFF01003B
:10F83000000000001E11FF04CF02010000000000C4
:10F840002B010AEFF540640032000A1255640010E3
:10F850000010001000000003001010000000000065
:10F860005F00A0C60C0025000C008000E4E9080041
:10F87000280008002800000018001800505D000053
:10F880003603FA004000308010005E018001E00184
:10F890003C1828640901000AD000080F0620020362
:10F8A0003F01210A01F104221003A20810004000C8
:10F8B0000000000880000A040D0D0A980130F800CD
:10F8C000079000200006040240006400A20320000C
:10F8D000138F0220180020010000003000002003D8
:10F8E0004302B40008003000012030701040800155
:10F8F00001040D000E000F001100120000000000B6
:10F9000000000000000000000000000000000000F7
:10F910000000FF010000000000000A0012000301C7
:10F9200001400000000000000000004126172300F5
:10F93000003218020F0510000F0407100E0B000014
:10F94000010312105A44100000410000005000FA58
:10F950006600AC0DB80B000C000C000C000C005E37
:10F960002BF0003200800C800C040000010000002D
:10F97000FB3F70006400101010003000C920100020
:10F98000FF01230000000010F040000008005001BB
:10F99000D7000604B4C018006000108000000010FA
:10F9A00050001E0100000190010412283060600028
:10F9B000E81028283C350030000100018000C0001C
:10F9C00001100030300806D91000300080005001CE
:10F9D000008000640080000308C8001020010000BF
:10F9E00051000020080050000A00010400021E031C
:10F9F00011D24000010000008402100000203220DB
:10FA0000FFFFFFFF00008022001F11121300000003
:10FA100002000200020000000008000000000000D8
:10FA200000220000000000000000000000000000B4
:10FA300000000000000000080000000000000000BE
:10FA40000000B400B40000002000C8000202000062
:10FA5000030303020203F000803E55002000000172
:10FA6000B408FF01FF01FF01FF014000000000009A
:10FA70000000002000000100000000000000000065
:10FA80001F500050004332430F14AA08000000002A
:10FA900028565A5C5E606264646462605E5C5A56BA
:10FAA0002864646464646464646464646464646452
:10FAB000646464646464E000000402020000000006
:10FAC000585A5C5E60626464646464646464646420
:10FAD000646464646464646462605E5C5A58646410
:10FAE00064646464646464646464646464646464D6
:10FAF000646464646464646464646464E000000076
:10FB000005DF000E800080000010000410070B00CD
:10FB10000101000000000000FFFFFFFF00000000E7
:10FB200000000000000000000000000000000000D5
:10FB300000000000000000000000000000000000C5
:10FB400000000000000000000000000000000000B5
:10FB500000000000000000000000000000000000A5
:10FB60000000000000000000000000000000000095
:10FB70000000000000000000000000000000000085
:10FB8000FAB2B240202828E0A2A240203C003C006B
:10FB90003C003C002020202020B2B240202807005A
:10FBA0008802F6000801180118010000000000009A
:10FBB0000000000000000000000000000000000045
:10FBC0000000000000000000000010001000030111
:10FBD00001FFF600080118011801050000000000EF
:10FBE000000000000000000021082042000000008A
:10FBF0003307E901BF00570028000A000A000A0085
:10FC00000A000A000A000A0028005700BF00E901A4
:10FC100033070000000000000000000000000000AA
:10FC200000000000000000000000000000000000D4
:10FC300000000000000000000000000000000000C4
:10FC400000000000000000000000008000800004B0
:10FC50000000000002000102030001020300000096
:10FC60000017A001090000000007C409100E100EC3
:10FC7000100EFC089808C05DC05D10272823000006
:10FC80000180008000000000000000000000000073
:10FC90001018000008001500360051007200920094
:10FCA000AF00CE004B01C6014402B7023403B103DA
:10FCB0002C044C046A048A04A604C604E604F8046E
:10FCC000FF04000002001200400062008200A20057
:10FCD000C100DF005601CD014402B7022E03A80384
:10FCE00020043A04590479049B04BC04DB04FF0497
:10FCF000FF040000070015003C0064008B00B0000A
:10FD000027019E01100237025F028702AE02C8027D
:10FD1000CF0200000200120043006A009800B90000
:10FD20002B019D01100232025C028A02AE02CF0258
:10FD3000CF020000000000000000000000000000F2
:10FD400000000000000000000000000000000000B3
:10FD500000000000000000000000000000000000A3
:10FD60000000000000000000000000000000000093
:10FD70000000000000000000000000000000000083
:10FD80000000000000000000000000000000000073
:10FD90000A0900001000300040018002C003C004C6
:10FDA000F004FF0400001000300048018002B0039E
:10FDB000B004D004FF0400003000F0006801F4013A
:10FDC00058028002A802BC02CF02000030000401E9
:10FDD0006801F40158028A02A802BC02CF020000A6
:10FDE0000000000000000000000000000000000013
:10FDF0000000000000000000000000000000000003
:10FE000000000000000000000000000000000000F2
:10FE100000000000000000000000000000000000E2
:10FE200000000000000000000000000000000000D2
:10FE300000000000000000000000000000000000C2
:10FE400000000000000000000000000000000000B2
:10FE500000000000000000000000000000000000A2
:10FE60000000000000000000000000000000000092
:10FE70000000000000000000000000000000000082
:10FE80000000000000000000000000000000000072
:10FE90001018000008001500360051007200920092
:10FEA000AF00CE004B01C6014402B7023403B103D8
:10FEB0002C044C046A048A04A604C604E604F8046C
:10FEC000FF04000002001200400062008200A20055
:10FED000C100DF005601CD014402B7022E03A80382
:10FEE00020043A04590479049B04C504F204FF0475
:10FEF000FF040000070015003C0064008B00B00008
:10FF000027019E01100237025F028702AE02C8027B
:10FF1000CF0200000200120043006A009800B900FE
:10FF20002B019D01100232025C028A02C002CF0244
:10FF3000CF020000000000000000000000000000F0
:10FF400000000000000000000000000000000000B1
:10FF500000000000000000000000000000000000A1
:10FF60000000000000000000000000000000000091
:10FF7000646432600133200022640001000000004C
:10FF80000000910341002800A70200006802500011
:10FF900001020404001E00000000098C040400009B
:10FFA00000000000000000F602530388000000007B
:10FFB0000000000000000000007220000F001A0086
:10FFC0000801A600000801A60000EA409300820391
:10FFD000820300000200009817000000600000107B
:10FFE00000000000000000000008200000010000E8
:10FFF0000000000000000000000000000000000001
:020000021000EC
:100000006284010000000000000000000000000009
:100010000000000000000000000000226ADEAA21AB
:00000001FF
